:020000040000FA
:060800005EEF60F0120043
:06080800AEEF47F0120004
:06082A000E00E6C1000013
:100830006B0400000F000000E4C10000D4040000BD
:1008400002000000E2C10000D2040000020000002B
:10085000DEC10000C004000004000000DBC1000095
:10086000C704000003000000A2C100004102000014
:100870003900000051C10000680D00005100000067
:1008800018C10000C20100003900000016C10000BC
:10089000D00400000200000014C10000CE040000DB
:1008A0000200000010C10000BC04000004000000B1
:1008B00069BE0000FF0D000001000000F8C000004C
:1008C000E802000018000000F6C00000CC040000A0
:0408D0000200000022
:0C08D4000401D36B0A0E0301286F296B8E
:1008E0000301000E266F090E276FFBEC39F00101A2
:1008F000A56BA66B0101000EA36F090EA46F5C0E21
:10090000CAEC11F0116E106A10C0E6FFE66E5B0EC5
:10091000CAEC11F0E552E7CF11F0E552E7CF10F045
:1009200001011010A16F11C0A2F1CCEC2CF0040158
:10093000D26F106E116A126A136AE868101805E126
:10094000115003E1125001E1135012000901016B33
:10095000026B0401D35124E103019E6BD2C4AEF1BA
:1009600047EC2EF0000901E15FD1620ECAEC11F0F4
:10097000010B03E1B4EC2EF053D10401010ED36F4F
:10098000620ECAEC11F0020B04E00301010E9F6F2E
:1009900002D003019F6B0901056B466B456B40D18B
:1009A000D30519E103019EA305D0B4EC2EF0040198
:1009B000D36B3AD19EB10DD09E6B0101000EB06F8A
:1009C000090EB16F66EC2EF0000913E103019E835E
:1009D00010D09E910ED0030ED35D04E1D35101E0FF
:1009E00023D122D1020ED35D04E1D35101E11CD108
:1009F0001BD103019F51080A01E1DED00F0A01E17A
:100A0000C2D0010A01E1ABD0030A01E1A4D0010A7E
:100A100001E184D0070A6BE0010A4EE0030A0FE00F
:100A2000010A01E0FDD0250E0901005D03E103018B
:100A3000050EA7D00301020E9F6F9E81F1D0200EFC
:100A40000901005D2CE10551CFEC11F0EF6A350E84
:100A500003011F6F206B0301060E1D6F090E1E6F31
:100A6000ABEC39F0000913E13E0E03011F6F206B60
:100A70000901465103011D6F1E6B060E1D27090E4D
:100A80001E23ABEC39F0000902E103019F6B030167
:100A90009F5101E0C4D00901056B466BC1D03A0EED
:100AA000005D03E1006B0529466FDCEC11F001E30A
:100AB000B7D00FEC12F0B4D03D0E0901005D14E187
:100AC000006B0301030E9F6F09010529106E116A67
:100AD000400E105C000E11580AE20529466F0529E8
:100AE000CFEC11F0EF6A03D0200E005D31E003017E
:100AF0009E51020B04E1260E0901005D05E1030190
:100B0000040E9F6F0901006BDCEC11F002E20FECA8
:100B100012F0040E03019F5D01E082D00301010E7B
:100B2000A46F090146510301A26FA36B060EA22711
:100B3000090EA3230301060EA06F090EA16FC2D8F0
:100B4000F35009010113F450021303019F6B0901D3
:100B5000466B056B65D000C948F9060E12D0610ED0
:100B60000901005D02E3270E04D0410E005D02E39F
:100B7000070E005F300E005D100DF3CF47F9030143
:100B8000070E9F6F4DD0610E0901005D02E3270E35
:100B900004D0410E005D02E3070E005F300E005DE1
:100BA0004713000E4B6F090E4C6F010E4D6F496BD2
:100BB0004A6B0301080E9F6F9E81D2C4A8F12CECF2
:100BC0002DF000092AE00301470EA56F090EA66F5C
:100BD000C9EC0DF0F3CF03F9F4CF04F90901000ECD
:100BE000D880F354000EF45404E200C9A9F138ECA3
:100BF0002DF049C910F04AC911F0126A136AE86869
:100C00001018E1E1E8681118DEE11250DCE1135040
:100C1000DAE1DEEC2DF0030102D003019F6B9E832D
:100C20000401D35101E095D609010151021149E0B7
:100C300001C910F0020E03EC12F001E0120001C92C
:100C400010F0040E03EC12F004E0E2EC3DF036EF9D
:100C50003EF001C910F0080E03EC12F002E08AEF3A
:100C60003EF001C910F0100E03EC12F002E0CDEFDF
:100C70003EF002C911F0106A010E111686EC11F057
:100C800002E0C7EF3FF002C911F0106A200E111602
:100C900086EC11F002E001EF40F002C911F0106A99
:100CA000080E111686EC11F002E0D2EF42F002C9F4
:100CB00011F0106A100E111686EC11F002E05BECD8
:100CC00043F0120009014F6B506BA0C3E9FFA1C3B1
:100CD000EAFFEF506B0808E0A0C3E9FFA1C3EAFFF9
:100CE000EF50750801E0EAD10901010E516F0901C9
:100CF000746B756B0301730E116F090E126F010E89
:100D00000301A02503010F6F000E0301A1210301C0
:100D1000106F18EC39F0000904E1F36AF46AC8EFC7
:100D20000DF0A0C3E9FFA1C3EAFFEF5075080CE185
:100D3000090173510901746F756B000E0901742765
:100D4000010E0901752305D0090173510901746F62
:100D5000756B030E0301EA6AA025E96EA151EA2230
:100D6000EF5062082CE1040E0301EA6AA025E96E47
:100D7000A151EA22EF50D00F106E010E105204E084
:100D8000E846FE0B1006FCE10901776F74C9DBF23F
:100D900075C9DCF2A7EC3DF00901766FA2C3E9FF4B
:100DA000A3C3EAFFEF50300805E10901771D0901EF
:100DB000761704D0090177510901761363D0A2C3D5
:100DC000E9FFA3C3EAFFEF50480818E10301760EDC
:100DD000116F090E126F010E0301A22503010F6F9F
:100DE000000E0301A3210301106F18EC39F0000974
:100DF00004E1F36AF46AC8EF0DF00AD0A2C3E6FF7B
:100E0000A3C3E6FFF4EC56F0E552E552F3CF76F9D2
:100E1000030E0301EA6AA025E96EA151EA22EF5010
:100E20006D0830E10301770E116F090E126F040E89
:100E30000301A02503010F6F000E0301A12103018F
:100E4000106F18EC39F0000904E1F36AF46AC8EF96
:100E50000DF00901771D106E10C0E6FF74C9DBF2BA
:100E600075C9DCF2A7EC3DF0E552E7CF10F01014A5
:100E70000901786F09017651090177150901781187
:100E80000901766F0901110ED8807455000E755551
:100E900006E20901160E741901E1755105E1090117
:100EA0004F830901516BF3D00901150ED880745599
:100EB000000E75550BE30901130E741901E175510C
:100EC00004E009014F8F0901516BE1D009011A0EAD
:100ED000D8807455000E755501E3D9D009011E0E56
:100EE000D8807455000E755501E3D1D00901220E4A
:100EF000D8807455000E75551BE309011F0E741937
:100F000001E1755106E00901210E741901E17551E5
:100F100007E109017651080802E30901516B02D08B
:100F20000901516B0901515102E109014F85AFD00F
:100F30000901300ED8807455000E755521E3870ED7
:100F40000201DB6FDC6BA7EC3DF0020814E1090144
:100F5000250E741901E1755104E1F36AF46AC8EFD2
:100F60000DF00901240E741901E1755104E1F36AD1
:100F7000F46AC8EF0DF009014F870901516B87D062
:100F80000901320ED8807455000E755505E309012C
:100F90004F890901516B7BD009015A0ED8807455D5
:100FA000000E755503E30901516B71D00901620E02
:100FB000D8807455000E755503E30901516B67D055
:100FC00009016F0ED8807455000E755505E30901AF
:100FD00050810901516B5BD00901750ED8807455A1
:100FE000000E755505E3090150830901516B4FD07F
:100FF00009017B0ED8807455000E755505E3090173
:1010000050850901516B43D00901860ED880745573
:10101000000E755503E30901516B39D00901900E9B
:10102000D8807455000E755515E30901870E7419A3
:1010300001E1755107E109017651020802E3090156
:10104000516B02D00901516B0901515102E10901B3
:10105000508B1DD00901000E745D010E75590CE313
:1010600009010F0ED8807455010E755505E309016D
:1010700050870901516B0BD00901170ED8807455A8
:10108000010E755504E3090150890901516B0901ED
:10109000515112E1A4C310F0116A126A136A105080
:1010A00011101210131008E076C9A8FF74C9DDF200
:1010B00075C9DEF2B8EC3DF0C3EF0DF0A0C3E9FF57
:1010C000A1C3EAFFEFCF10F0610E105C01E21BD26A
:1010D000A0C3E9FFA1C3EAFFEF50670801E213D202
:1010E000A0C3E9FFA1C3EAFFEF50640807E0A0C373
:1010F000E9FFA1C3EAFFEF50650804E1F36AF46A6F
:10110000C8EF0DF0870E0201DB6FDC6BA7EC3DF042
:1011100002080BE1A0C3E9FFA1C3EAFFEF50630897
:1011200004E1F36AF46AC8EF0DF0A0C3E9FFA1C3BC
:10113000EAFFEF509F0F09017A6F7B6B890E09015F
:101140007A270F0E09017B23010E0301EA6AA0250D
:10115000E96EA151EA22EF5014E10301510E116F23
:10116000090E126FA2C30FF3A3C310F318EC39F0EA
:10117000000906E07AC9E9FF7BC9EAFF51C9EFFF20
:10118000C1D1010E0301EA6AA025E96EA151EA224C
:10119000EF50780833E1020E0301EA6AA025E96EF8
:1011A000A151EA22EF50D00F106E010E105204E050
:1011B000E846FE0B1006FCE109017D6FA2C3E9FFC2
:1011C000A3C3EAFFEF5031080AE109017D1D106E4B
:1011D0007AC9E9FF7BC9EAFF1050EF160ED0A2C30F
:1011E000E9FFA3C3EAFFEF50300807E17AC9E9FF3E
:1011F0007BC9EAFF09017D51EF1284D1010E030181
:10120000EA6AA025E96EA151EA22EF50630801E0E5
:1012100079D0020E0301EA6AA025E96EA151EA2203
:10122000EF50D00F09017D6F09017D51070869E377
:10123000010E7DC9E7FFE75204E0E846FE0BE70632
:10124000FCE109017D6FA0C3E9FFA1C3EAFFEF50F4
:101250009F0F09017A6F7B6B920E09017A270F0E9F
:1012600009017B23A0C3E9FFA1C3EAFFEF509F0F51
:10127000230F0201DB6FDC6BA7EC3DF009017C6FF3
:10128000A2C3E9FFA3C3EAFFEF5031080CE17AC91A
:10129000E9FF7BC9EAFF09017D51EF1209017D5188
:1012A00009017C1316D0A2C3E9FFA3C3EAFFEF50E4
:1012B00030080FE109017D1D09017D6F7AC9E9FF41
:1012C0007BC9EAFF09017D51EF1609017D51090132
:1012D0007C17030E0301EA6AA025E96EA151EA22F8
:1012E000EF5072080EE17CC9A8FFA0C3E9FFA1C3BB
:1012F000EAFFEF509F0F230F0201DD6FDE6BB8ECAA
:101300003DF000D1010E0301EA6AA025E96EA1516A
:10131000EA22EFCF10F0300E105C01E2F3D0010EA4
:101320000301EA6AA025E96EA151EA22EF503908CB
:1013300001E2E8D0010E0301EA6AA025E96EA1519D
:10134000EA22EF50D00F09017D6F020E0301EA6A15
:10135000A025E96EA151EA22EF500AE0020E030136
:10136000EA6AA025E96EA151EA22EF5072085BE11A
:10137000010E7DC9E7FFE75204E0E846FE0BE706F1
:10138000FCE109017D6FA0C3E9FFA1C3EAFFEF50B3
:101390009F0F2A0F0201DB6FDC6BA7EC3DF0090108
:1013A0007C6FA2C3E9FFA3C3EAFFEF50300810E14E
:1013B00009017D1D09017D6F7AC9E9FF7BC9EAFF3B
:1013C00009017D51EF1609017D5109017C1712D0E9
:1013D000A2C3E9FFA3C3EAFFEF5031080BE17AC9CA
:1013E000E9FF7BC9EAFF09017D51EF1209017D5137
:1013F00009017C13020E0301EA6AA025E96EA151DE
:10140000EA22EF5072080EE17CC9A8FFA0C3E9FFF1
:10141000A1C3EAFFEF509F0F2A0F0201DD6FDE6BC1
:10142000B8EC3DF06FD0020E0301EA6AA025E96E28
:10143000A151EA22EF5070080AE0020E0301EA6AA5
:10144000A025E96EA151EA22EF506E085BE1010E82
:101450007DC9E7FFE75204E0E846FE0BE706FCE142
:1014600009017D6FA2C3E9FFA3C3EAFFEF50D00FCC
:101470000901516F000E0901515D04E30901515149
:10148000090802E20901516B020E0301EA6AA02574
:10149000E96EA151EA22EF50700817E17AC9E9FF1D
:1014A0007BC9EAFF09017D51EF1209015151510732
:1014B000000901E0FAD709017D1D106E7AC9E9FF24
:1014C0007BC9EAFF1050EF161DD0A2C3E9FFA3C3EA
:1014D000EAFFEF50310816E109017D1D106E7AC94F
:1014E000E9FF7BC9EAFF1050EF160901515151077E
:1014F000000901E0FAD77AC9E9FF7BC9EAFF0901CF
:101500007D51EF1240D3A0C3E9FFA1C3EAFFEF5022
:101510006C0801E082D1010E0301EA6AA025E96EA0
:10152000A151EA22EF506B0A01E17FD0070A01E1E5
:101530007CD0020A35E00F0A1BE0030A01E06CD1FF
:10154000A4C310F0116A126A136A1050111012101D
:1015500013100DE00301080E176FA2C315F3A3C308
:1015600016F33E0E0301136F146B3DEC39F054D1AA
:10157000A4C310F0116A126A136A105011101210ED
:1015800013100DE00301080E176FA2C315F3A3C3D8
:1015900016F3350E0301136F146B3DEC39F03CD19B
:1015A000A4C310F0116A126A136A105011101210BD
:1015B00013103AE00901010E516F0901526B0F0E31
:1015C0000901525D2AE2090151510AE00901525113
:1015D0000301EA6AA225E96EA351EA22EFCF51F98D
:1015E000090151510BE1200EA86E470E0901522549
:1015F0000201DD6FDE6BB8EC3DF00AD051C9A8FFE7
:10160000470E090152250201DD6FDE6BB8EC3DF09B
:1016100035EC48F00901522BD2D7A86A560E0201C8
:10162000DD6FDE6BB8EC3DF0F7D0A2C37FF9A3C34A
:1016300080F90901526B0901816B0901826B020E6D
:101640000301EA6AA025E96EA151EA22EFCF10F06A
:10165000300E105C15E3020E0301EA6AA025E96E64
:10166000A151EA22EF5039080BE3020E0301EA6AA6
:10167000A025E96EA151EA22EF50D00F0901826F37
:101680001F0E0901525D01E39FD009017FC9E9FFE7
:1016900080C9EAFF7F2B000E8023EFCF7EF909017E
:1016A0007E5101E191D00901815112E15F0E0901E2
:1016B0007E5D03E10901812B0AD009015251522BB1
:1016C000EA6A530FE96E090EEA227EC9EFFF7BD06A
:1016D0000901810562E15F0E09017E5D0DE10901ED
:1016E0005251522BEA6A530FE96E090EEA227EC963
:1016F000EFFF0901816B50D0010E0301EA6AA025BA
:10170000E96EA151EA22EF506C0833E10901516BF7
:1017100009017E51740A19E0160A13E0100A0DE05F
:10172000140A07E0080A01E014D009010A0E516FFB
:1017300010D009010C0E516F0CD009010D0E516F24
:1017400008D00901080E516F04D00901090E516F2C
:1017500000D0090151510AE009015251522BEA6AA5
:10176000530FE96E090EEA2251C9EFFF0901816B9F
:1017700013D0010E0301EA6AA025E96EA151EA2205
:10178000EF506B0809E17EC90EF3FDEC38F0100D47
:10179000F3CF51F90901812B16D0020E0901815DA9
:1017A00012E17EC90EF3FDEC38F009015113090175
:1017B0005251522BEA6A530FE96E090EEA2251C9BF
:1017C000EFFF0901816B5CD7010E0301EA6AA025D6
:1017D000E96EA151EA22EF506C0812E10901525161
:1017E000EA6A530FE96E090EEA22EF6A0401530E0A
:1017F000186F090E196F82C917F481EC4CF00BD0E9
:1018000052C916F40401530E146F090E156F82C9E4
:1018100013F44CEC4CF000D0B6D1A0C3E9FFA1C347
:10182000EAFFEF506D0821E1A4C310F0116A126ABB
:10183000136A105011101210131016E0A2C3E9FF22
:10184000A3C3EAFFEF50720A01E00ED0B9EC25F015
:10185000FF0E986E966E956E936E000E866E846E79
:10186000836E816EFF0000D08ED1A0C3E9FFA1C3BB
:10187000EAFFEF50770801E0EFD0010E0301EA6ABA
:10188000A025E96EA151EA22EF5066081CE1A2C32F
:10189000E9FFA3C3EAFFEF50D00F0901516F020E19
:1018A0000301EA6AA025E96EA151EA22EF5072080D
:1018B00002E0000E01D0010E0201E56F51C9E4F211
:1018C00057EC3FF0C8D0010E0301EA6AA025E96E8B
:1018D000A151EA22EF50650821E10301510E116F79
:1018E000090E126FA2C30FF3A3C310F318EC39F063
:1018F000000913E0020E0301EA6AA025E96EA15176
:10190000EA22EF50720802E0000E01D0010E02013F
:10191000E76F51C9E6F29BEC3FF09DD0010E030149
:10192000EA6AA025E96EA151EA22EFCF10F0310E4C
:10193000105C37E3010E0301EA6AA025E96EA151AC
:10194000EA22EF5035082DE3A2C3E6FFA3C3E6FF6A
:10195000F4EC56F0E552E552F3CF85F9F4CF86F971
:10196000020E0301EA6AA025E96EA151EA22EF50B6
:10197000720802E0000E01D0010E0201E26F85C97B
:10198000E0F286C9E1F2010E0301EA6AA025E96EE0
:10199000A151EA22EF50D00F0201DF6FD5EC3EF0EB
:1019A0005AD0010E0301EA6AA025E96EA151EA228C
:1019B000EF506D0850E10901010E526F650E0201F2
:1019C000DB6FDC6BA7EC3DF0FE0B0901516FA2C38E
:1019D000E9FFA3C3EAFFEF50380808E13F0ECB5CF4
:1019E00004E00901526B3F0ECB6E14D0A2C3E9FF95
:1019F000A3C3EAFFEF5061080DE1CB50106E116AEE
:101A0000FF0E101801E1115003E00901526BCB6881
:101A100009015181090152510CE10201E56B640E8B
:101A20000201DB6FDC6BA7EC3DF00201E46F57ECC9
:101A30003FF0020E0301EA6AA025E96EA151EA22F5
:101A4000EF50720808E151C9A8FF650E0201DD6F71
:101A5000DE6BB8EC3DF097D0A0C3E9FFA1C3EAFF6D
:101A6000EF50780801E08FD0A2C3E9FFA3C3EAFFDB
:101A7000EF50300802E1000E01D0010E0901876F1E
:101A8000010E0301EA6AA025E96EA151EA22EF5096
:101A9000720834E1020E0301EA6AA025E96EA15141
:101AA000EA22EF50D00F0901886F870E0201DB6F29
:101AB000DC6BA7EC3DF00901516F0901510509E10B
:101AC00087C9E3F3090188050301E26FD6EC53F0FF
:101AD00014D0020E0901515D10E1010E0901885D6B
:101AE0000CE309018851050808E387C93EF20901A2
:101AF000880502013D6F11EC37F045D0010E03015E
:101B0000EA6AA025E96EA151EA22EF506F083BE195
:101B1000020E0301EA6AA025E96EA151EA22EF5004
:101B2000D00F0901886F870E0201DB6FDC6BA7EC19
:101B30003DF00901516F0901510511E1010E090143
:101B4000885D0DE309018851060809E387C9E5F3BB
:101B5000090188050301E46FECEC53F014D0020E88
:101B60000901515D10E1010E0901885D0CE30901D5
:101B70008851060808E387C940F209018805020177
:101B80003F6F4FEC37F04FC9F3FF50C9F4FF00D05F
:101B90001200F8EC11F0EF500901506F010EEB50FC
:101BA000516F020EE926000EEA22EECF54F9EDCF76
:101BB00055F9F5EC11F0EF6A610E515D67E3515193
:101BC000680864E34F6B610E515D536F070E50154B
:101BD000106E010E105204E0E846FE0B1006FCE108
:101BE0000901526F5351566F576B920E56270F0EC5
:101BF0005723DBDB09E15351566F576B890E56278C
:101C00000F0E57234F8107D05351566F576B800EDD
:101C100056270F0E5723F00E5015536FE85004E16E
:101C2000C4DB01E185D030D0100E535D04E1BDDB93
:101C300001E17DD275D2200E535D03E1010E4F15F7
:101C400006E0300E535D08E1010E4F1505E0080E69
:101C5000501501E1B5D1C9D1400E535D0EE150A739
:101C600003D04FB17FD202D04FA17CD20301000E2E
:101C7000AA6FC00EAB6F000E60D2500E535D01E034
:101C800071D2010E4F1554E1310E55D06B0E515DDE
:101C900003E0750E515D18E140DB13E06B0E515D02
:101CA00005E150510201DB6FDC6B08D0505102019D
:101CB000DB6FDC6B000EDB27010EDC23A7EC3DF0B5
:101CC00058D00301BE6B57D06C0E515D56E15005E4
:101CD00007E10301F00EAA6FC00EAB6F000E2DD20C
:101CE000020E505D07E10301A00EAA6FC00EAB6F9C
:101CF000000E23D2040E505D07E10301E30EAA6F2C
:101D0000960EAB6F000E19D250510AE106DB01E0CE
:101D10007DD10301DD0EAA6F960EAB6F000E0DD2C2
:101D2000030E505D0AE164DB060EEB5070DB02E14E
:101D3000300E01D0310E79DB05D0060E505D04E186
:101D400054DB300EEF6EE6D1050E505D02E1470E1A
:101D500063D1100E505D01E205D25051210801E21D
:101D600001D2100E505DEA6AB10FE96E020EEA224E
:101D7000EF500301BE6FBF6B0ED16E0E515D01E0DF
:101D800082D04F6B0F0E5015106EC11C0F0B105CE4
:101D900001E24F83F00E5015536FE8500BE12DDB3D
:101DA00003E1542B000E5523BEDAEECFB9F3EDCF8D
:101DB000BAF3DDD0100E535D06E1B5DAEECFBEF317
:101DC000EDCFBFF3E8D0200E535D3FE1ACDAEECFAC
:101DD00058F9EDCF59F911DB2BE158C910F059C969
:101DE00011F0CC0EC2DAF0DA0301986F2E0E996F63
:101DF000CC0EBBDA02C058F903C059F902C010F08A
:101E000003C011F00A0E9BDADFDA03019A6F0A0EA3
:101E1000ACDA06C058F907C059F906C010F007C07F
:101E200011F0640E8CDA300E062403019B6F9C6B5C
:101E300009015451A8DAF9DAEF6E5451A4DA01E13C
:101E400069D19BDAEE2AEF228AD1300E535D04E18C
:101E5000020E4F1501E0B4D0500E535D04E1020EA6
:101E60004F1501E1ADD0400E535D04E1020E4F1558
:101E700001E0BBD0600E535D01E074D1020E4F153E
:101E800001E070D1B2D0770E515D01E0B5D04F6B5B
:101E90000F0E50155B6F5A6BE80403E1BDCF5AF982
:101EA00011D0020E5B5D03E1BACF5AF90BD0030EDD
:101EB0005B5D03E1B7CF5AF905D0040E5B5D02E12B
:101EC00073CF5AF90F0E5A1501E04F87F00E5015D7
:101ED000536FF00E535D3CE15B5104E185EC3FF044
:101EE000300F16D1040E5B5D13E1CB50106E116AFA
:101EF000FF0E101801E1115002E0000E01D0010E9A
:101F0000010803E172DA610E04D16FDA380E01D1F3
:101F1000080E5B5D01E026D1536B0F0EBD1401E08E
:101F200053810F0EBA1401E053830F0EB71401E072
:101F300053850F0E731401E0538753C9B5F3E0D9ED
:101F4000EECFB3F3EDCFB4F354C9B2F35DD9FED005
:101F5000535116E152DA03E1542B000E55235BC9AD
:101F6000E3F220EC3FF0F3CFB9F3F4CFBAF3C8D9E2
:101F7000EECFB7F3EDCFB8F354C9B6F367D9E6D0D7
:101F8000100E535D11E15BC9E3F220EC3FF0F3CF9B
:101F9000BEF3F4CFBFF3B4D9EECFBCF3EDCFBDF3B6
:101FA00054C9BBF384D9D2D0300E535D03E1080E7F
:101FB0004F1506E1500E535D0AE1080E4F1507E17B
:101FC0000301110EAA6FC00EAB6F000EB6D0400E0B
:101FD000535D03E1080E4F1508E1600E535D01E00B
:101FE000C1D0080E4F1501E0BDD00301160EAA6F37
:101FF000C00EAB6F000EA1D0730E515D19E18DD9EB
:1020000003E1F3D9300E85D0505102E1350E04D0F2
:10201000500501E0A7D03E0E0301B06FB16B70D93F
:10202000EECFAEF3EDCFAFF354C9ADF3CCD88ED035
:10203000780E515D01E096D05F6B010E616F0F0E5F
:1020400050155C6F0F0E5015606FF00E50155D6FE0
:10205000870EA0D909015E6F5D5103E0100E5D5D32
:1020600031E15E050EE1B7D904E0E846FE0BE70674
:10207000FCE1106EE66E24EC54F0B2D911E0010ED2
:1020800012D0020E5E5D12E1A6D904E0E846FE0B16
:10209000E706FCE1106EE66EA0EC37F0A1D902E194
:1020A000000E01D0010E09015F6F01D0616B61511B
:1020B00059E05D5104E15F5128E1300E29D05F51B4
:1020C00036E02ED0200E5D5D03E0300E5D5D4AE10E
:1020D000020E5E5D12E17FD904E0E846FE0BE706E2
:1020E000FCE1106EE66E05EC37F07AD902E1000EE5
:1020F00001D0010E09015F6F01D0616B615132E0C7
:10210000200E5D5D0BE15F5102E0310E01D0300E1B
:102110008CD9EF6E32D9EE68ED6821D05F5107E0BF
:1021200003011A0EAA6FC00EAB6F000E06D003019A
:102130001D0EAA6FC00EAB6F000EAC6FE1D8EECFD4
:10214000A8F3EDCFA9F354C9A7F312D8F4CF11F037
:102150004FD9020EF3CFEBFF030E11C0EBFF010EC0
:10216000F36E04D00AD9EE68ED68F36AF46A1200DF
:10217000A7C310F0116A126A0301AA511024F36E6A
:10218000AB511120F46EAC511220F86EF4CFF7FF72
:10219000F3CFF6FF0800F550A8C3E9FFA9C3EAFF93
:1021A000EF6EA8C3E9FFA9C3EAFFEF5003E1F368AC
:1021B000F4681200A72BA751106E116AA7C3F3FF92
:1021C00011C0F4FF12000301AD51B0250901626F87
:1021D000000E0301B121AA6E62C9A9FF3F0EA61627
:1021E000A680A850AEC3E9FFAFC3EAFFEF6EA850C8
:1021F00003E1F368F4681200AD2BAD51116AADC371
:10220000F3FF11C0F4FF12000301B251010815E3FE
:10221000B25103E1B5390F0BB56F0F0EB517B551BC
:10222000090802E2370E01D0300EB525B3C3E9FF2D
:10223000B4C3EAFFEF6EB20503E1F368F46812007D
:10224000B229116AF36E11C0F4FF12000301B651F6
:10225000030824E3030ED880B655040DF350B9C328
:1022600010F0BAC311F005E0D89011321032E80432
:10227000FBE110C062F90F0E0901621762510908F3
:1022800002E2370E01D0300E6225B7C3E9FFB8C3B2
:10229000EAFFEF6E030E0301B65D03E1F368F46835
:1022A0001200B629116AF36E11C0F4FF1200030187
:1022B000BB5111E1980EE66E030EE66EBEC3E6FF5B
:1022C000BFC3E6FF69EC57F0E552E552E552E5522F
:1022D00003019D6BBB6BBB5156D8BCC3E9FFBDC3AB
:1022E000EAFFEF6EBB514FD803E1F368F4681200C8
:1022F000BB2BBB51116ABBC3F3FF11C0F4FF12002B
:1023000077D8040EE926000EEA221200126A136A38
:10231000105011101210131012006AD8060EEB5054
:10232000106E07EF12F00F0E5015E96EEA6AD890A2
:10233000E936EA36C30EE926020EEA22120011023D
:10234000F3CF11F01002F3CF10F0F4501126CC0EA1
:102350000B6E0C6AF3CF06F011C007F019EF60F0B6
:10236000EE50EFCFEAFFE96E12000B6E0C6A58C90F
:1023700006F059C907F019EF60F03AD8020EE926C5
:10238000000EEA221200EA6A980FE96E030EEA22B2
:10239000EF5012000201DB6FDC6BA7EF3DF0EA6A41
:1023A000060FE96E090EEA22120056C9E9FF57C965
:1023B000EAFFEF50521512000551106E116A3F0EE0
:1023C000105C000E1158120006C010F007C011F08A
:1023D000300E06241200010E60C9E7FFE75212001A
:1023E000E552E7CF10F0101412008ADFB0EF11F0C1
:1023F000A5C3E9FFA6C3EAFF120054C910F055C9EE
:1024000011F086EF11F01016116A86EF11F0116AC3
:10241000126A136AE85011101210131012000551BD
:10242000052BBDDF00C9EFFF1200E66EDEDFE552CF
:04243000E75012005F
:0C2434000901006B0A0E005D2BE2005154
:10244000240DF3CF01F9F4CF02F9000E01270C0E91
:102450000223CDEC1CF00A0EEF6E69EC1EF0EF903B
:1024600069EC1EF0EF8269EC1EF0EF8469EC1EF05F
:10247000EF9869EC1EF0EF96CDEC1CF013EC1EF01B
:10248000CDEC1CF036EC1EF0CDEC1CF04DEC1EF04B
:10249000002BD2D712000901006B0A0E005D48E242
:1024A0000051240DF3CF01F9F4CF02F9000E0127FA
:1024B0000C0E0223B9EC1CF0EF500A0837E1B9EC1E
:1024C0001CF0EF6AB9EC1CF00B0E62C0EBFF0C0EB7
:1024D00063C0EBFFB9EC1CF00D0EEB6A0E0EEB6A5D
:1024E000B9EC1CF0EE524AEC1EF088EC1DF089ECC1
:1024F0001EF0EF8089EC1EF0EF96B9EC1CF047EC73
:102500001CF005E1115003E1125001E1135008E005
:10251000B9EC1CF0C7EC1CF0B9EC1CF013EC1EF08D
:1025200089EC1EF0EF82090100511200002BB5D793
:10253000FE0C09016F6B6C6B0A0E6C5D14E26C5142
:10254000240DF3CF6DF9F4CF6EF9000E6D270C0E4C
:102550006E236FEC1CF0EF500A0803E1010E6F6F61
:1025600002D06C2BE9D76F5101E1FE0C0401CC2B9A
:10257000000ECD236FEC1CF00B0ECCC4EBFF0C0E49
:10258000CDC4EBFFCCC410F0CDC411F0126A136AB5
:10259000D880880E1054130E3AEC1EF003E2CC6B78
:1025A000040ECD6F6FEC1CF09CEC1DF0EF906FEC07
:1025B0001CF00D0E66C0EBFF0E0E67C0EBFF2BECA0
:1025C0001EF01A0E3EEC1CF088EC1DF00A0EE66EB2
:1025D000E66A64C0E6FF65C0E6FF6FEC1CF079ECCC
:1025E0001CF020EC1DF00001020E966F6FEC1CF049
:1025F00003EC1EF06FEC1CF09FEC1EF06FEC1CF077
:1026000007EC1EF06FEC1CF00BEC1EF06FEC1CF0F6
:10261000B2EC1CF06FEC1CF0010EEF6E2BEC1EF018
:1026200031EC1DF009016C5112000001685165EC9C
:102630001CF0EF50030801E0000C010C000169518F
:10264000240DF3CF6CF9F4CF6DF9000E09016C275E
:102650000C0E6D23D2EC1CF0EF5003080BE0D2EC13
:102660001CF0EF50020806E06CC9A0F06DC9A1F0A3
:10267000C1EF19F069C073F092D920EC1DF0000190
:10268000110E966FD2EC1CF003EC1EF0D2EC1CF095
:102690009FEC1EF0D2EC1CF007EC1EF0D2EC1CF00C
:1026A0000BEC1EF0D2EC1CF0B2EC1CF0D2EC1CF0E7
:1026B0006CEC1EF08DEC1DF0D2EC1CF0040EEF6EF5
:1026C000120000016A51240DF3CF7AF9F4CF7BF99F
:1026D000000E09017A270C0E7B2391EC1CF047ECCD
:1026E0001CF007E1115005E1125003E1135001E124
:1026F000000C91EC1CF052EC1EF0020B01E1000CFE
:1027000091EC1CF043EC1EF091EC1CF00F0EEB5022
:102710000001976F0001180E966F03EC1EF091EC0C
:102720001CF09FEC1EF091EC1CF007EC1EF091ECFD
:102730001CF00BEC1EF091EC1CF0B2EC1CF091ECD8
:102740001CF0100ED9EC1DF0126A136A91EC1CF00B
:102750006CEC1EF056EC1DF091EC1CF09CEC1DF0A6
:10276000EF9291EC1CF09CEC1DF0EF98010C0A0E1E
:1027700000016B5D01E3000C6B5165EC1CF0140E65
:102780000FEC1EF001E1000C6B5165EC1CF00F0E1C
:102790003EEC1CF0EFCF10F08CEC1EF00AE1115073
:1027A00008E1125006E1135004E10301746B1FEFBE
:1027B00020F06B5165EC1CF052EC1EF0020B01E0B6
:1027C000010E120000016C51240DF3CF78F9F4CF03
:1027D00079F9000E090178270C0E7923D7EC1CF04B
:1027E000140E0FEC1EF001E1000CD7EC1CF047ECCE
:1027F0001CF024E1115022E1125020E113501EE19F
:102800000301756B58EC20F0E66ED7EC1CF00F0E50
:1028100090EC1EF0D7EC1CF047EC1CF007E11150D7
:1028200005E1125003E1135001E1000CD7EC1CF05C
:102830005FEC1DF0D7EC1CF038EC1DF0D7EC1CF071
:102840009CEC1DF0EF886DC076F3A2EC20F0D7EC85
:102850001CF0140E3EEC1CF0EE06EF5AD7EC1CF008
:10286000100E3EEC1CF0EE2AED22EECF10F0EDCF74
:1028700011F026EC1DF003E36CC06AF022DF010CBE
:1028800000016E51240DF3CF6CF9F4CF6DF9000EF9
:1028900009016C270C0E6D239BEC1CF0140E0FEC41
:1028A0001EF001E1000C9BEC1CF047EC1CF024E155
:1028B000115022E1125020E113501EE10301756B0B
:1028C00058EC20F0E66E9BEC1CF00F0E90EC1EF026
:1028D0009BEC1CF047EC1CF007E1115005E1125095
:1028E00003E1135001E1000C9BEC1CF05FEC1DF0C8
:1028F0009BEC1CF038EC1DF07CEC1EF000017151DB
:10290000EE24106E7251EE20116E126A136AD88096
:10291000CA0E1054030E3AEC1EF014E2CA0E146EE6
:10292000030E156E166A176A7CEC1EF0EECF18F0D7
:10293000EFCF19F01A6A1B6AFDEC1CF010C071F0A1
:1029400011C072F09BEC1CF09CEC1DF0EF8871C084
:1029500079F372C07AF36FC077F370C078F3CEEC7E
:1029600020F09BEC1CF0140E3EEC1CF000017151A9
:10297000EE5E7251ED5A7CEC1EF07151EE267251F2
:10298000ED229BEC1CF0100ED9EC1DF026EC1DF096
:1029900003E36EC06AF095DE000171511200000180
:1029A0007351240DF3CF00F9F4CF01F9000E0901A2
:1029B00000270C0E012300C9E9FF01C9EAFF99ECC9
:1029C0001EF001E1000C27EC23F000C9E9FF01C96A
:1029D000EAFF9CEC1EF0010C00017451240DF3CFB2
:1029E00000F9F4CF01F9000E090100270C0E0123B4
:1029F000F3EC1CF099EC1EF03CE0F3EC1CF052EC14
:102A00001EF0040B0CE00001AB6BAC6B74C0AAF0C1
:102A1000EBEC1BF0F3EC1CF09CEC1DF0EF94F3ECF2
:102A20001CF0120ED9EC1DF000017751105C7851AA
:102A3000115808E2F3EC1CF096EC1EF0EECF77F0A4
:102A4000EDCF78F0F3EC1CF0120E0FEC1EF007E166
:102A500027EC23F0F3EC1CF09CEC1EF00AD077C0BE
:102A60007DF378C07EF375C07BF376C07CF311EF05
:102A700022F0F36AF46A120000017951240DF3CFB9
:102A800087F9F4CF88F9000E090187270C0E8823F7
:102A9000896B8A6B8B6BF8EC1CF099EC1EF052E0A2
:102AA000F8EC1CF052EC1EF0040B0CE00001AB6BD8
:102AB000AC6B79C0AAF0EBEC1BF0F8EC1CF09CECD2
:102AC0001DF0EF94F8EC1CF0120ED9EC1DF0000193
:102AD0007C51105C000E115809E2F8EC1CF096ECE9
:102AE0001EF0EFCF7CF00901100E896FF8EC1CF09E
:102AF000120E0FEC1EF00AE127EC23F0F8EC1CF0AC
:102B00009CEC1EF0F36A100EF46E12007DC082F38E
:102B10007CC081F37AC07FF37BC080F36BEC22F042
:102B2000F3CF8AF9F4CF8BF927EC1EF0200EF418BE
:102B30000BE1115009E1125007E1135005E10901C1
:102B4000200E01D0300E896F89C98BF98AC9F3FF35
:102B500089C9F4FF120000017E51240DF3CF87F9DB
:102B6000F4CF88F9000E090187270C0E88231BEC8F
:102B70001DF099EC1EF02DE01BEC1DF052EC1EF048
:102B8000040B0CE00001AB6BAC6B7EC0AAF0EBEC6D
:102B90001BF01BEC1DF09CEC1DF0EF941BEC1DF0EA
:102BA000120E0FEC1EF007E127EC23F01BEC1DF0DA
:102BB0009CEC1EF0000C1BEC1DF096EC1EF0EE06DB
:102BC000EF5AB6EC21F07FC0E9FF80C0EAFFEF6E5C
:102BD000010C000C0A0E0001815D01E3000C815123
:102BE00065EC1CF099EC1EF001E0010E12000901E9
:102BF0007B6B6C6B0A0E6C5D01E31FD16C51240D75
:102C0000F3CF75F9F4CF76F9000E75270C0E762305
:102C10004CEC1CF099EC1EF001E00CD14CEC1CF0DB
:102C200052EC1EF0100B01E005D14CEC1CF0EF5003
:102C30000A0801E1FFD04CEC1CF0EF50000907E15D
:102C40004CEC1CF052EC1EF0010B01E0F3D04CEC0C
:102C50001CF01F0E3EEC1CF00401EE50A15D106E46
:102C6000EE50A259116E4CEC1CF0210E3EEC1CF003
:102C700065EC1DF01050125C1150135801E3DAD0CE
:102C80006EEC1DF001E112004CEC1CF031EC1DF07B
:102C90004CEC1CF0210E3EEC1CF0010ED890EE36F0
:102CA000ED36E806FBE14CEC1CF01E0E3EEC1CF091
:102CB000EF2A4CEC1CF0EF50090A6EE0010A64E0C8
:102CC0000F0A71E0020A6FE0030A6DE0020A56E0A3
:102CD000070A1FE0010A05E0030A6AE10901020E82
:102CE00060D040EC1EF003E30901120E5AD04CEC08
:102CF0001CF052EC1EF0010B04E04CEC1CF0EF6AEF
:102D000052D00901020E7B6F4CEC1CF0010EEF6EED
:102D10004AD040EC1EF018E34CEC1CF047EC1CF0E1
:102D200005E1115003E1125001E113500AE00301E3
:102D3000966B976B4CEC1CF038EC1DF060EC25F0BA
:102D400037D00901100E2DD04CEC1CF047EC1CF0D4
:102D500005E1115003E1125001E1135008E04CEC81
:102D60001CF0C7EC1CF04CEC1CF013EC1EF009013D
:102D7000110E7B6F4CEC1CF0040E0CD040EC1EF0DE
:102D800012E30901010E0DD00901010E7B6F4CEC1D
:102D90001CF0090EEF6E0CD040EC1EF004E30901AC
:102DA000110E7B6F05D075C9A0F076C9A1F0E9DAE4
:102DB00009017B513FE07BC910F0100EDCEC1CF0E8
:102DC0000DE04CEC1CF06CEC1EF0EECF77F9EECF82
:102DD00078F9EECF79F9EFCF7AF910D04CEC1CF0FE
:102DE0006CEC1EF0EFCF77F9EE2AEFCF78F9EE22F8
:102DF000EFCF79F9EE22EFCF7AF9EF2220EC1DF038
:102E00007BC996F04CEC1CF003EC1EF077C98EF0F9
:102E100078C98FF079C990F07AC991F04CEC1CF028
:102E200007EC1EF04CEC1CF00BEC1EF04CEC1CF014
:102E3000B2EC1CF009016C2BDDD6120082C0E9FF58
:102E400083C0EAFF4AEC1EF0EECF80F9EECF81F9A5
:102E5000EECF82F9EFCF83F984C0E9FF85C0EAFFA6
:102E6000EECF84F9EECF85F9EECF86F9EFCF87F973
:102E70000901886B060E896F86C08AF987C08BF9B5
:102E800086C002F387C003F3F2EC37F0F3CF8AF980
:102E9000F4CF8BF90C0E03010A6F0B6B0301800E4C
:102EA000086F090E096F26EC38F0F3CF8DF9F4CFD7
:102EB0008EF909018D1F8E1F86C00CF387C00DF39C
:102EC00092EC38F0F3CF8FF9F4CF90F90901F45078
:102ED0008D5D61E18F518E5D5EE10401476B486B52
:102EE00053EC4EF0140E03017D6F7E6B03016C0EEC
:102EF0007B6F090E7C6F11EC22F000016C0E9E6F4F
:102F0000090E9F6FF5D93EEC1DF0106E116A140E7C
:102F1000105E000E115A10C091F91050106E116A17
:102F2000E8500001865D866F11508759876F140E37
:102F3000865F000E875B3EEC1DF00401476F486B17
:102F400053EC4EF082C09CF083C09DF000016C0EEB
:102F50009A6F090E9B6F3BD909018C6F106E27EC9D
:102F60001EF0FE0E101805E1115003E1125001E1B0
:102F7000135011E086C0A7F087C0A8F000016C0EC6
:102F8000A56F090EA66F82C0A3F083C0A4F08CC900
:102F9000A2F02FDA010C27EC23F0010C6EEC1DF0EF
:102FA00003E135EC48F0FAD76AEC1DF00DE1115061
:102FB0000BE1125009E1135007E10301010E756F97
:102FC00058EC20F00001976F6AEC1DF007E11150FA
:102FD00005E1125003E1135001E11200140E0AEC56
:102FE0001DF08AC048F98BC049F98CC04AF98DC0E0
:102FF0004BF98EC04CF98FC04DF990C04EF991C07D
:103000004FF992C050F993C051F994C052F995C04C
:1030100053F90901549154935495549796C055F916
:103020003BEC23F0F3CF56F9F4CF57F9F3CF10F080
:10303000F4CF11F0126A136A000EF35C040EF45818
:10304000000E1258000E135805E30901566B040ECA
:10305000576F0ED00901360ED8805655000E5755C1
:1030600005E2360E565F000E575B02D0566B576B6B
:10307000586B596B5A6B5B6B0001480E9E6F090EC3
:103080009F6F36D9140E00019827000E992396C021
:1030900010F0020EDCEC1CF00EE0040E9827000E7F
:1030A00099230901020E5C6F040E5D6F5E6F5F6B0A
:1030B0005499548B03D009015489549B548D549FC7
:1030C000B1C260F9B2C261F9B3C262F9B4C263F9C4
:1030D00088C0E9FF89C0EAFF4AEC1EF0EECF64F930
:1030E000EECF65F9EECF66F9EFCF67F9686B060EA4
:1030F000696F98C06AF999C06BF998C002F399C0DA
:1031000003F3F2EC37F0F3CF6AF9F4CF6BF90C0E5E
:1031100003010A6F0B6B0301600E086F090E096F44
:1031200026EC38F0F3CF58F9F4CF59F90901581FBC
:10313000591F58C946F959C947F998C045F499C06B
:1031400046F40401060E446F88C042F489C043F47B
:10315000E4EC4DF0140E0301796F7A6B0301480E15
:10316000776F090E786FCEEC20F096C010F0020E4B
:10317000DCEC1CF00BE0040E0301796F7A6B0301A9
:103180005C0E776F090E786FCEEC20F0140E0AEC0F
:103190001DF098C00CF399C00DF392EC38F0F3CF0A
:1031A00046F9F4CF47F9240E0AEC1DF047C976F32F
:1031B000A2EC20F046C976F3A2EC20F00301966B56
:1031C000976B97C095F318EC26F060EF25F0090196
:1031D000FE0E036F026B0A0E025D51E2025148ECD3
:1031E0001DF0AEDBEF500A0847E0AADB0B0ED9EC6E
:1031F0001DF092EC1DF0020E41DB65EC1DF00001AC
:103200001250101839E11350111836E199DBEF50C4
:10321000000902E102C903F993DB0D0ED9EC1DF0A0
:1032200092EC1DF065EC1DF01250101825E11350C2
:10323000111822E19CC0E9FF9DC0EAFF4AEC1EF094
:10324000EECF14F0EECF15F0EECF16F0EFCF17F073
:1032500077DBEE524AEC1EF0EE5014180DE1EE5002
:1032600015180AE1EE50161807E1EE50171804E1A0
:1032700003E10901025112000901022BACD703C975
:1032800010F027EC1EF0FE0E101807E1115005E1BA
:10329000125003E1135001E1FE0C035148EC1DF004
:1032A0000A0EE66EE66A9CC0E6FF9DC0E6FF48DBBC
:1032B00020DB125092EC1DF039DB42DB75EC1DF087
:1032C0003FDB9CEC1EF03CDBE2DA05E1115003E150
:1032D000125001E1135005E033DB59DB31DB13EC15
:1032E0001EF02EDB9CEC1DF0EF8209010351120051
:1032F000DDDAEFCF07F983EC1EF0D4DBD7DAEAECA6
:103300001DF0020EFBEC1DF0020EC1EC1DF0020ED2
:1033100000EC1EF0020E93EC1EF0040EC4EC1DF047
:10332000040E30EC1EF0080EC4EC1DF0080E30EC5C
:103330001EF00E0EFBEC1DF00E0EC1EC1DF00E0E7D
:1033400000EC1EF00E0E93EC1EF0100EFBEC1DF0C8
:10335000100EC1EC1DF0100E00EC1EF0100E93ECE0
:103360001EF0120EFBEC1DF0120EC1EC1DF0120E41
:1033700000EC1EF096EC1EF0010E80DA07C9EFFF9C
:103380001200B2DA84DA05E1115003E1125001E1D2
:10339000135008E0A9DAFBDAA7DA13EC1EF0A4DA7E
:1033A000CBDBEF82A1DAEE524AEC1EF0B1DB9CDA05
:1033B0000D0EEB6A0E0EEB6A97DA99EC1EF002E046
:1033C00027EC23F091DA9CEC1EF08EDA36EC1EF03E
:1033D0008BDAB2DBEF9888DA52EC1EF0010B03E0D7
:1033E00083DAEF6A03D080DA0A0EEF6E7DDA4DEFF2
:1033F0001EF00001A251240DF3CFB6F9F4CFB7F9B6
:10340000000E0901B6270C0EB723A7C060F0A8C0B4
:1034100061F0B86B37DA1E0E31DAEF6A33DA21DB8E
:1034200031DA36EC1EF083DB040B0EE027EC23F0E0
:1034300029DA52EC1EF0010B02E0000E01D0010E61
:10344000E66E20DA52EF1DF099DBF1DB0E0E16DA94
:10345000EECF14F0EFCF15F0166A176A22DA080ED5
:103460000DDAEE50AA5D186EEE50AB59196EEE50A3
:10347000AC591A6EEE50AD591B6EBFDA03DA100E5E
:10348000FDD9EECF1CF0EFCF1DF01E6A1F6A1C5055
:10349000105CA66F1D501158A76F1E501258A86FD0
:1034A0001F501358A96F800EA91506E0EBD9140E12
:1034B000EB6A150EEB6A07D0E5D9140EA6C9EBFF2F
:1034C000150EA7C9EBFF80EC1EF0010820E12FDBF1
:1034D000020B06E165EC1EF0100B01E16BD11ED072
:1034E0002EDBE3DB70DAA5EC1EF006E1CBD9020E91
:1034F000EF6E27EC23F02BD0C5D9030EEF6E100E24
:10350000B86FEDDB0001A751A81168E1C1D080ECD4
:103510001EF0000920E1D9DB020B03E10901040ED2
:1035200018D00DDBDCDB0A0EE66EE66AA3C0E6FF10
:10353000A4C0E6FFA7D9DDD91250B3D9F7D9A2D9D3
:10354000D4DAA0D9020EEF6E19DB36DB3CDA0901C2
:10355000120EB86FDAD0A9DBEECFAEF9EECFAFF92D
:10356000EECFB0F9EFCFB1F909DBEECFB2F9EECF84
:10357000B3F9EECFB4F9EFCFB5F993D9040E7ED9F4
:1035800022DA0001A7510901A6270001A85109016B
:10359000A723000EA823A923F1DA49DB040E6ED974
:1035A000EE50AE1901E0A4D0EE50AF1901E0A0D06A
:1035B000EE50B01901E09CD0EE50B11901E098D066
:1035C00001E096D09DDB02080BE1BFDB61E008DB88
:1035D000030EEF6E0001A751A8115AE06ADB95D0E7
:1035E000FFDAEF50030857E1B0DB29E05AD9080EA3
:1035F00045D9EECF10F0EECF11F067DABFDA1050F8
:10360000EE181DE11150EE181AE11250EE1817E1F4
:103610001350EE1814E113E135D944DB020B0FE12E
:1036200031D935D905E1115003E1125001E11350B0
:1036300006E028D9ACD926D9F6DA84DBEF8277DA2E
:10364000010B09E00901110EB86F98DAB5DA7DD9DE
:1036500019D9090EEF6E0001A751A81119E012D96E
:1036600068DB04E126DB0901B8894FD087DAB2C9EB
:10367000EEFFB3C9EEFFB4C9EEFFB5C9EEFF15DB2F
:10368000AEC9EEFFAFC9EEFFB0C9EEFFB1C9EEFFA4
:1036900027EC23F03AD034DB090804E116DB100BE9
:1036A00034E020D02DDB04080FE10FDB010B06E036
:1036B000C8DA4BDB17E1E6D8060E04D046DB25E07E
:1036C000E1D8050EEF6E21D01BDB050805E1FDDA20
:1036D000010B1BE0B6DA06D013DB060816E1F5DABB
:1036E000100B13E0B6C9A0F0B7C9A1F04ADE0DD0A7
:1036F00027EC23F00901100EB86FAEC9A6F9AFC9C7
:10370000A7F9B0C9A8F9B1C9A9F90901B85152E09E
:10371000B9D8C8DA020B2FE1B5D8B9D805E11150F4
:1037200003E1125001E1135026E0ACD8100E77DA15
:1037300022E0DBDA1050EE5E1150EE5A1250EE5AD3
:103740001350EE5A9FD89FDA9DD80F0EEB50000110
:10375000976FB8C910F07BDA108610C096F053DA74
:103760000DDA0CD98FD853DA8DD855DA8BD8FAD830
:10377000BCDA56EF1DF064D9B8C996F0A6C992F02C
:10378000A7C993F0A8C994F0A9C995F0AAC98EF069
:10379000ABC98FF0ACC990F0ADC991F082D841D9D6
:1037A00080D8020E6BD842D9A3C088F0A4C089F09B
:1037B000CEEC17F012000001A951240DF3CF10F048
:1037C000F4CF11F0000E10260C0E112210C0F3FFE2
:1037D00011C0F4FF12000001AA51240DF3CF8DF99E
:1037E000F4CF8EF9000E09018D270C0E8E230C0EDE
:1037F0000401476F486B53EC4EF0B6EC21F0E84003
:10380000E8403F0B3C0B09018C6F0001AB51605D40
:10381000106E6151AC55116E8DC9E9FF8EC9EAFF7A
:10382000120E10C0EBFF130E11C0EBFF09018C51FB
:103830000001AB250401476F000E0001AC2104011B
:10384000486F53EF4EF00001AD51240DF3CF00F956
:10385000F4CF01F9000E090100270C0E012300C965
:10386000E9FF01C9EAFF62DA0001EE50605D106E07
:10387000EE50615910C0F3FFF46E1200E926000EFD
:10388000EA221200B6C9E9FFB7C9EAFF12000F0E1B
:10389000EB50106E8CEF1EF075C9E9FF76C9EAFF98
:1038A0001200A5C0E9FFA6C0EAFF12009EC0E9FF12
:1038B0009FC0EAFF12001E0EEB50106EC8D9D880D0
:1038C000030E1054000E3AEF1EF0240DF3CFE9FF63
:1038D000F4CFEAFF000EE9260C0EEA2212006DC9B1
:1038E000E9FF6EC9EAFF1200A0C0E9FFA1C0EAFF2C
:1038F0001200EE52E9CF10F0EACF11F0E9CFE6FF67
:10390000EACFE6FF22EC58F0126E060EE15E1200DE
:10391000EECF92F0EECF93F0EECF94F0EFCF95F0A4
:1039200012007AC9E9FF7BC9EAFF1200EECF10F05E
:10393000EFCF11F012006CC9E9FF6DC9EAFF120068
:1039400000C9E9FF01C9EAFF1200EF2AEECFA6F98C
:10395000EF22EECFA7F9EF22EECFA8F9EF22EFCFBB
:10396000A9F91200EE52E9CF88F0EACF89F0CEEF44
:1039700017F001C9E9FF02C9EAFF1200EECF8EF08D
:10398000EECF8FF0EECF90F0EFCF91F012000F0E50
:10399000EB500301846F09EF23F001C9E9FF02C96D
:1039A000EAFF12006CC9E9FF6DC9EAFF120078C98D
:1039B000E9FF79C9EAFF1200101649D91050111019
:1039C000121013101200EECFA6F9EECFA7F9EECF2A
:1039D000A8F9EFCFA9F9120011C0EEFF12C0EEFF57
:1039E00013C0EEFF120000C9E9FF01C9EAFF12008F
:1039F00087C9E9FF88C9EAFF12001850145C106EED
:103A000019501558116E1A501658126E1B5017582F
:103A1000136E12000301966F976B97C095F318EF22
:103A200026F0EECF8CF0EDCF8DF01200EECF8AF0C5
:103A3000EDCF8BF0120087C9E9FF88C9EAFF1200B9
:103A40000001986B996B000197691200126A136A62
:103A5000CA0E105C030E1158000E1258000E1358B7
:103A600012001F0EA1C4EBFF200EA2C4EBFF120038
:103A70000F0EEB500301956F18EF26F009017851F6
:103A8000F00BE842E842E842E842040DF35012002D
:103A9000240DF3CF00F9F4CF01F9000E00270C0E2E
:103AA00001231200E552E750EF6E12001050EE268F
:103AB0001150EE221250EE221350EE221200EDD8D9
:103AC000280E0301966F976B1200EECF12F0EFCF26
:103AD00013F0120097C010F08CEF1EF00301010EDE
:103AE000746F1FEC20F0000912000D0E10C0EBFFE8
:103AF0000E0E11C0EBFF1200140E10C0EBFF150EDE
:103B000011C0EBFF12002C0EEE6E010EED6E1200D6
:103B1000EE6AEE6AEE6AEE6A1200EE2AEE22EE22FB
:103B2000EE2212009AC0E9FF9BC0EAFF1200B9DE44
:103B30000D0EA4DEEF501200230E3EEF1CF0A7C0C6
:103B400014F0A8C015F0166A176AABDE040E96DEF4
:103B5000EE501424106EEE501520116EEE5016200B
:103B6000126EEE501720136E102A000E1122122230
:103B700013229BD810C0EEFFECEF1CF083DE6CEF3D
:103B80001EF07CDE83EF1EF079DEEECF04F3EECF85
:103B900005F3EECF06F3EFCF07F3F7EC37F004C0F1
:103BA00010F005C011F006C012F007C013F056EF78
:103BB0001CF064DE96EF1CF0EFCFAAF9EE2AEFCFEF
:103BC000ABF9EE22EFCFACF9EE22EFCFADF9EF2259
:103BD00055EF1EF0010E52DE07C9EFFF56EF1CF045
:103BE00064D8A6C9EEFFA7C9EEFFA8C9EEFFA9C910
:103BF000EEFF42EF1CF042DEEFCF07F956EF1CF06C
:103C00008FD856EF1CF01A0E39DE88EF1CF00D0E1F
:103C100035DE11EF1DF00B0E31DE16EF1DF02EDE3E
:103C2000EE50ED1012000F0E29DEEF681200EECFFD
:103C3000AAF9EECFABF9EECFACF9EFCFADF951EF7A
:103C40001CF00901100EB86F30D8A5EF1CF0116AF6
:103C5000126A136A120043DE3FD85FDF6FEF1CF079
:103C60000DDE04C0EEFFB8DE56EF1CF0210E06DEBE
:103C700083EF1DF01154000E1254000E1354120065
:103C80000BDE5BEF1CF0100EF9DDEECF98F0EDCF00
:103C900099F01200060E3EEF1CF0100EEB6A110EAA
:103CA000EB6A120049DFEF501200ECDD1A0E3EEF16
:103CB0001CF048D8EF86E6DD120EA7C0EBFF130E0E
:103CC000A8C0EBFF3FD8EF84120027EC23F097EF5A
:103CD0001DF063DE9CEF1DF0160E3EEF1CF0E1DDE3
:103CE0000E0E67DFCFDD7CEF1DF0CCDD100E61DF47
:103CF000126A136ABEEF1DF01EDE100E3EEF1CF0BE
:103D0000C1DDEF501200010EB9DDEF50E66E56EF47
:103D10001CF02FDE9CEF1DF09ADFE86810181200EF
:103D2000ADDD52EF1DF0AADDEAEF1DF0120E3EEF01
:103D30001CF0B8DF080B1200FFDEEF961200CCDF9C
:103D4000BEEF1CF09FDD9CEF1DF0F1DE100B1200AA
:103D5000966A8688988803016E6B6F6B706B716BC7
:103D6000726B736B0901006B00C910F0116A126A63
:103D7000136A030E105C000E1158000E1258000E4C
:103D800013582EE200C910F0116A126A136A020E6B
:103D9000D8901036113612361336E806F9E1400E87
:103DA0001026000E11221222132209010051E96E81
:103DB000EA6AD890E936EA36660EE926030EEA2268
:103DC00010C0EFFF0051E96EEA6AD890E936EA3692
:103DD000660EE926030EEA22EE52EF80002BC4D7CE
:103DE000236A03016C69B9EC25F00401050ECB6F61
:103DF000F2EC5FF003011F0E906FD8EC25F0030189
:103E00008F6F03011F0E8E6FCCEC25F00401050EA1
:103E1000CB6FF2EC5FF00301210E8F6F03018E6B0D
:103E2000CCEC25F00401050ECB6FF2EC5FF0030142
:103E3000080E8F6F03010E0E8E6FCCEC25F0030180
:103E40008F6B03010A0E8E6FCCEC25F003018F6B94
:103E500003010B0E8E6FCCEC25F00301040E8F6F67
:103E600003010C0E8E6FCCEC25F00301020E8F6F58
:103E700003010D0E8E6FCCEC25F02350E96EEA6A3B
:103E8000D890E936EA36660EE926030EEA22EFCF2D
:103E90008FF30301040E8E6FCCEC25F003014C0E62
:103EA0008F6F0301010E8E6FCCEC25F00301600EC5
:103EB0008F6F0301020E8E6FCCEC25F003014C0EC8
:103EC0008F6F0301030E8E6FCCEC25F003018F6919
:103ED0000301070E8E6FCCEC25F003018F6B0301FD
:103EE0000F0E8E6FCCEC25F00301610E8F6F030176
:103EF0008E6BCCEC25F0B5C28FF30301010E8E6FF3
:103F0000CCEC25F0B6C28FF30301020E8E6FCCEC21
:103F100025F0B7C28FF30301030E8E6FCCEC25F0B2
:103F2000B8C28FF30301040E8E6FCCEC25F0B9C23A
:103F30008FF30301050E8E6FCCEC25F0BAC28FF320
:103F40000301060E8E6FCCEC25F00901006B080E04
:103F5000005D14E203018F6900C910F0116A126A52
:103F6000136A080E1026000E11221222132210C00E
:103F70008EF3CCEC25F00901002BE9D703014C0EA0
:103F80008F6F0301070E8E6FCCEC25F04C0E206E68
:103F90000301220E8F6F03018E6BCCEC25F0030121
:103FA0008F6B03010D0E8E6FCCEC25F00301E00E3C
:103FB0008F6F03018E6BCCEC25F00301C00E8F6F69
:103FC0000301010E8E6FCCEC25F003018F6B030112
:103FD000040E8E6FCCEC25F003018F6B0301010EF4
:103FE0008E6FCCEC25F00301200E8F6F03018E6BDA
:103FF000CCEF25F003010D0E906FD8EC25F0106E7C
:10400000116AE85003016E2711506F2303010E0E51
:10401000906FD8EC25F0106E116AE85003017027FC
:104020001150712303010F0E906FD8EC25F0106E24
:10403000116AE85003017227115073231200030123
:10404000745108E00301906BD8EC25F0040B01E0FB
:10405000000C010C6C51235C08E10301906BD8EC5F
:1040600025F0040B01E0000C010C0901010E926F18
:1040700092C910F0116A126A136A030E105C000EE6
:104080001158000E1258000E135811E29251E96EA9
:10409000EA6AD890E936EA36660EE926030EEA2285
:1040A000EE52EF50010B01E0010C922BE1D7000C16
:1040B000030175510BE00301906BD8EC25F0040B64
:1040C00002E1106A01D01068105012000901010EBF
:1040D000926F92C910F0116A126A136A030E105C93
:1040E000000E1158000E1258000E13582AE2925179
:1040F000E96EEA6AD890E936EA36660EE926030EDA
:10410000EA22EE52EF50010B1AE09251E96EEA6A90
:10411000D890E936EA36660EE926030EEA22EE5218
:10412000EF909251E96EEA6AD890E936EA36660E67
:10413000E926030EEA22EE52EF9292511200922BE0
:10414000C8D7FF0C956A6A0E8D6E010E836E8D9C2A
:1041500086A8FED78D8C6B0E8D6E836A8D9C86A88B
:10416000FED78D8C600E8D6E120E836E8D9C86A890
:10417000FED78D8C670E8D6E400E836E8D9C86A84B
:10418000FED78D8C700E8D6E76C383FF8D9C86A8B6
:10419000FED78D8C212A000E2222120003017951B4
:1041A0007A1101E11200010E7915106E116A795130
:1041B00010240901CF6F03017A5111200901D06F3A
:1041C000956A670E8D6E400E836E8D9C86A8FED715
:1041D0008D8C6A0E8D6ECFC983FF8D9C86A8FED70D
:1041E0008D8C6B0E8D6ED0C983FF8D9C86A8FED7FB
:1041F0008D8C600E8D6E120E836E8D9C86A8FED700
:104200008D8C0301795121267A512222700E8D6EF8
:1042100077C3E9FF78C3EAFF772B000E7823EF50CE
:10422000836E8D9C86A8FED78D8C79C3CDF97AC319
:10423000CEF90901010ECD5F000ECE5B0901CDC99B
:1042400010F0CEC911F0CD07000ECE5B105011104A
:1042500001E18BD0080ECD5D000ECE5901E276D083
:10426000030177C3E9FF78C3EAFF772B000E7823B9
:10427000EF50836E8D9C86A8FED78D8C030177C38B
:10428000E9FF78C3EAFF772B000E7823EF50836EA7
:104290008D9C86A8FED78D8C030177C3E9FF78C378
:1042A000EAFF772B000E7823EF50836E8D9C86A853
:1042B000FED78D8C030177C3E9FF78C3EAFF772B24
:1042C000000E7823EF50836E8D9C86A8FED78D8CD0
:1042D000030177C3E9FF78C3EAFF772B000E782349
:1042E000EF50836E8D9C86A8FED78D8C030177C31B
:1042F000E9FF78C3EAFF772B000E7823EF50836E37
:104300008D9C86A8FED78D8C030177C3E9FF78C307
:10431000EAFF772B000E7823EF50836E8D9C86A8E2
:10432000FED78D8C030177C3E9FF78C3EAFF772BB3
:10433000000E7823EF50836E8D9C86A8FED78D8C5F
:10434000080E0901CD5F000ECE5B84D7030177C351
:10435000E9FF78C3EAFF772B000E7823EF50836ED6
:104360008D9C86A8FED78D8C69D71200956A6A0E3F
:104370008D6E010E836E8D9C86A8FED78D8C6B0E84
:104380008D6E836A8D9C86A8FED78D8CFF0E215C76
:1043900031E12250106E116A126A136A5F0E221800
:1043A00029E1115027E1125025E1135023E10901C1
:1043B00093695F0E946F93C991F3E8CF92F3E6ECA3
:1043C00025F0600E8D6E0A0E836E8D9C86A8FED73A
:1043D0008D8C0301100E906FD8EC25F00901926FBF
:1043E000936B4C0E946F93C991F3E8CF92F3E6EC84
:1043F00025F014D0600E8D6E0A0E836E8D9C86A8FB
:10440000FED78D8C9568700E8D6E8D9A86A8FED71E
:1044100083CF92F98D8A212A000E2222090192511E
:1044200012007DC392F97EC393F903017D517E1181
:1044300003E1F36AF46A1200956A6A0E8D6E92C9FE
:1044400083FF8D9C86A8FED78D8C6B0E8D6E93C9D5
:1044500083FF8D9C86A8FED78D8C600E8D6E0A0E14
:10446000836E8D9C86A8FED78D8C090192512126E2
:10447000935122222250116A126A136A600E225C42
:10448000000E1158000E1258000E135802E3140EBD
:10449000225E9568700E8D6E090192C910F093C965
:1044A00011F09207000E935B105011100FE08D9ADF
:1044B00086A8FED703017BC3E9FF7CC3EAFF7B2B01
:1044C000000E7C2383CFEFFF8D8AE6D77DC3F3FFF9
:1044D0007EC3F4FF120081C38CF909018D6B0301C7
:1044E000815103E1F36AF46A1200956A6A0E8D6ED7
:1044F00081C383FF8D9C86A8FED78D8C6B0E8D6E3D
:10450000836A8D9C86A8FED78D8C600E8D6E0A0EF8
:10451000836E8D9C86A8FED78D8C9568700E8D6EEF
:1045200009018C5131E08C078D9A86A8FED783CF84
:104530008EF98D8A03017F51801109E07FC3E9FF65
:1045400080C3EAFF7F2B000E80238EC9EFFF8251CC
:1045500009018E5DE5E1200E8D6F956A600E8D6E0E
:10456000200E836E8D9C86A8FED78D8C6A0E8D6E74
:10457000836A8D9C86A8FED78D8C6B0E8D6E836AA8
:104580008D9C86A8FED78D8C09018C510301815D1D
:1045900009018C6FE850116AE8502126115022223F
:1045A0002250116A126A136A600E225C000E1158C2
:1045B000000E1258000E135802E3140E225E8DC92D
:1045C00010F0116A126A136A200E10180BE11150D4
:1045D00009E1125007E1135005E121C091F322C017
:1045E00092F3F4DA126A09018C5100011210F36E91
:1045F0008DC9F4FF120003018351E96EEA6AD89075
:10460000E936EA36660EE926030EEA22EE52EF900C
:10461000120084C310F0116A126A136A030E105C50
:10462000000E1158000E1258000E13580FE203012D
:104630008451E96EEA6AD890E936EA36660EE926D0
:10464000030EEA22EE52EF8084C323F0120020C052
:1046500097F90901010E966FE8CF91F320C092F30C
:10466000B5DA84DE0901956FE8CF8FF30301030EFD
:104670008E6FCCEF25F00301600E8F6F03018E6B00
:104680008BDA0301070E906F93DA0901006F0301C3
:10469000200E8F6F03018E6B7FDA20500901005DC1
:1046A00026E2600E146E156A166A176A2050186E9C
:1046B000196A1A6A1B6A2050145C106E195015583A
:1046C000116E1A501658126E1B501758136E00C9EF
:1046D0001CF01D6A1E6A1F6A1C5010261D501122F4
:1046E0001E5012221F50132210C001F903D0205077
:1046F000005D016F140E146E156A166A176A01C9FF
:1047000018F0196A1A6A1B6A1850145C106E195056
:104710001558116E1A501658126E1B501758136EFA
:1047200010C001F910C003F9026B02C9F3FF10C0F9
:10473000F4FF12000301E00E8F6F03018E6B2CDA81
:104740000301030E906F34DA0901006F0301200E9C
:104750008F6F03018E6B20DA09010051040B01E019
:10476000000C010C87C3E9FF88C3EAFFEF6803016F
:10477000600E8F6F03018E6B0FDA0301070E906FCF
:1047800017DA0901126F0301200E8F6F03018E6B80
:1047900003DA0301030E906F0BDA0901136F0301B3
:1047A000070E906F05DA100B6BE00301906B00DAD7
:1047B000040B0901166F0301210E8F6F03018E6B2D
:1047C000EBD90401020ECB6FF2EC5FF003018F6BAB
:1047D00003010A0E8E6FE0D903018F6B03010B0EEC
:1047E0008E6FDAD9090116510BE00301070E906FA5
:1047F000DFD90A0B02E0000E01D0010E0901166F8D
:104800000301020E8F6F03010D0E8E6FC5D90301D8
:10481000220E8F6F03018E6BBFD912C920F017DFF4
:1048200003014C0E8F6F0301030E8E6FB5D9030188
:10483000620E8F6F03018E6BAFD903014C0E8F6F29
:104840000301070E8E6FA8D90301220E8F6F03019B
:104850008E6BA2D903018F690301070E8E6F9CD95D
:1048600003018F6B03010D0E8E6F96D9090116514E
:1048700006E00301260E8F6F03018E6B8DD9000CAD
:1048800009011351125D01E19DD013C915F9146B93
:1048900014C991F313C992F399D9120E03017D6FD4
:1048A0007E6B0301000E7B6F090E7C6FBADD090180
:1048B0000051010B01E183D002C910F003C911F0CE
:1048C000126A136A400E105C000E1158000E125846
:1048D000000E135874E302C914F003C915F0166AE8
:1048E000176AD880EE0E1454050E1554000E165497
:1048F000000E175464E301C918F0196A1A6A1B6A9A
:10490000600E185C000E1958000E1A58000E1B5845
:1049100056E201C91CF01D6A1E6A1F6A4C0E1C5C1F
:10492000000E1D58000E1E58000E1F5848E310C9F7
:1049300002F311C903F3F2EC37F0F3CF10F9F4CF1F
:1049400011F9060EE66EE66A0A0EE66E090EE66ECE
:1049500085C3E9FF86C3EAFF85C310F086C311F063
:1049600085C3E6FF86C3E6FF22EC58F0126E060E02
:10497000E15E1250080E0901115D1EE110C910F030
:10498000116A126A136A10501110121013100EE0FF
:1049900010C914F0156A166A176A060E14180CE18D
:1049A00015500AE1165008E1175006E187C3E9FFE8
:1049B00088C3EAFF10C9EFFF13C920F0010C12C928
:1049C00020F045DE000C03010A0E8F6F0301070E75
:1049D0008E6FE2D82350E96EEA6AD890E936EA365B
:1049E000660EE926030EEA22EFCFD2F90901D16B58
:1049F000D1C991F3D2C992F3E9D8060E0301796FB8
:104A00007A6B89C377F38AC378F3CEEC20F0B5C212
:104A100076F3A2EC20F0B6C276F3A2EC20F0B7C297
:104A200076F3A2EC20F0B8C276F3A2EC20F0B9C283
:104A300076F3A2EC20F0BAC276F3A2EC20F08BC39E
:104A400010F0116A126A136A10501110121013102C
:104A500003E10901D36B03D00901060ED36F0301F3
:104A6000080E766FA2EC20F0D3C976F3A2EC20F00A
:104A70000E0E03018C27000E8D238CC310F08DC306
:104A800011F0126A136A3C0E105C000E1158000EF1
:104A90001258000E135803E23C0E8C6F8D6B8CC3C2
:104AA000D1F98DC3D2F98CC38FF30301050E8E6F3C
:104AB00073D8D2C98FF30301060E8E6FCCEF25F0A9
:104AC0002350E96EEA6AD890E936EA36660EE9269E
:104AD000030EEA22EFCF8FF30301040E8E6F5CD832
:104AE0000301240E8F6F03018E6B56D823C06CF325
:104AF0002350E96EEA6AD890E936EA36660EE9266E
:104B0000030EEA22EE52EF802350E96EEA6AD89053
:104B1000E936EA36660EE926030EEA22EE52EF8205
:104B20000901926B92C910F0116A126A136A030E9E
:104B3000105C000E1158000E1258000E135818E2A7
:104B40009251E96EEA6AD890E936EA36660EE926AD
:104B5000030EEA22EE52EF50010B07E092510301DF
:104B60006C5D03E092C923F012000901922BDAD7A1
:104B700012009568600E8D6E8D8C8D8A8D8E966A72
:104B80000401010ECA6FE5EC5FF00401050ECB6F66
:104B9000F2EC5FF08D9E1200600E03018E118D6E9F
:104BA0008FC383FF956A8D9C86A8FED78D8C1200DB
:104BB0009568600E030190118D6E8D9A86A8FED7C0
:104BC00083CF98F98D8A09019851120091C321F081
:104BD00092C322F091C38FF30301080E8E6FDCDFC6
:104BE00092C38FF30301090E8E6FCCEF25F0030102
:104BF000090E906FDDDF0901016F0301080E906F50
:104C0000D7DFF36E01C9F4FF120020C093F9090148
:104C1000120E926F030193510901922703019451DF
:104C20000901932392C991F393C992F3E6EF25F01A
:104C300095C323F02350E96EEA6AD890E936EA3644
:104C4000660EE926030EEA22EFCF93F909010E0E54
:104C5000926F0301965109019227030197510901AF
:0E4C6000932392C991F393C992F3E6EF25F0E6
:024C6E00A1C4DF
:104C70003CFFA2C43DFF0901036B060E035D2DE25C
:104C8000750E8BEC2CF0116E106A10C0E6FFE66E0C
:104C9000740E8BEC2CF0E552E7CF11F0E552E7CF24
:104CA00010F000011010626F11C063F04BEC12F0B5
:104CB000E66E0901DCEC2BF0E552E750EF6EDCEC20
:104CC0002BF0020EA9EC2BF0EF6ADCEC2BF0090EB6
:104CD000A9EC2BF0EF6A032BD0D712000901D56B9A
:104CE000060ED55D06E2D5C943FF96D80901D52B3E
:104CF000F7D712003ECF00F93FCF01F9090100C9F3
:104D0000E9FF01C9EAFF002B000E0123EF502E0836
:104D100007E000C9E9FF01C9EAFFEF50EFE10A0C23
:104D2000026B0251106E116A100E105C000E1158C9
:104D300021E230EC2CF002C916F0176A186A020E54
:104D4000D890163617361836E806FAE1B5EC2BF08F
:104D500000C9E6FF01C9E6FF87EC58F0196E050EA1
:104D6000E15E1950000903E1090102511200090135
:104D7000022BD7D70A0C04EC2CF004E0200E09011A
:104D8000005DF9E00901016B2B0E0901005D02E1F4
:104D9000200E006F2F0E005D20E05C0E005D1DE018
:104DA000200E005D1DE03F0E005D1AE00D0E005D5F
:104DB00017E00A0E005D14E00C0E015D0EE2610EBC
:104DC000005D05E300517A0802E3200E005F015107
:104DD000012B37EC2CF000C9EFFF04EC2CF0D4E1F0
:104DE0000901015137EC2CF0EF6A090101510EE184
:104DF000550EE66EBE0EE66E000EE66E41CFE6FF85
:104E000042CFE6FF9DEC58F0050EE15E3F0E090132
:104E1000005D01E1010C000C0F0143510A0DF3CFBD
:104E2000C5F9F4CFC6F9000E0901C5270F0EC62338
:104E3000010EC36F0901C35101E143D2C36BCC6BB7
:104E4000A4EC2BF03EEC2CF00DE1BAEC2CF0020BB4
:104E500002E0B5EC2CF05CEC2CF0EF9460EC2CF064
:104E6000EF6A1200A4EC2BF0020EEB50080AE2E00D
:104E70000F0A01E112D2010A01E1E2D1030A01E1C4
:104E8000DFD1010AD7E0070A01E103D2010A01E1FB
:104E9000B7D1030A01E172D1010ACCE1A4EC2BF0F5
:104EA0004BEC2CF0C7E00901010EC36FA1C43CFF1D
:104EB000A2C43DFF5CEC2CF0EF6A97EC2CF00F01E4
:104EC000496F5CDA0901C26F0F01B50E416F090E1F
:104ED000426F97EC2CF00F01406F4DDF0901CC9130
:104EE000E8B0CC8197EC2CF00001AD6F23EC1CF006
:104EF000F3CFCAF9F4CFCBF90F01B50E516F090EFC
:104F0000526F43CF50FF95DB0F01B50E3E6F090E78
:104F10003F6FF0DEE66E5AEC2CF0E552E750EF6E94
:104F2000AEEC2CF0060E101805E1115003E1125002
:104F300001E113502CE05AEC2CF0EFCF14F0156A7D
:104F4000166A176A010E141805E1155003E1165090
:104F500001E1175002E0000E01D0010E000E000921
:104F600016E15AEC2CF0EFCF18F0196A1A6A1B6A96
:104F7000040E181805E1195003E11A5001E11B5005
:104F800002E0000E01D0010E000E000904E05CEC0E
:104F90002CF0EF8003D05CEC2CF0EF90E3DB020B05
:104FA00025E1AEEC2CF0060E101809E1115007E1D6
:104FB000125005E1135003E1D5DB100B17E1580E39
:104FC0000901B55D03E1CEDB010B10E1BAEC2CF079
:104FD000010B03E0C7DB080B09E1C4DB040B0DE0A8
:104FE0000901C2510AE1CC51010B07E0BAEC2CF0E7
:104FF000040B03E19EEC2CF03CD00901C25101E00E
:10500000B7D05CEC2CF0CC93EF50040B01E0CC83D8
:10501000A9DB200B03E15CEC2CF0EF840901CCA1AF
:1050200015D0CAC9ABF0CBC9ACF097EC2CF000019D
:10503000AA6FEBEC1BF00401B50E936F090E946F91
:10504000C5C991F4C6C992F403EC5AF05CEC2CF09B
:105050000901CC51020B02E0EF8401D0EF949EECE9
:105060002CF0BAEC2CF0100B0CE0BAEC2CF0040B8A
:1050700008E1ACEC2CF0020EEF6E66DB6ADB060E8C
:105080000AD160EC2CF0050EEF6E66EC2CF0A1EC72
:105090002CF0060ED5DB46E3AEEC2CF0D880040EE7
:1050A000D7DB40E3B50EE66E090EE66EB6EC58F0BF
:1050B000E552E552F3CFC4F9AEEC2CF0D880030EE4
:1050C000C7DB02E3030E01D0020E0901C45FAEECA0
:1050D0002CF00B0E1026000E112212221322EADBF6
:1050E00010C0EFFFBDDBE6DBEFCF16F0176A186AE2
:1050F000020ED890163617361836E806FAE135DB78
:105100000901C4511A6AB50F196E090E1A2219C085
:10511000E6FF1AC0E6FF9DEC58F01B6E050EE15E3F
:105120001B50D4DBA1EC2CF0E86810180AE11150F8
:1051300008E1125006E1135004E1ACEC2CF0EF6AE8
:105140000FD0A1EC2CF0FE0E10180DE111500BE168
:10515000125009E1135007E1ACEC2CF0010EEF6E98
:10516000AFDB050E98D0A8DBEF82AADB010E93D04F
:10517000C20501E05FD6A4DB030E8DD0E5DB01E1C3
:1051800059D60901010EC36F0F01DE0E4D6FBD0E22
:105190004E6F000E34DB8ADB0F01EE0E4D6FBD0E3D
:1051A0004E6F000E2CDB86DB7DDBC20EE926010E86
:1051B000EA22EECF4DFFEECF4EFFEFCF4FFF43CFB2
:1051C0004CFF0DDA73DBCADB0B0E3ADB07E30F0192
:1051D000FD0E4D6FBD0E4E6F000E11DBCBDB010BD4
:1051E00007E10F01780E4D6F930E4E6F000E07DB37
:1051F0005DDBAADA030EADDAEF6A62DB020E4BD09A
:10520000A3DA49DB01E09ADB57DB0901CC93EF50CD
:10521000040B01E0CC83A6DA200B02E14DDBEF8426
:1052200043CF4AFFEED8000904E09FDB49DB070EBD
:10523000EF6E42DB0901CC51020B41E0EF84FAD55D
:1052400083DB01E1F7D588DB2DDBF20EE926010EC9
:10525000EA22EECFC7F9EECFC8F9EFCFC9F90901BD
:10526000C7C9F6FFC72BC8C9F7FF000EC823C9C9B5
:10527000F8FFC9230800F5CFC4F9F55005E0C4C90B
:105280006DF062DAACDAEBD752DB00016A6F61ECE9
:1052900013F016DB070EEF6ECDD556DAEFDA0AE023
:1052A00053DB08E044DB0001696F1EEC13F008DB00
:1052B000080EEF6E49DA090EE926000EEA22EF9495
:1052C000B9D5120047CFE9FF48CFEAFFEF04090143
:1052D0004A6F496BEF6A4B6B4A510F01EA6A4525E9
:1052E000E96E4651EA22EF6A09014B5141E10001A2
:1052F000480E7F6F090E806F44CF7EF0ABEC15F047
:10530000000936E03D0E0901485D0BE1486B4A514A
:10531000495D1EE2492947CFE9FF48CFEAFFEF6E1A
:1053200017D0260E485D02E1020E0AD0200E485D1D
:1053300006E00D0E485D03E00A0E485D04E1010E33
:105340004B6F486B05D02B0E485D02E1200E486F75
:105350004A51495D06E245CFE9FF46CFEAFF48C919
:10536000EFFF0F01452B000E46230901492BBCD747
:1053700009014B5101E1000C4B0512000901056BBD
:105380000001060E7F6F090E806F49CF7EF0ABECF7
:1053900015F0000916E0200E0901065D12E0055126
:1053A000106E116A040E105C000E1158E9E20551EE
:1053B000052BEA6A000FE96E090EEA2206C9EFFF23
:1053C000DFD709010551EA6A000FE96E090EEA22EA
:1053D000EF6A470E005D07E1450E015D04E1540EE2
:1053E000025D01E1000C500E005D0AE14F0E015D0F
:1053F00007E1530E025D04E1540E035D01E1010C6F
:10540000020C0F014A510A0DF3CF6EF9F4CF6FF978
:10541000000E09016E270F0E6F239FD9D9D901E124
:10542000C3D009016C6B99D9030EEB5004081AE044
:1054300094D9DAD9400EF8D90EE18FD9010EEB508C
:105440000D01F16F44EC46F009016D6F86D9CCD99E
:10545000200EEAD907E081D9EF5000016A6F61ECB4
:1054600013F0010C7AD9090E74D9EF50010B01E148
:1054700094D073D9030EEB50040A64E0070A35E0B8
:10548000010A1CE0030A0CE0010A01E084D0250EA9
:105490006D5D03E12BDA010E26D0010E6C6F7BD01F
:1054A000250E6D5D03E1010E6C6F73D00DDA030EF6
:1054B00050D96DC9EFFF1ADA020E15D0610E6D5D7D
:1054C00002E3270E04D0410E6D5D02E3070E6D5F0F
:1054D000300E6D5D100DF350E66E43DAE552E75085
:1054E000EF6E04DA030EEF6E56D0610E6D5D02E3CF
:1054F000270E04D0410E6D5D02E3070E6D5F300E86
:105500006D5D106E2EDA1050EF12F0D9040EEF6EB2
:1055100024D91FD9EE6AED6A726B736B22DAEFCF72
:1055200070F9D2D9030E15D9EFCF71F96D0E746FE2
:10553000090E756F6EC953FF6FC954FFFCD809017E
:10554000766F29D0C1D9EECF72F9EDCF73F903018F
:10555000700EA56F090EA66FC9EC0DF0B5D972C912
:10556000EEFF73C9EDFF0901010E6C6F72C910F0F7
:1055700073C911F0126A136AE86810180CE1E86840
:10558000111809E1125007E1135005E16D5101E1D5
:105590006C6BACD9EF6A6C5104E06DC96DF0DDD86D
:1055A0001ED935EC48F039D7D8D8010EEB500D0193
:1055B000F06F16EC46F0000C0F014B510A0DF3CFC3
:1055C0006CF9F4CF6DF9000E09016C270F0E6D23F5
:1055D00000010D0EA5D900010A0E90EF2CF00F016D
:1055E0004C510A0DF3CF6CF9F4CF6DF9000E09019F
:1055F0006C270F0E6D234DCFF6FF4ECFF7FF4FCF29
:10560000F8FF0800F55014E00F014DCFF6FF4D2BC9
:105610004ECFF7FF000E4E234FCFF8FF4F23080069
:10562000F5CF6DF06CC9E9FF6DC9EAFFD8D8E3D7B3
:1056300012000F0150510A0DF3CF00F9F4CF01F918
:10564000000E090100270F0E0123040E836F0001D5
:105650000A0EA5D805E1115003E1125001E11350E3
:1056600006E00901835183070009F1E112000001FE
:105670000D0E7D6F0001800E7C6F0001020E7A6FAF
:10568000090E7B6F37D9F3CF85F9F4CF86F9F4CFC4
:1056900010F050D9F45011101210131015E1090137
:1056A000040E836F00010D0E7AD805E1115003E15D
:1056B000125001E1135005E00901835183070009ED
:1056C000F1E10901200E866F86C910F033D9200E52
:1056D000101805E1115003E1125001E1135001E0EF
:1056E00012000901850501E112000001830E7F6FA0
:1056F000090E806F00C9E9FF01C9EAFFEF50000100
:105700007E6FABEC15F009018505EA6A020FE96EC0
:10571000090EEA22EF6A51CF82F452CF83F40401DA
:10572000020E806F090E816F00C97EF401C97FF4FB
:1057300014EC49F09CD7E7D8040B05E0E4D8080B3B
:1057400001E0020C010C000CC5C9E9FFC6C9EAFF63
:105750001200E926000EEA2212006EC9E9FF6FC9A5
:10576000EAFF1200720E8BEF2CF013501624F36E2A
:1057700014501720F46E15501820F86EF4CFF7FF70
:10578000F3CFF6FFF6CF10F0F7CF11F0F8CF12F00D
:1057900010C0E6FF11C0E6FF12C0E6FF12007D6FE9
:1057A00000017C6900017A6B7B6BA4D8F4CF10F008
:1057B000C1D8200EF418120003510A0DC8D8000EEB
:1057C000E9260F0EEA221200EFCF10F09AEF2CF02C
:1057D000EF5000016B6FB7EC13F000091200EF50AF
:1057E00000016C6FE2EF13F0010EEB50080DAFD823
:1057F000B90EE9260D0EEA22EFCF10F012004F6F1E
:1058000043CF4CFFEFEF2AF00001000E7F6F090E2F
:10581000806F40CF7EF0ABEC15F000091200010E56
:10582000EB50106E9AEF2CF0101684D81050111017
:10583000121013101200EF500001736FCFEF14F02D
:10584000105C000E1158000E1258000E1358120072
:105850001054000E1154000E1254000E1354120076
:105860009E0E136EBD0E146E000E156E12000F010B
:10587000EA6A4125E96E4251EA221200EF50000126
:10588000686F15EC13F000091200010EEB500D01CA
:10589000EF6F0EEF46F0EF500001816FEAEC15F06C
:1058A00000091200EF50030DA7EF2CF043CF4BFF80
:1058B000DCEF2AF051D861D047DF090EA9EF2BF0B9
:1058C00043DF020EA9EF2BF048DF57D00D01EE6B3E
:1058D0000D01B50EEC6F090EED6F5AEC45F0E66E5A
:1058E00033DFEE52E552E750EF6E120036DF030E63
:1058F000A9EF2BF000C9E9FF01C9EAFFEF50000151
:10590000796F3CEF15F053CFE9FF54CFEAFF090E52
:1059100020DFEF5012000201DB6FDC6BA7EF3DF0E0
:105920006D6F6CC9E9FF6DC9EAFFEFEF2BF00CDF7B
:10593000EF501200116A126A136A120005DF1BEFA2
:105940002CF002DF0FEF2CF0FFDEE8EF2BF0F3CFAF
:10595000E9FFF4CFEAFF1200F7DE0FD0ABDFE4EF90
:105960002BF0B2DF020EA9EF2BF0A6DFEF92ECDEF8
:1059700045EF2CF0A1DFEF501200040EA9EF2BF041
:105980000901006B080E005D06E200C9A7F151D8BD
:105990000901002BF7D712000901000E5B6F010E01
:1059A0005C6F5A6B080E5A5D43E25EDB0C0E49DBFE
:1059B0004CDB126A136A105011101210131032E1EE
:1059C00053DB0C0EA1C1EBFF0D0EA2C1EBFF0101D9
:1059D000A351A41111E00A0EE66EE66AA3C1E6FF28
:1059E000A4C1E6FF41DB5BC910F05CC911F05BC9E3
:1059F000E6FF5CC9E6FF63DB37DB0A0EA5C1EBFF00
:105A00000B0EA6C1EBFF30DB0E0EEB6A0F0EEB6A3E
:105A10002BDB100EEB6A110EEB6A5AC9A0F10901DB
:105A20005A511200140E5B27000E5C235A2BBAD772
:105A3000FF0C0101A751FBDA0C0E03DBEE6AED6AE5
:105A4000A751F5DA060EFDDAEE6AEE6AEE6AEE6A44
:105A5000A7515DDBEF901200080E0101A85D07E27F
:105A6000A8C1A0F10301010E746F1FEF20F0000C1C
:105A70000101A051140DF3CF59F9F4CF5AF9000EDA
:105A800009015927010E5A234ADBEE50ED1016E1A9
:105A90001DDBEFDA48DBEDDA120EEB50106EF3DAB5
:105AA00007E1115005E1125003E1135001E1000C30
:105AB0001C0E0301966F976BDCDAFBDAA9C176F353
:105AC000A2EC20F02CDBEE2AEF2229DBBEDAE6DAAC
:105AD00001E374D8010C0101A051140DF3CF41F979
:105AE000F4CF42F9000E09014127010E422313DBD6
:105AF000EE50ED1018E1EADAADDA15DBABDA120E92
:105B0000EB50106EC0DA09E1115007E1125005E1C7
:105B1000135003E1F36AF46A12001C0E0301966F3E
:105B2000976B98DAC6DAF7DA0101AC51EE24106E01
:105B3000AD51EE20116E126A136AD880D60E105441
:105B4000030E1154000E1254000E13541DE2D60E13
:105B5000146E030E156E166A176ADDDAEECF18F0B2
:105B6000EFCF19F01A6A1B6A1850145C106E1950A6
:105B70001558116E1A501658126E1B501758136E86
:105B800010C0ACF111C0ADF1ACC179F3ADC17AF385
:105B9000AAC177F3ABC178F3CEEC20F0BCDA0101F7
:105BA000AC51EE26AD51ED22B6DA4FDA77DA01E3E9
:105BB00005D8ACC1F3FFADC1F4FF12000301010E23
:105BC000746F1FEC20F0000903E135EC48F0F6D7C4
:105BD0000101A051140DF3CF57F9F4CF58F9000E7D
:105BE00009015727010E58233ADA0C0E2ADA75DA22
:105BF000F3CF4FF9F4CF50F932DA0A0E22DA6DDA28
:105C0000F3CF51F9F4CF52F92ADA0E0E1ADAEECFA9
:105C100053F9EFCF54F9080E09015327000E54230E
:105C2000556B566B140E0301966F976B18DA41DAB9
:105C300053C945F454C946F40401110E446F0FDAF8
:105C400057C942F458C943F4E4EC4DF053C902F388
:105C500054C903F3F2EC37F0F3CF53F9F4CF54F90E
:105C6000080E0301796F7A6B03014F0E776F090EEF
:105C7000786FCEEC20F060EC25F0F1D9120EE1D96E
:105C8000EF68EDD90E0EEB6A0F0EEB6A1200080EEC
:105C90000101AE5D0AE2AEC1A0F134DAD880EE5463
:105CA000000EED5401E3000C010C000C080E010184
:105CB000AF5D09E2AFC1A0F125DAC7D910C0F3FF8B
:105CC00011C0F4FF1200F36AF46A120036DA01E13F
:105CD000000CA0511CDAEF50010B01E032DAB6ECF7
:105CE00021F0B0C1E9FFB1C1EAFFEF6E30DAEE0694
:105CF000EF5A08DAEE50ED1002E127EC23F0010C28
:105D00001CDA03E1F36AF46A1200A05100DAEF50E2
:105D1000010B01E016DA1BDA98D9B451105CB551C9
:105D2000115805E2EFD9EECFB4F1EDCFB5F1B4C122
:105D30007DF3B5C17EF3B2C17BF3B3C17CF311EC4B
:105D400022F0F3CF41F9F4CF42F901DA09014151D0
:105D5000EE5E4251ED5AF1D902E127EC23F0B4C1D5
:105D6000F3FFB5C1F4FF1200E8D902E027EC23F0FD
:105D7000EED9EE6AED6A1200080E03017D6F7E6BAC
:105D80000301460E7B6F090E7C6F11EC22F046C9B1
:105D90005DF947C946F95DC947F948C95DF949C97F
:105DA00048F95DC949F9080E106E09014B51D880B8
:105DB000105403E24A055D6F02D04AC95DF9080E2E
:105DC0004B5D4A6F5DC94BF94C514D116AE04CC9AE
:105DD0005DF94DC94CF95DC94DF9B6C1E9FFB7C1CF
:105DE000EAFF060E2ED9EECF4FF9EECF50F9EECFE7
:105DF00051F9EFCF52F977D9EFCF53F9010E21D9ED
:105E0000EFCF54F970D9020E1CD9EFCF55F96BD9E9
:105E1000030E17D9EFCF56F9576B110E586FBAC151
:105E200059F9BBC15AF9BAC102F3BBC103F3F2EC91
:105E300037F0F3CF59F9F4CF5AF90C0E03010A6F7A
:105E40000B6B03014F0E086F090E096F26EC38F03B
:105E5000F3CF5BF9F4CF5CF909015B1F5C1F060E01
:105E600018D95BC976F3A2EC20F0070E12D95CC9F1
:105E700076F3A2EC20F00401476B486B53EC4EF034
:105E8000BAC10CF3BBC10DF392EC38F0F3CF5BF960
:105E9000F4CF5CF909014C51F3181CE14D515C1928
:105EA00019E1B8C1C0F1B9C1C1F1B6C1BEF1B7C104
:105EB000BFF10101460EBC6F090EBD6F22D809016A
:105EC0004E6F106EE0D809E1115007E1125005E164
:105ED000135003E127EC23F0010C4E51A8D8100E0B
:105EE000B0D84AC9EEFF4BC9EDFF4E5110D9EF8033
:105EF000010C0101A0519BD8E9CFF3FFEACFF4FFD9
:105F0000120009010169000E026F010E036F006BA0
:105F1000080E005D5BE2B2D80C0E0BD9020E91D8D0
:105F2000ECD80001125010184AE11350111847E143
:105F3000A5D80A0EFED8E1D8125010183EE1135031
:105F400011183BE19BD8100E7CD8EECF14F0EFCFA8
:105F500015F0166A176A14501510161017102DE157
:105F6000BEC1E9FFBFC1EAFF060E6BD8EECF10F04D
:105F7000EECF11F0C2D882D8060E63D8EE501018BA
:105F800008E1EE50111805E1EE50121802E1EE5052
:105F9000131810E0C0C1E9FFC1C1EAFFE868EE18BC
:105FA0000CE1E868EE1809E1E868EE1806E1E86837
:105FB000EE1803E109010051120000C901F90901BD
:105FC000140E0227000E0323002BA2D701C910F0E4
:105FD0005AD805E1115003E1125001E1135024E0B9
:105FE0000151140DF3CF02F9F4CF03F9000E02278B
:105FF000010E03230A0EE66EE66ABEC1E6FFBFC1CC
:10600000E6FF3CD802C910F003C911F002C9E6FF4F
:1060100003C9E6FF54D86CD818D830D80A0E10C07F
:10602000EBFF0B0E11C0EBFF090101511200140D23
:10603000F3CFE9FFF4CFEAFF000EE926010EEA22D2
:106040001200E926000EEA221200EECF10F0EFCF88
:1060500011F0120041C9E9FF42C9EAFF120057C915
:10606000E9FF58C9EAFF12005BC9E9FF5CC9EAFF12
:10607000120059C9E9FF5AC9EAFF120002C9E9FF33
:1060800003C9EAFF1200116A126A136AE86810185D
:1060900012000401476F486B53EF4EF0126A136A07
:1060A000D60E105C030E1158000E1258000E135835
:1060B0001200120EEB500301956F18EF26F022EC40
:1060C00058F0126E060EE15E125012000301010E2E
:1060D000756F58EC20F0E66E1200EECF02F3EDCFB4
:1060E00003F3F2EF37F0B8C1E9FFB9C1EAFF1200DC
:1060F000BCC1E9FFBDC1EAFF1200EECF12F0EFCF45
:1061000013F01200A05193DF100E21EF30F08FDF5B
:10611000130E21EF30F09EDF0E0E21EF30F0A9DFDD
:106120000E0E21EF30F0120E8CDFE552E750EF6ECD
:10613000120087DF8ADF78EF30F009D8EE50ED10DB
:106140001200A051E4DFEF90080E49EF30F001019A
:0461500082EF30F0BA
:0C6154000401C05101E112007DDB05E1F7
:10616000115003E1125001E1135002E0020E01D080
:10617000010EC06FC36BC19112006EDB05E11150BF
:1061800003E1125001E1135001E053DB0401C06B45
:106190006DDBFE0B2FEF34F00401C05108E166DB2C
:1061A00001095DDB0401010EC06FC36BC1911200D8
:1061B0000401C051080A01E1E1D0020A01E1DED088
:1061C000060A01E1DBD00B0A01E1C9D00E0A01E1A8
:1061D000C6D0020A01E1C3D00D0A01E19DD0030A35
:1061E00062E0010A56E0070A42E0010A0EE0030AF3
:1061F00001E01200FBDA07E1115005E1125003E162
:10620000135001E11200020EC06F1ADB01E112000F
:106210000A0EE66EE66AE6680401C251140DF3CF79
:10622000E9FFF4CFEAFF000EE926010EEA22E9CFEA
:1062300010F0EACF11F0E9CFE6FFEACFE6FF4DEC30
:1062400058F0126E050EE15E125004013C0E226FF2
:10625000236B246B256B326B0401C36BC191C1931B
:106260000401386B0401010E1DDB030E07D0B1DA07
:1062700007E287DA01E2A5D00401020EC06F120026
:106280000401C1859FD8020801E012000401040E38
:10629000C06FD6DA01E112000401386B0401030E6D
:1062A00001DB050E07D095DA07E26BDA01E289D04F
:1062B0000401020EC06F120085D8060A29E0030A05
:1062C00001E01200B6DA7CDA060EC06FC181C32B82
:1062D000040132A108D026C4B1F227C4B2F228C406
:1062E000B3F229C4B4F232A508D02EC4BBF22FC435
:1062F000BCF230C4BDF231C4BEF232A30CD02AC409
:10630000BFF22BC4C0F22CC4C1F22DC4C2F21200E1
:106310000401020EC06F120034DA01E21200020E14
:106320000401225D000E2359000E2459000E255948
:106330000BE3640E3327000E342335233623220764
:10634000235B245B255B120051DA07E1115005E164
:10635000125003E1135001E11200070EC06F70DA12
:1063600001E112000401010E386F0401030E376FC2
:1063700057D90401C19324DAC02B12002ADA12E2A1
:1063800000DA1FE30401C02B0C0EE76EC019E8AE63
:1063900002D0C03503D0E750D880C05512E2020EBB
:1063A000C06F12000FD8060A08E0030A01E01200CD
:1063B00040DA06DAC32B060E02D00401020EC06FCB
:1063C000120012000901036BD6D9020E0901005D0B
:1063D00001E0FFD0016B0F0E015D02E257DAFBD73F
:1063E0000401C1A307D00901016B040E015D08E29D
:1063F0004DDAFBD72BDA260EB26F040E42DA328169
:106400000901016B080E015D02E240DAFBD7016B66
:10641000060E015D0EE2AFD909010151EA6AB50F1E
:10642000E96E020EEA22EF50005D01E0F6D0012B8A
:10643000EFD7016BCE0E015D02E228DAFBD7046BC9
:106440009AD9000904E10901010E046FC2D00901C3
:106450000051330A01E171D0CC0A6CE0C90A55E061
:10646000350A2FE0020A18E0340A01E09DD083D9F2
:106470000901000501E0D1D00101030EB06F090E42
:106480000EDA0401C151020B01E19DD0020E090197
:10649000035D01E098D0C1D0FDD901E0BED0040178
:1064A000C1A308D00901016B040E015D01E38BD08B
:1064B000EDD9FAD7CBD92E0EB26F040EE2D93285C0
:1064C00082D00101020EB06F090EE9D9040E090154
:1064D000025D01E2A2D00401C1A307D00901016B52
:1064E000040E015D08E2D2D9FBD7B0D92A0EB26FF3
:1064F000040EC7D93283040E0901025F090102515B
:106500000207000960E037D9F9D7C4D901E085D086
:106510000101080EB06F090E7ED9070EB06F090E8B
:106520007AD9060EB06F090E76D9050EB06F090E36
:10653000B6D949D0010E046F46D0ACD96EE1040142
:10654000C1A307D00901016B040E015D3CE29ED995
:10655000FBD70101250EB06F040E5DD9240EB06F7C
:10656000040E59D9230EB06F040E55D9220EB06F08
:10657000040E95D922C410F023C411F024C412F0E3
:1065800025C413F0050ED890133212321132103296
:10659000E806F9E110500401225F1150235B12500C
:1065A000245B1350255B0FD00101020EB06F090E62
:1065B00076D9090102510207000905E00101000E28
:1065C000B06F090EF5D735EC48F00901045101E12F
:1065D00037D7020E035D0BE105C91EF406C91FF48F
:1065E00007C920F408C921F40401C18311D01E0E8B
:1065F000E96E040EEA6EEE50051908E1EE50061938
:1066000005E1EE50071902E1EE50081901E0036BB5
:10661000B4EC2EF0090103511200B4EC2EF0000C82
:106620000101010EC8D8010EC6D8060EC4D84AD939
:106630000101120EC0D8230EBED8340EBCD8560E9F
:10664000BAD8E5D80101800EB6D83CD9030E0401B2
:10665000375D04E1385102E0E1D804D00101D7D818
:106660000101D5D80901006B0C0E005D02E204D9CE
:10667000FBD7060E0101AC6FAD6B0101B50EAA6F21
:10668000020EAB6F6BEC2DF00901006BCA0E005DC2
:1066900002E2F2D8FBD70101630E8DD8820E8BD8AF
:1066A000530E89D8630E87D8350E85D8010EA96F91
:1066B00038EC2DF037C4A9F138EC2DF00401370582
:1066C00002E10401C193030E0401375D15E1385165
:1066D00013E10101360EEBD821C4A9F138EC2DF0FD
:1066E00020C4A9F138EC2DF01FC4A9F138EC2DF02D
:1066F0001EC4A9F138EC2DF00101370E5CD8040E50
:106700005AD8010E58D8030E56D8060E54D80C0E7F
:10671000A96F38EC2DF0030E0401375D02E138510A
:1067200007E0370509E1265127112811291104E056
:106730000101320EBCD872D80101A96938EC2DF0E4
:10674000B1C201F9B2C202F9B3C203F9B4C204F989
:106750000401385105E10201B16BB26BB36BB46B4C
:10676000DEEC2DF001C9B1F202C9B2F203C9B3F2F5
:1067700004C9B4F212000101000EB06F090E4FEF10
:1067800034F0330EE96E040EEA6EEE500401A15DA2
:10679000106EEE50A259116EEE50A359126EEE50CB
:1067A000A459136EC80E105C000E1158000E12583A
:1067B000000E13581200A96F38EC2DF001011200E1
:1067C000A1C433F4A2C434F4A3C435F4A4C436F48D
:1067D0001200C2C4AFF156EC2EF0F3CF10F0F4CF9C
:1067E00011F0FA0EF35C000EF4581200430E010192
:1067F000A56FA66B0101A36BA46B440E0101A16FF1
:10680000A26BCCEC2CF00401C26F106E55D05AD89C
:10681000010162EF34F043D801011200040E0101BE
:10682000AC6FAD6B0101260EAA6F040EAB6F6BEF60
:106830002DF0C2C4A7F119EC2DF00401C2691200B9
:10684000C2C4A8F12CEC2DF000091200040E0101C5
:10685000B46FB56B01011200C2C410F02DD0A86E48
:10686000160E0201DD6FDE6BB8EF3DF0160E020171
:10687000DB6FDC6BA7EF3DF0010124D80901002B91
:106880001200B36F80EC2EF00401120074DF0901D6
:10689000012B120070DF040E0901005D1200B16FC0
:1068A00066EF2EF0376FBCDE8BDF0401120083DF52
:1068B000040EA96F38EF2DF0116A126A136AE868A6
:0A68C00010181200A96B38EF2DF03C
:0668CA0094909492949456
:1068D000938093829388938A0201010E036F046B65
:1068E000056B006B016B026B066B09014F6B050EAC
:1068F0004F5D0EE232DBEE6AED6A2FDB020E3FDB0C
:106900002CDB040E3CDB29DB060E39DB4F2BEFD7EB
:1069100002013A6B3B6B0301FC6BFD6B0301FE6BE9
:10692000FF6B12008150010B106E02010151200B10
:1069300001E0010E105C06E18150010B02E0019BB9
:1069400001D0018B8150020B01E0010E106E01514C
:10695000800B01E0010E105C06E18150020B02E0A9
:10696000019F01D0018F8150100B01E0010E106ECC
:106970000151100B01E0010E105C06E18150100B7B
:1069800002E0019901D001898150200B01E0010E44
:10699000106E0151400B01E0010E105C06E18150C8
:1069A000200B02E0019D01D0018D8050010B106E83
:1069B0000051800B01E0010E105C05E0009F80504B
:1069C000010B01E0008F8050020B01E0010E106E00
:1069D0000151020B01E0010E105C05E001938050B3
:1069E000020B01E001838050040B01E0010E106EE8
:1069F0000151080B01E0010E105C05E00197805089
:106A0000040B01E001878050080B01E0010E106EBD
:106A10000051400B01E0010E105C05E0009D80502C
:106A2000080B01E0008D8050200B01E0010E106E7C
:106A30000151010B105C05E001918050200B01E039
:106A400001818050100B01E0010E106E0151040B0A
:106A500001E0010E105C05E001958050100B01E093
:106A60000185000EE96E020EEA6EEE50031905E193
:106A7000EE50041902E1EE50051928E08B9409014B
:106A8000016B030E015D18E2800E006F8B920151C5
:106A9000EA6A000FE96E020EEA22EF50001502E0EA
:106AA0008B8001D08B908B82000503E18B92012BB0
:106AB000E8D700417F0BE9D78B848B94949A8B9A0B
:106AC00000C203F201C204F202C205F29250010BAD
:106AD00019E050DA010E37DA15E18050010B36DA91
:106AE000010E31DA02E1000E01D0010E025D0AE072
:106AF0000301FE810901025103E00301FC8102D080
:106B00000301FC919250020B1BE034DA020E1BDAF7
:106B100017E18050020B01E0010E18DA020E13DAC1
:106B200002E1000E01D0010E025D0AE00301FE83C6
:106B30000901025103E00301FC8302D00301FC932D
:106B40009250040B1BE016DA040EFDD917E18050B9
:106B5000040B01E0010EFAD9040EF5D902E1000E92
:106B600001D0010E025D0AE00301FE850901025118
:106B700003E00301FC8502D00301FC959250080B51
:106B80001BE0F8D9080EDFD917E18050080B01E0AF
:106B9000010EDCD9080ED7D902E1000E01D0010E9A
:106BA000025D0AE00301FE870901025103E00301CF
:106BB000FC8702D00301FC979250200B1BE0DAD92E
:106BC000100EC1D917E18050200B01E0010EBED993
:106BD000100EB9D902E1000E01D0010E025D0AE0EB
:106BE0000301FE890901025103E00301FC8902D07F
:106BF0000301FC999250100B1BE0BCD9200EA3D9C5
:106C000017E18050100B01E0010EA0D9200E9BD996
:106C100002E1000E01D0010E025D0AE00301FE8BCD
:106C20000901025103E00301FC8B02D00301FC9B2C
:106C30009350010B1AE09ED9400E85D916E1815080
:106C4000010B010A83D9400E7ED902E1000E01D06A
:106C5000010E025D0AE00301FE8D0901025103E00D
:106C60000301FC8D02D00301FC9D9350020B1CE03C
:106C700081D9800E68D918E18150020B020A01E027
:106C8000010E64D9800E5FD902E1000E01D0010E21
:106C9000025D0AE00301FE8F0901025103E00301D6
:106CA000FC8F02D00301FC9F9350100B20E0FFC328
:106CB00011F0126A136A106A010E5AD918E1815054
:106CC000100B100A01E0010E60D9010E51D902E14A
:106CD000000E01D0010E025D0AE00301FF810901EF
:106CE000025103E00301FD8102D00301FD919350A5
:106CF000200B20E0FFC311F0126A136A106A020E23
:106D000037D918E18150200B200A01E0010E3DD94E
:106D1000020E2ED902E1000E01D0010E025D0AE042
:106D20000301FF830901025103E00301FD83120007
:106D30000301FD9312000901416BC6C410F0010E5E
:106D400002D95DE0C4C4A8F12CEC2DF0000957E095
:106D5000010E0901436F446B426B0A0E425D4FE224
:106D600043510301FE15106E090144510301FF1543
:106D7000116E105011103DE043C910F044C911F0DC
:106D8000101E111E1050FE171150FF1709014181EE
:106D90000101780E02D9060E0901425D07E20101E8
:106DA000340EFBD8300E0901422507D00101320E06
:106DB000F4D8300E09014225FA0F0101EED8010185
:106DC0003D0EEBD80301FC5109014315106E030180
:106DD000FD5109014415116E1050111002E1300EE1
:106DE00001D0310E0101D9D801013B0EA96F38EC59
:106DF0002DF00901D89043374437422BAED7090113
:106E000041511200F36AF46A12000901626B81A019
:106E1000628181A2628381A8628581AA62876251B0
:106E2000120002013D51040A31E0070A25E0010A7F
:106E300019E0030A0DE0010A01E012003E5100933F
:106E4000E8B000833E510291E8A028D002811200F0
:106E50003E510097E8B000873E510293E8A01ED053
:106E6000028312003E51009BE8B0008B3E51029518
:106E7000E8A014D0028512003E510095E8B00085CC
:106E80003E510297E8A00AD0028712003E510099B5
:106E9000E8B000893E510299E8B00289120002016F
:106EA0003F51050A42E0010A35E0070A28E0010ADD
:106EB0001BE0030A0EE0010A01E012004051009FAE
:106EC000E8B0008F4051E8B08980E8B037D08990B1
:106ED000120040510193E8B001834051E8B089822B
:106EE000E8B02CD08992120040510197E8B0018798
:106EF0004051E8B08984E8B021D089941200405113
:106F0000009DE8B0008D4051E8B08986E8B016D009
:106F10008996120040510191E8B001814051E8B0DA
:106F2000898AE8B00BD0899A120040510195E8B0E7
:106F300001854051E8B08988E8A0899812001200C4
:106F40000201025112001016116A2AD00901026FC3
:106F5000FCC310F0126A136A12004F51080DF3CFF0
:106F6000E9FFF4CFEAFF120EE926020EEA22120030
:106F7000111616D0FEC310F0126A136A1200E92629
:106F8000000EEA22EE6AED6A12000901026FFDC3EB
:106F900011F0126A136A106A1200A96F38EF2DF00F
:0E6FA000126A136A1050111012101310120012
:026FAE000F0EC4
:106FB000030100170051090804E2410E0025F60FF5
:106FC0001200300E00251200030101390F0B016F72
:106FD000E850090804E2410E0125F60F1200300EB8
:106FE0000125120003C3F3FF02C3F4FF120004C320
:106FF00001F905C302F906C303F907C304F909013E
:10700000010E056F090E066F05C9E9FFEA6E030E52
:10701000B6DAEF50E66E030EACDA00C9EFFF7CDAA9
:10702000020EADDA010E82DAEF50E66E75DA020E6C
:10703000A0DA010E7BDA00C9EFFF01C904F002C932
:1070400005F003C906F004C907F012000901D16B6D
:10705000D26BD36BD46B08C3CFF909C3D0F90AC381
:10706000CDF90BC3CEF9D890CE33CD33CDC910F0C6
:10707000CEC911F0CD07000ECE5B1050111018E0F4
:10708000CFC9E9FFD0C9EAFF020ECF27000ED023F7
:10709000EECF10F0EFCF11F0000110500901D12711
:1070A000000111500901D223000ED323D423DED7CF
:1070B00003010A51010B0EE0CFC9E9FFD0C9EAFF75
:1070C000EFCF10F0000110500901D127000ED2239C
:1070D000D323D4230901D351D41119E0D1C910F01D
:1070E000D2C911F0126A136AD3C914F0D4C915F0C9
:1070F000166A176A10501424D16F11501520D26FE0
:1071000012501620D36F13501720D46FE3D7D1C974
:1071100010F0D2C911F0101E111E10C0F3FF11C0E3
:10712000F4FF12000901010E006F016B026B0301F5
:107130000C510D115AE00CC314F00DC315F0166A72
:10714000176A400E145C000E1558000E1658000EFB
:10715000175804E3400E106E116A04D00CC310F0EF
:107160000DC311F0126A136A10C005F9090110501D
:1071700003017D6F7E6B0301060E7B6F090E7C6F32
:1071800011EC22F009010551106E116A1050030133
:107190000C5F11500D5B0901046B0551045DC7E2E2
:1071A0000451EA6A060FE96E090EEA22EFCF03F9ED
:1071B00000510AE103510125016F0351015D0DE208
:1071C000022B0BE1012B09D003510225026F035161
:1071D000025D03E2012B01E1022B005102E0000EEF
:1071E00001D0010E006F042BD8D70901021D026FD8
:1071F000011DF36E02C9F4FF120003010E5139089C
:1072000005E3300E0E5D02E3300E0FD00E5146083E
:1072100005E3410E0E5D02E3370E07D00E516608FE
:1072200006E3610E0E5D03E3570E0E5D1200FF0CC8
:10723000010E0301EA6A0F25E96E1051EA22EFCF31
:107240000EF3DBDF09018D6F0FC3E9FF10C3EAFF07
:10725000EFCF0EF3D2DF09018E6FFF0E8D5D03E0DD
:10726000FF0E8E5D01E1000C8E39F00B8D1111C304
:10727000E9FF12C3EAFFEF6E010C09018D6BA6A2B4
:1072800003D035EC48F0FBD72F0EA616A6840301D9
:1072900015C3E9FF16C3EAFF152B000E1623EF50A6
:1072A000A86E09018D2B030117510901D8808D5556
:1072B00001E2A86A14C310F0116A1050AA6E03010B
:1072C00013C310F014C311F0132B000E142310502D
:1072D000A96E550EA76EAA0EA76EA6820000A6A2E2
:1072E00003D035EC48F0FBD7A850D1E1A6940901B2
:1072F0008D0500D012000901CD6BA6A203D035EC9C
:1073000048F0FBD73F0EA6160901CD2B03011C51F7
:107310000901D880CD5506E218C3E9FF19C3EAFF79
:10732000EF6A16D01AC3A9FF1BC310F01050AA6E43
:1073300003011A2B000E1B23A680A85018C3E9FFD7
:1073400019C3EAFFEF6E182B000E1923A850DCE1D9
:107350000901CD05120020C310F01050AA6E1FC302
:10736000A9FF3F0EA61603011DC3E9FF1EC3EAFFD6
:107370001D2B000E1E23EFCF4FF9A680A850090148
:107380004F5D01E0010C4F5101E1000CA92AEBE136
:10739000AA2AE9D7030121C3E9FF22C3EAFF212B6F
:1073A000000E2223EFCFCDF9EF5024E0610E09014A
:1073B000CD5D05E3CD517A0802E3200ECD5F0301D8
:1073C00023C3F6FF232B24C3F7FF000E242325C37A
:1073D000F8FF25230800F5500901CD5D01E0000C00
:1073E00023C3F6FF24C3F7FF25C3F8FF0800F550B9
:1073F000D1E1010C000C26C35CF927C35DF909013A
:107400005A6B5B6B0301285109015A5D0301295135
:1074100009015B590BE25CC9E9FF5DC9EAFF5C2B1E
:10742000000E5D23EF6A5A2B5B23ECD7120012008B
:10743000030E0301335D2EE394D861D8010E66D8A4
:10744000EF380F0B166E6DD8EF38F00B300B1610AF
:1074500051D855D8060E176E020E58D8EF5017C0E7
:10746000E7FFE75204E0E8427F0BE706FCE1166E17
:10747000010E030189D816103DD841D8020E46D816
:10748000EF503F0B37D8030E3127000E3223030E87
:10749000335FCED73351000827E263D842D8EF38A4
:1074A000F00B300B0901CD6F03013351010806E2E7
:1074B000010E2CD8EF380F0B0901CD1320D8CDC900
:1074C00013F038D8E66E030147D8020E335D02E2AE
:1074D0003D0E05D014D8010E57D8136E2BD8E66E8A
:1074E0003BD858D83D0EEF6E2FC3E9FF30C3EAFFFB
:1074F000EF6A1200136E1ED8E66EACEF3AF0880EFB
:10750000106EBF0E116E000E126E1200EA6A312567
:10751000E96E3251EA22120005C9E9FF06C9EAFF05
:10752000120031C3E9FF32C3EAFF1200E926000E60
:10753000EA221200146A156A10501324F36E1150D7
:107540001420F46E12501520F86EF4CFF7FFF3CF2D
:10755000F6FF0800F55012001DD8E552E750EF6E17
:107560001200CDDFDEDFEF50E840E8403F0B7AEF5E
:107570003AF0DCDFE552E750EF6E8CEF3AF0D6DF01
:10758000EFCF00F98CEF3AF0C1DFEF50040DF3506C
:107590003C0B12002FC3E9FF30C3EAFF2F2B000E74
:0475A0003023120082
:0C75A4000F01555101E112000401C70E57
:1075B000B36FB70EB46F000EB56F97EC5DF00401BA
:1075C000EA0EB36FB50EB46F000EB56F97EC5DF0B9
:1075D00055CFA9F90901A951000815E2A951070BD6
:1075E00005E104012E0EAF6F49EC5DF002018451FC
:1075F00002E06DD908D00401320ECB6FF2EC5FF0DF
:107600000901A907E7D70401120EB36FB60EB46FD4
:10761000000EB56F97EC5DF00F01B10E566F020EC4
:10762000576F13EF3BF05FDA0DDA010EE926000E1B
:10763000EA2208DA020EE926000EEA2203DA030E35
:10764000E926000EEA2266EF3DF00901016B020116
:1076500084511EE035EC5DF00901006F0D0E005DF8
:107660001AE00A0E005D17E0012B0F0158CFE9FF69
:1076700059CFEAFF582B000E592300C9EFFF58CF0E
:10768000E9FF59CFEAFFEF6A5A515A07000903E0B0
:1076900035EC48F0DCD70901015112005BCF01F94C
:1076A0005CCF02F90901036B5BCFE9FF5CCFEAFF16
:1076B000EFCF00F9EF5021E02E0E0901005D11E13E
:1076C0000F015BCFE9FF5CCFEAFF5B2B000E5C2371
:1076D000EF6AD6D9032BEAD95BCF01F95CCF02F967
:1076E00007D0300E005D03E30051390801E2000CC1
:1076F0000F015B2B000E5C23D7D7C2D9D7D9030E5D
:107700000901035D01E0000C010C0201845103E159
:1077100035EC48F0FAD735EC5DF00901006F310E19
:10772000005D05E3390E005D02E200511200390CE4
:1077300004010D0ED5D904010A0ED2D9300E0F0165
:107740005F5DFF0F030DF3CFE9FFF4CFEAFFE80E13
:10775000E926020EEA22EECFB3F4EECFB4F4EFCF77
:10776000B5F497EC5DF00F015F51380A01E1AED03E
:107770000F0A01E1A9D0010A01E19FD0030A01E14A
:1077800098D0010A50E0070A47E0010A3EE0030AE8
:1077900001E01200330E85D90901A16F340E81D9A1
:1077A0000901A26F870EE66E090EE66EA1C9E6FF1B
:1077B000A2C9E6FFA6D9870EB16F090EB26F84EC9D
:1077C0005DF046D9000949E0870EE66E090EE66EC7
:1077D000F4EC56F0E552E552F3CFA1F9F4CFA2F95B
:1077E000F3CFA8FF330E47D9A2C9A8FF340E43D95F
:1077F000A2C9A8FF080E3FD9A1C9A8FF090E3BD90D
:10780000A2C9B9F2A1C9BAF212000901B10E9F6F63
:10781000020EA06FA36B0ED00901BF0E9F6F020E68
:10782000A06F0E0E06D00901BB0E9F6F020EA06F57
:107830000A0EA36F9FC956FFA0C957FFF4DE08D9EF
:107840000F019B0E5D6F090E5E6F0F01870E5B6F60
:10785000090E5C6F23DF000911E104017D0EB36F97
:10786000B70EB46F000EB56F97EC5DF00201845156
:1078700003E135EC48F0FAD735EF5DF09FC9E9FF39
:10788000A0C9EAFF9BC9EEFF9CC9EEFF9DC9EEFFB0
:107890009EC9EEFF9BC9A8FF2FD99CC9A8FF2CD970
:1078A0009DC9A8FF29D99EC9A8FF0901A351A32BEF
:1078B00009D0160EF6D8010903D0160EF2D8FE0B29
:1078C000A86E160E3BEF3DF080EF3CF01200040175
:1078D000470EB36FB60EB46F000EB56F97EC5DF048
:1078E00014DF0901AA6F390EAA5D03E0AAC95FFF80
:1078F0001FDF35EC48F0380E0901AA5DE8E11200FF
:107900000901006B026BCAEC46F0A1C485F9A2C460
:1079100086F9090185510401A15D106EA25109018A
:107920008655116E320E105C000E115809E3A1C489
:1079300085F9A2C486F90401150EAF6F49EC5DF01C
:1079400035EC48F002018451E4E00901025101E004
:1079500078D035EC48F002018451F7E035EC5DF069
:107960000901016F0051030A2FE0010A2AE0030A0E
:1079700023E0A6D8010E101808E1115006E11250BC
:1079800004E1135002E1010E1DD09AD8040E101824
:107990000FE111500DE112500BE1135009E112EC0F
:1079A00047F00401060E9CD80901010E026FCDD7E5
:1079B0000401150E95D8C9D7060E046F036B020E8D
:1079C00001D0030E006FC1D70351032BEA6A050FE4
:1079D000E96E090EEA2201C9EFFF03C910F0116A2E
:1079E000126A136AD880800E1054000E1154000ED3
:1079F0001254000E1354A9E2060E046F016B60D8F6
:107A0000800E105C000E1158000E1258000E135814
:107A10000DE20151EA6A050FE96E090EEA22EFCF85
:107A2000FEFDE5EC46F00901012BE9D70D01F06BF5
:107A300016EC46F004C9AFF449EC5DF00901006BA7
:107A400084D7010C43D804012E0E4AD873EF3DF0C1
:107A50000401290E45D804013A0E42D80401200E33
:107A60003FD80F01140E5A6F0F01870E586F090E81
:107A7000596F25EF3BF00201DD6FDE6BB8EF3DF093
:107A800001C9E6FF02C9E6FFF4EC56F0E552E55203
:107A9000F350E66E5DCF10F05ECF11F00901035197
:107AA00012000201DB6FDC6BA7EF3DF00F01102429
:107AB000E96E000E1120EA6EE552E750EF6E1200FB
:107AC00001C910F0116A126A136A1200EF50E66ED3
:107AD000E66A17D8000EB16F090EB26F84EF5DF041
:107AE000AF6F49EF5DF0000EE66E090EE66E56CF01
:107AF000E9FF57CFEAFF12000901A351A32B3BEF87
:107B00003DF069EC57F0E552E552E552E5520401CB
:027B1000120061
:0E7B1200AA6AA96A3F0EA6160901B10E006FFD
:107B2000020E016FA950106E116A120E105C000E49
:107B300011580CE2A68000C9E9FF01C9EAFF002B39
:107B4000000E0123A8CFEFFFA92AECD71200DBC259
:107B5000A9FFDCC210F0116A1050AA6EA6A203D0D1
:107B600035EC48F0FBD73F0EA616A680A8501200B1
:107B7000A8CFA4F9DDC2A9FFDEC210F0116A10502F
:107B8000AA6EA6A203D035EC48F0FBD73F0EA6168E
:107B9000A6800901A451A85C01E112D0A4C9A8FFE4
:107BA0002F0EA616A684550EA76EAA0EA76EA68245
:107BB0000000A6A203D035EC48F0FBD7A69400D075
:107BC00012001200200E26DA0901516F51A14CD08B
:107BD000AC84080E7E6E1F0E1DDA080A36E00F0A0E
:107BE00032E0010A2AE0030A23E0010A1CE0070A46
:107BF00015E0010A0EE0030A07E0010A28E1090185
:107C0000340E4F6F820E1DD009018C0E4F6F200E67
:107C100018D00901450E4F6F100E13D00901220E26
:107C20004F6F080E0ED00901100E4F6F040E09D0D1
:107C30000901080E4F6F020E04D00901030E4F6FA9
:107C4000010E506F08D0AC0E03D0560E01D0AC0E12
:107C500009014F6F506B4FC9AFFF50C910F0116A47
:107C600010507F6ED4EF5CF0DBEF5CF0220ED2D9C7
:107C70000901516F51A14CD06C84080E7C6E210E0D
:107C8000C9D9080A36E00F0A32E0010A2AE0030ADD
:107C900023E0010A1CE0070A15E0010A0EE0030ACE
:107CA00007E0010A28E10901340E4F6F820E1DD052
:107CB00009018C0E4F6F200E18D00901450E4F6F31
:107CC000100E13D00901220E4F6F080E0ED00901BD
:107CD000100E4F6F040E09D00901080E4F6F020EEF
:107CE00004D00901030E4F6F010E506F08D0AC0E87
:107CF00003D0560E01D0AC0E09014F6F506B4FC927
:107D00006FFF50C910F0116A10507D6EEDEF5BF0FF
:107D1000F4EF5BF0230E7ED9926E240E7BD909011D
:107D20004F6F96D904E1330E09014F1305D09BD94B
:107D300003E1CF0E09014F174FC993FF250E6AD9F2
:107D4000D80909014F6F84D902E1D80E03D08BD92D
:107D500003E1F80E09014F174FC994FF280E5AD9B5
:107D6000976E290E57D91009986E12002A0E52D913
:107D7000896E2B0E4FD98A6E2C0E4CD90901006FDB
:107D800067D902E10901008B00C98BFF2F0E42D990
:107D90008E6E300E3FD98F6E1200310E3BD9C16E00
:107DA000320E38D98009C06E1200010E0201DF5D6B
:107DB00046E3DF51050801E21200E2510DE0E0C2A6
:107DC000A8FFDF05E824660F34D9E1C2A8FF02014D
:107DD000DF05E824670F2DD90201DF052FD9EECF8B
:107DE0008DF9EDCF8EF98DC98FF98EC990F9090102
:107DF000010E8F5F000E905B060E0201D890E037F7
:107E0000E137E806FBE10201E051E840E8403F0BC2
:107E1000300B106E8FC9E9FF90C9EAFFEF50CF0B0E
:107E200010100901916F8DC9E9FF8EC9EAFFE1C207
:107E3000EFFF8FC9E9FF90C9EAFF91C9EFFF120078
:107E40000901666B676B010E0201E35D03E3E35119
:107E5000050803E2F36AF46A1200E305EFD8EECFF7
:107E600062F9EDCF63F962C964F963C965F9090183
:107E7000010E645F000E655B62C9E9FF63C9EAFF3A
:107E8000EF50666F676BD89066376737D890663764
:107E9000673764C9E9FF65C9EAFFEF50300BE8387E
:107EA0000F0B661366C9F3FF67C9F4FF1200E4C243
:107EB0008DF90201E55104E08DC9A8FF640EB9D81F
:107EC000CB50106E116AFF0E101801E1115002E044
:107ED000000E01D0010E010808E1030E09018D5DBD
:107EE00002E18D6B0BD0020E06D009018D5102E12B
:107EF000020E03D0030ED8808D558D6F030E8D17A3
:107F0000FC0ECA168D51CA121200030ECA140901C2
:107F1000626F030E625D01E16207CB50106E116A61
:107F2000FF0E101804E1115002E1020E01D0030E01
:107F3000D880625512000201E75104E0E6C2A8FFB2
:107F4000630E77D80201E6A103D00C0EBD1202D059
:107F5000F00EBD16E6A303D00C0EBA1202D0F00E3E
:107F6000BA16E6A504D00C0EB7123C0E01D0F00EE6
:107F7000B716E6A704D00C0E73123C0E01D0F00E1B
:107F80007316E65102E0CA841200CA941200630E0E
:107F900041D8000901E11200B70EB116650E3AD8BA
:107FA000010B02E0CB6802D03F0ECB6E0201E56B05
:107FB000640E30D80201E46F7ADF660E4DD8670E8A
:107FC0004FD8010EDF6FF1DE680E46D8690E48D833
:107FD000020EDF6FEADE6A0E3FD86B0E41D8030E49
:107FE000DF6FE3DE6C0E38D86D0E3AD8040EDF6F0B
:107FF000DCDE0201E76B630E0DD80201E66F9BEF3A
:108000003FF031D802E11AEF53F022D802E165ECDB
:1080100034F012000201DB6FDC6BA7EF3DF00901C9
:10802000506F0201E26B4FC9E0F2E8CFE1F20201CA
:1080300012000201DD6FDE6BB8EF3DF0030DF3CFF0
:10804000E9FFF4CFEAFF6B0EE926040EEA221200E4
:10805000870EE0DF02081200DDDF09014F6F12001A
:0E806000D9DF0FEF40F0870ED5DF01081200C8
:02806E00150EED
:108070000001626F636B4BEC12F00001AF6FB36BEA
:10808000E16BAE6B140EB16FB26B1200AFC068F053
:1080900015EC13F0000908E10001E16B080EB56F63
:1080A000B36BAE6BB46B010CAFC081F0EAEC15F0B2
:1080B000000940E05EDA0001700E7F6F090E806FEC
:1080C000AFC07EF0ABEC15F000091AE00001E15101
:1080D000E12BEA6AC00FE96E000EEA2270C9EFFFD9
:1080E000E1C010F0116A126A136A1F0E1018E3E162
:1080F0001150E1E11250DFE11350DDE1E16BDBD71C
:10810000AFC073F0CFEC14F00A0E0901705D27E1E7
:108110000001E151EA6AC00FE96E000EEA22EF6A3F
:10812000E16BC3D9E2C0F4F0E3C0F5F08CD90001F3
:10813000B56F15D00001B35112E0F1510401A15DFA
:10814000106EA2510001F255116E500E105C460ED9
:10815000115805E30EDA020EB56F010EB36F000180
:10816000B351010A3DE0050A04E0040A57E1B66B89
:1081700000DAAFC06BF0B7EC13F0000901E1010CBD
:10818000B6C0E9FFEA6AE9BEEA68DDD9560EE9261B
:10819000020EEA22EECF71F9EECF72F9EFCF73F94A
:1081A000090171C9F6FF712B72C9F7FF000E722326
:1081B00073C9F8FF73230800F5CF70F9F55007E095
:1081C00070C96DF0AFC06CF0E2EC13F0E9D7AFC04E
:1081D0006AF061EC13F000010C0EB66F010EB36F84
:1081E000080EB55D1BE0B5C0F3F019D800090FE02B
:1081F0000C0E0001B65D03E0040EB36F04D0020E56
:10820000B55D01E1B36B080EB56FB46B010C0C0EDC
:108210000001B65D03E0040EB36FABD7010C0001A3
:10822000F351060A54E0030A50E0060A4CE0070A3C
:1082300034E0060A30E0030A18E0010A59E1AE8191
:10824000AE93010EB66F090EE66EE66AE4C0E6FF75
:10825000E5C0E6FFB70EE66E000EE66EC4EC58F021
:10826000106E060EE15E1050010CAEA112D0E4C0FB
:1082700086F4E5C087F40401B70E846F000E856FA5
:1082800085EC49F0000904E00001AE83020E31D014
:108290000001060E2ED07BEF41F0ECC0E6FFEDC0F2
:1082A000E6FFF4EC56F0E552E552F3CFB2F0EEC043
:1082B000E6FFEFC0E6FFF4EC56F0E552E552F3CFEF
:1082C000B1F0000102D0AEEF41F00B0E12D00B0E58
:1082D000B66FB0C010F041D905E1115003E1125062
:1082E00001E1135007E0B0C069F01EEC13F0010C7F
:1082F000050EB66F010C0001B451030A1EE0020A1C
:1083000015E0010A2AE1020EB45D02E112EC47F029
:10831000B0C010F022D905E1115003E1125001E183
:10832000135006E030D90001010E05D01CD915E12B
:108330000001030EB66FB46F000CAFC06BF0B7EC6A
:1083400013F000090AE0AFC068F015EC13F0000963
:1083500004E0AFC069F01EEC13F0000C0001B45152
:10836000020A45E0030A2CE0010A6CE1AEB302D038
:10837000060E66D0070EB66FB1C066F0B2C067F0E9
:10838000AF51240DF3CFE9FFF4CFEAFF000EE92649
:108390000C0EEA22EE52E9CF64F0EACF65F099ECD8
:1083A00012F00001B06F106ED8D805E1115003E152
:1083B000125001E1135002E0010E17D00A0E40D016
:1083C000D2D840E0EACD10F0116A126A136A010EA9
:1083D0001016116A126A136A10501110121013103D
:1083E00031E0CAEC46F00001020EB46F000CB0C0E0
:1083F00081F0EAEC15F000091CE0BBD80001740E16
:108400007F6F090E806FB0C07EF0ABEC15F00009F5
:1084100007E074C9FEFDE5EC46F035EC48F0EED718
:108420000D01F06B16EC46F0B0C073F0CFEC14F019
:10843000000C99D807E1A7D80001FE0EB06F090E15
:10844000B66F010C000C0901006B070EE76E0019F6
:10845000E8AE02D0E73402D0E750005D25E2040E1A
:10846000E66EE66A00C9E9FFEA6AE9BEEA686BD827
:10847000410EE926020EEA22EECFE6FFEECFE6FF3E
:10848000EFCFE6FFF4C0E6FFF5C0E6FF03EC58F0DF
:10849000106E070EE15E1050000903E10901005162
:1084A00012000901002BD1D7070C0901036BC00E84
:1084B000006F000E016F62D8EF50200804E1002B1E
:1084C000000E0123F8D700C9E2F001C9E3F0000172
:1084D000010EF06F53D8EFCF02F9EF5033E00901EE
:1084E0000351010A16E0010A29E1200E025D03E0B2
:1084F0002C0E025D05E142D8EF6A010E036F1ED01B
:108500000D0E025D03E00A0E025D18E137D8EF6A36
:1085100015D0200E025D12E00001F051F02BE96E43
:10852000EA6AD890E936EA36E20EE926000EEA2237
:1085300000C9EEFF01C9EDFF0901036B002B000E1E
:108540000123C8D71200030EEA02F3CFEAFFE902C3
:10855000F3CFE9FFF450EA261200116A126A136A97
:10856000FE0E10181200B0C068F015EC13F00009F0
:108570001200A1C4F1F0A2C4F2F0120000C9E9FF98
:1085800001C9EAFF120012EC47F0B0C069F01EEF1B
:0285900013F0E6
:0E859200360ED7D906D8CDEC5CF0E6EC5BF0E7
:1085A00051EF5EF00901506B516B300ECBD90901D0
:1085B0004F6B040E4F5D1BE2D3D9A7EC3DF0E66E86
:1085C000090120DAE552E750EF6E1CDAE6D9C8D986
:1085D000DB27000EDC23A7EC3DF0E66E090117DA7D
:1085E000E552E750EF6E13DAD8D94F2BE2D750C9D6
:1085F00010F051C911F0126A136AD880000E10549D
:10860000020E1154000E1254000E13541EE2020109
:10861000640E7F6F856F8B6F916F976B9D6BA36BF4
:10862000A96B09014F6B040E4F5D0FE2EBD97ED9A8
:10863000B8EC3DF00901EBD979D9DD27000EDE2336
:10864000B8EC3DF009014F2BEED70201000E7A6F16
:108650000A0E7B6F7F517A25806F000E7B21816F20
:1086600085518025866F000E8121876F8B5186256D
:108670008C6F000E87218D6F91518C25926F000EAB
:108680008D21936F97519225986F000E9321996FCA
:108690009D5198259E6F000E99219F6FA3519E2595
:1086A000A46F000E9F21A56FA951A425AA6F000EEB
:1086B000A521AB6F12000A0E0301286F296B03017D
:1086C000500E266F090E276FFBEC39F00201120ED7
:1086D00003D909014F6F4FA11AD0AFD926E111502C
:1086E00024E1125022E1135020E144D9110EF4D8B4
:1086F0005CD9100EF1D80DD90401D46F106EF1D8E9
:1087000014E1115012E1125010E113500ED095D91E
:1087100005E1115003E1125001E1135006E0D4C409
:10872000A7F119EC2DF00401D4690201150ED4D87B
:1087300009014F6F4FA11AD084D917E1115015E1EB
:10874000125013E1135020E115D9140EC5D82DD9BC
:10875000130EC2D8DED80401D56F106EC2D805E161
:10876000115003E1125001E1135012006AD905E1E2
:10877000115003E1125001E1135006E0D5C4A7F1F6
:1087800019EC2DF00401D56912000201160E4FD923
:1087900038E30251010835E350D905E1115003E1F6
:1087A000125001E113502DE0D4C4AEF147EC2EF08D
:1087B000000916E09CD8800B11E0E6D80BE01DD92B
:1087C00004E1CAD835EC48F0FAD708D901E124D938
:1087D00026D9F3D78CD8020B01E1BED8B4EC2EF029
:1087E0003BD90FE0D4C4A8F12CEC2DF0000909E02E
:1087F00033D905E0E2D801E117D932D9F9D7DEEC57
:108800002DF00201170E13D938E30251010835E3A8
:1088100018D905E1115003E1125001E113502DE088
:10882000D5C4AEF147EC2EF0000916E060D8800BFD
:1088300011E0AAD80BE0E1D804E18ED835EC48F07D
:10884000FAD7CCD801E1E8D8EAD8F3D750D8020B50
:1088500001E182D8B4EC2EF0FFD80FE0D5C4A8F126
:108860002CEC2DF0000909E0F7D805E0A6D801E1CD
:10887000DBD8F6D8F9D7DEEC2DF00901026B040E37
:10888000025D04E269D80901022BF9D71200020146
:10889000B051030A10E0010A0BE0030A06E0010AE6
:1088A00001E00BD01FEC5DF008D038EC5CF005D097
:1088B00054EC5EF002D0000000D012000C0DF3CF9B
:1088C000E9FFF4CFEAFF7A0EE926020EEA2212004F
:1088D000E926000EEA221200DB6F010EDC6FA7EF23
:1088E0003DF0116A126A136AE86810181200090153
:1088F0000251EA6AAC0FE96E020EEA22EF50120052
:108900001050EE24E76E1150EE20EA6EE7CFE9FF3B
:108910001200E552E7CF11F0E552E7CF10F0010168
:108920001010A16F11C0A2F1CCEF2CF0EF50A86E87
:108930004F51E8240201DD6FDE6B000EDD27010ED2
:10894000DE2312000301286F296B03017A0E266FC4
:10895000020E276FFBEF39F002C9B0F247EF44F087
:108960004F51E8240201DB6FDC6B000EDB27010EA8
:10897000DC2312000101A56BA66B0101500EA36F51
:10898000090EA46F020112000101000EB06F090E62
:10899000B16F66EC2EF000091200EF50106E116AF4
:1089A000E8505027115051231200106E116E106ABA
:1089B00010C0E6FFE66E0201120058D8EF50106EAC
:1089C000116A43D8060E84DF9BDFEFCF00F94ED843
:1089D000EF2AEFCF10F039D80B0E3AD04BD8EF502A
:1089E000106E116A32D88CDF00C9EFFF43D8EF2A2E
:1089F00045D02BD80A0E68EF44F0090126D8040EA2
:108A000067DF3CD04F515ADF050E68EF44F04F51FD
:108A100055DF0B0E68EF44F02DD8EF6A120015D821
:108A2000040E56DFEF2A120021D8EF6A120054DF3D
:108A30000901026F000E025D1200D4C410F071EF44
:108A400044F0D5C410F071EF44F002515EEF44F0F1
:108A50003FDFEF50105C12000901CBDFEF50120036
:108A6000C8DFEF0600C9A9F138EF2DF0EEDF090EDF
:108A700068EF44F0EADF020E68EF44F0EFCF10F049
:068A8000E4DF050EE5D75E
:0A8A86000D01E96B010EEA6F040117
:108A9000180E5C6F07EC59F00901006B00C910F06B
:108AA00036DA060ED3D905E20051D8D9EF6A002B89
:108AB000F5D7010C0901FE0E026FEACD10F034DA91
:108AC00001E1FE0C016BF4D9060EC0D908E2015198
:108AD00039DA03E101C902F902D0012BF4D702C946
:108AE00010F015DAFE0E101807E1115005E11250D2
:108AF00003E1135001E1FE0C450E036F046B056B9F
:108B0000ECCDE9FFEDCDEAFFEF5001E1FF0CECCD3C
:108B1000E6FFEDCDE6FFF2EC58F0E552E552F3CF7B
:108B2000ECFDF4CFEDFD03C961F404C962F4D1D9C1
:108B300004E00901FE0E026F6CD091EC59F00901BE
:108B4000006F106EE4D9800E71D902E0026961D025
:108B5000016BAED90C0E7AD922E291EC59F00901E1
:108B6000006F01510D01EA6AEC25E96EED51EA2230
:108B7000EF500901005D06E0120E0327000E0423EA
:108B800005230DD0005109E10901012B91D90C0EEB
:108B90005DD905E291EC59F0F7D7012BDAD788D9E6
:108BA0000C0E101831E111502FE112502DE113502D
:108BB0002BE10251080DF3CF06F9F4CF07F9B90EF6
:108BC00006270D0E0723A7D9010EEF6EA4D9EB6A75
:108BD000020EEB6A91EC59F0E66E9DD9030E2DD989
:108BE000030E9ED9010E29D9030E9AD9020E25D95A
:108BF000060E23D9060E94D9010E92D9E552E750FC
:108C0000EF6E0D01E92B05D098EC59F035EC48F0EA
:108C10008AD798EC59F0090102511200EFCDF0FD0E
:108C200005D80D01EF511AD9EF6A12000D01F0516C
:108C3000080DF3CFA4F9F4CFA5F9B90E0901A427C3
:108C40000D0EA5235BD9EF50106E126A136A6FD90F
:108C500003E098EC59F010D051D92ED96BD90CE023
:108C600087EC59F00401A00E6A6FD1EC59F00009AD
:108C700003E035EC48F0F6D7F90E106E3FD9E85016
:108C8000EF160D01EA9312000D01F151080DF3CF1B
:108C900001F9F4CF02F9B90E090101270D0E0223E3
:108CA0009F0EE6D8E850EF16E3D806D93DD915E077
:108CB000DFD802D93CD914E140D90FE1D9D810D975
:108CC000D7D8E0D810C061F411C062F402D905E130
:108CD000CFD8EF820D01EA8303D0CAD8EF8A000C07
:108CE00091EC59F00901006FC3D8EAD8C1D8D6D8A1
:108CF00005E11350111802E1BBD8EF8C09010051B6
:108D00001200010C0D01F251080DF3CF00F9F4CF60
:108D100001F9B90E090100270D0E0123AED8EF505D
:108D2000106E126A136A06D903E012D901E3EBD878
:108D3000A4D8C2D8FFD815E100D903E09ED8EF8AA5
:108D4000000C9BD8CDD899D89DD810C05EF411C026
:108D50005FF4CDD805E191D8EF840D01EA8301D00D
:108D6000000CF3CD63F473EC59F087D8A9D885D8FB
:108D700095D805E11350111802E17FD8EF8C010C52
:108D800012001200F36AF46A1200056A066A076AA2
:108D90001200000CEACD10F0C7D801E1000C090167
:108DA000A46BA4C910F0B3D8060E50D806E2A451A3
:108DB000C9D801E0000CA42BF4D70D01010EB96F46
:108DC000400EBC6FBD6BBE6B010C0901B90EA66FE6
:108DD0000D0EA76FB9CD10F0ADD803E0B9D801E3FF
:108DE00092D8B9CD10F093D8A5D811E1A6D803E058
:108DF0000D01B98B000CBCCD5EF4BDCD5FF477D80E
:108E000005E10D01B985EA83EB6B01D0000CFECDC5
:108E100063F473EC59F00D01EB2BBC2B000EBD235A
:108E2000BE23010C70D80D01B96B010C10166FD860
:108E30001050111012101310120072D8E552E750A2
:108E4000EF6E91EC59F0E66E8BEF47F0105C000E80
:108E50001158000E1258000E13581200080DF3CFCF
:108E6000E9FFF4CFEAFFB90EE9260D0EEA2212005F
:108E700001C9E9FF02C9EAFF120000C9E9FF01C9FF
:108E8000EAFF1200030E4CD8EE501324106EEE5081
:108E90001420116EEE501520126E1200060E40D8EE
:108EA000EECF12F0EFCF13F00001125010181200A5
:108EB00001C910F087EF47F0EF50106E87EF47F0D1
:108EC000EE52EE2A000EED22EECF10F0EDCF11F0B3
:108ED00012000401A00E606F46EC59F00009120068
:108EE000EE52EECF13F0EFCF14F0156A120004012A
:108EF000A00E5D6F10EC59F000091200A4C9E9FF43
:108F0000A5C9EAFF12000D01F06B16EF46F0116AD9
:108F1000126A136A120006C9E9FF07C9EAFF1200C4
:108F2000E926000EEA221200010E16EF47F0020EAB
:108F300016EF47F0040E16EF47F0EACD10F0E7DF2A
:108F400097EF47F08BDFEFCF10F0E1DF94EF47F0C2
:0C8F5000EBCD10F0DCDF400E26EF47F008
:048F5C00DACFE4FF85
:108F6000E2CFDAFFE9CFE4FFEACFE4FFF6CFE4FF98
:108F7000F7CFE4FFF8CFE4FFF5CFE4FFF3CFE4FF52
:108F8000F4CFE4FFFACFE4FFFBCFE4FF00EE00F004
:108F9000100EE80403E3EECFE4FFFBD700EE10F081
:108FA000100EE80403E3EECFE4FFFBD7E652F2A491
:108FB00014D09E0ED76E580ED66E0401A12B000E53
:108FC000A223A323A4230401A70706E1640EA76F2D
:108FD0000401A52B000EA623F2949E50200B05E061
:108FE0009D50200B02E0EFEC5CF09E50100B05E072
:108FF0009D50100B02E00EEC5DF0A450200B05E03C
:10900000A350200B02E008EC5CF0A450100B05E02C
:10901000A350100B02E027EC5CF0E55200EE1FF0CD
:10902000100EE80403E3E5CFEDFFFBD700EE0FF0F1
:10903000100EE80403E3E5CFEDFFFBD7E5CFFBFF20
:10904000E5CFFAFFE5CFF4FFE5CFF3FFE5CFF5FF7E
:10905000E5CFF8FFE5CFF7FFE5CFF6FFE5CFEAFF75
:10906000E5CFE9FFE5CFDAFF1100CD9ECFAE0FD0FF
:1090700004017B510BE004017B6BFF0E04017A5D60
:1090800005E004017A5102E004017A0703D00401EB
:10909000010E7B6F04017A5101E00400120004010B
:1090A000010E7C6FD1807A694AD92FEC60F0C9EC4F
:1090B00042F05BD902E0E2EC3DF057D902E036EC39
:1090C0003EF0F28EF28C43EC45F002EC5AF089EC63
:1090D0003DF0B6EC3EF08AEC3EF0CDEC3EF0C7EC55
:1090E0003FF0140E32D90F01556FD2EC3AF07BEC01
:1090F0004BF001EC40F0AEEC51F037EC26F037ECE1
:1091000040F05BEC43F07AEC54F06AEC04F06AEC6B
:1091100060F00401260E7A6F150E17D9020B20E0BD
:109120000401BD510401A15D106E320E105C18E304
:10913000A1C4BDF4240E09D9400B0AE0240E05D9C0
:10914000BF0BA86E240E0201DD6FDE6BB8EC3DF0A4
:10915000939C8A7C870EF9D8020802E10201007113
:10916000C1EC51F0BDEC4BF0A6EC04F0B7EC54F0C0
:10917000C5EC43F084EC5FF06EEC26F046EC40F07A
:109180002FEC50F008D80401BC510401C35DC1E0CC
:10919000C3C4BCF4BED70401BE510401A15D106E6E
:1091A000010E105C0DE3A1C4BEF4870ECED8020AF6
:1091B00005E0030A05E138EC53F002D092EC34F0FC
:1091C0000401BF5119E104017D2B0C0E7D5D01E30B
:1091D0007D6BC11C0F0B7D5D0CE2C30EC2167D5171
:1091E000040DF350C212C280C2820401010EBF6F8F
:1091F00003D0B0D8EE6AED6A0401BF5114E0C2504A
:10920000020B11E1C450136E126AC3500001121018
:10921000106E13C011F004019DD810C0EEFF11C0F4
:10922000EDFF0401BF6B12000301A60E236FC00EF9
:10923000246F000E256F80C421F381C422F3CAEC91
:1092400039F0000961E00301080E1C6F350E0301BF
:109250001A6F1B6B0301880E186F090E196F7BECD8
:1092600039F00901876FE850872BEA6A880FE96EA9
:10927000090EEA223A0EEF6E0301080E1C6F3E0E35
:1092800003011A6F1B6B090187510301186F196BDA
:10929000880E1827090E19237BEC39F0880EE66E2C
:1092A000090EE66EB6EC58F0E552E552F3CF33F313
:1092B0000301880E316F090E326F03019C0E2F6F70
:1092C000090E306F18EC3AF09C0EE66E090EE66E51
:1092D000150E0401116A8025106E8151112210C0F3
:1092E000E6FF11C0E6FF67EC58F0E552E552E552A3
:1092F000E552000909E17EC4E9FF7FC4EAFF090ED7
:10930000E926000EEA22EF841200350E03011F6FDA
:10931000206B84C41DF385C41EF3ABEC39F0000947
:109320000DE13E0E03011F6F206B86C41DF387C441
:109330001EF3ABEC39F0000901E1010C000CB10E99
:10934000CD6ECD9EF18ED56A12000201DB6FDC6B13
:10935000A7EF3DF07D51E96EEA6AD890E936EA362A
:10936000C30EE926020EEA2212000201DB6BDC6B5F
:08937000A7EC3DF0000912001A
:0893780043616368652D436F3A
:109380006E74726F6C3A206D61782D6167653D3641
:1093900030302C206D7573742D726576616C696444
:1093A0006174650D0A00485454502F312E3020341A
:1093B000303120556E617574686F72697A65640D1D
:1093C0000A5757572D41757468656E7469636174E7
:1093D000653A204261736963207265616C6D3D225C
:1093E00064656661756C74220D0A0D0A41757468B6
:1093F000656E7469636174696F6E20526571756919
:10940000726564210D0A00485454502F312E3020CB
:10941000353033200D0A0D0A536572766963652075
:10942000556E617661696C61626C650D0A00485425
:1094300054502F312E3020343034204E6F7420663B
:109440006F756E640D0A0D0A4E6F7420666F756E2F
:10945000642E0D0A00617564696F2F782D7761762F
:1094600065006170706C69636174696F6E2F6A6109
:1094700076612D6172636869766500696D61676503
:109480002F6A70656700696D6167652F676966009F
:10949000746578742F6A61766173637269707400A1
:1094A000746578742F637373006170706C696361A5
:1094B00074696F6E2F6A6176612D766D00746578C0
:1094C000742F68746D6C00746578742F706C6169AA
:1094D0006E000D0A4E6F772072756E6E696E672092
:1094E0006170706C69636174696F6E2E2E2E000D51
:1094F0000A526561647920746F20646F776E6C6FB7
:1095000061642046696C652053797374656D2049E8
:109510006D616765202D2055736520586D6F6465FA
:109520006D2070726F746F636F6C2E0D0A000D0AE0
:1095300044484350202620495020476C65616E699D
:109540006E672064697361626C65642E0D0A000D9C
:109550000A44484350202620495020476C65616EDC
:10956000696E6720656E61626C65642E0D0A000D80
:109570000A44656661756C74205375626E6574206B
:109580004D61736B2028000D0A44656661756C742B
:1095900020476174657761792041646472657373F3
:1095A0002028000D0A44656661756C7420495020BE
:1095B000416464726573732028000D0A53657269F3
:1095C000616C204E756D626572202800323030204B
:1095D0004F6B0D0A003432352043616E27742063CF
:1095E0007265617465206461746120736F636B657B
:1095F000742E2020496E637265617365204D415859
:109600005F534F434B4554532E0D0A0032323620E0
:109610005472616E7366657220436F6D706C657411
:10962000650D0A0031323520446F6E650D0A003138
:109630003530205472616E7366657272696E672090
:10964000646174612E2E2E0D0A00353330204C6F6C
:1096500067696E2072657175697265640D0A0035FF
:109660003032204E6F7420696D706C656D656E745C
:1096700065640D0A00353030200D0A003232312089
:109680004279650D0A00323330204C6F676765649C
:1096900020696E0D0A003333312050617373776F88
:1096A00072642072657175697265640D0A003232E8
:1096B000302052656164790D0A0041424F520054D6
:1096C00059504500504F52540053544F5200515579
:1096D0004954005041535300555345520047756556
:1096E000737400596573006C34303D323B006C3448
:0596F000303D313B009C
:0A96F6000901006B00C910F05FD9F4
:1097000008E2005168D9EF6A00516BD9EF6A002B6B
:10971000F4D71200C750040B01E0010E72D9FAE130
:10972000C580C5B0FED704010A5143D9C5BC21D0BC
:109730000BC4BBF4B4EC5FF0C5BC1BD0C582C5B292
:10974000FED704010A516FD9010F10240401BB6F29
:10975000B4EC5FF0C5BC0DD00401B96B96EC5FF0C2
:109760000CC4E9FF0DC4EAFFEF6EC584C5B4FED793
:10977000000CC584C5B4FED7010C0401CE51040110
:10978000A15D106E040E105C4DE3A1C4CEF43ED971
:10979000D00E0B6FCFC40AF4BDDF00093CE1090114
:1097A00000AF39D00401CF511CD9EF28106E070E3D
:1097B0001016116A126A136ACF510DD9EFCF14F047
:1097C000156A166A176A1050141808E11150151816
:1097D00005E11250161802E1135017181CE016D9B3
:1097E000D10E0B6FCFC40AF495DF0401CF51FFD81F
:1097F000CF51F7D8EF50EF2A0F011024E96E000E79
:109800001120EA6E00C9EFFF070E106E0401CF5160
:10981000E8D81050EF160401CF2BCFC410F0CFD8EA
:1098200001E3CF6B12000EC410F0C9D801E3000CA5
:1098300004010E51DCD80E51CED8EF50EF2A10247F
:10984000E96E000E1120EA6EEFCF44F9070E106E9C
:109850000E51C1D81050EF160901445112001200E8
:10986000040112519F0805E212390F0B0F0B570F1D
:1098700004D012390F0B0F0B300FCFD80F0E04018D
:109880001215090804E20F0E1215570F03D00F0E20
:109890001215300F0DEF4DF009018E6B04011651BA
:1098A00001E1000CC750040B01E0010EAAD8FAE157
:1098B000C580C5B0FED7040113517BD8C5BC18D0F4
:1098C00009018D6B0401165109018D5D14E204013B
:1098D00014C4E9FF15C4EAFF142B000E1523EFCFC3
:1098E000BBF4B4EC5FF0C5BC03D009018D2BEAD703
:1098F0000901010E8E6FC584C5B4FED709018E51D2
:109900001200C750040B01E0010E7BD8FAE1C580BC
:10991000C5B0FED7040117514CD8C5AC04D0C584DE
:10992000C5B4FED7010C0401800EBB6FB4EC5FF030
:10993000040118C4E9FF19C4EAFF182B000E19230B
:10994000EFCF8DF9EF5003E08DC9BBF4EFD7C5849D
:10995000C5B4FED7000CC750040B01E0010E51D86E
:10996000FAE1C580C5B0FED704011A5122D8C5ACB2
:1099700004D0C584C5B4FED7010C0401800EBB6FB2
:10998000B4EC5FF004011BC4F6FF1B2B1CC4F7FFF3
:10999000000E1C231DC4F8FF1D230800F5CF00F99D
:1099A000F55003E000C9BBF4EBD7C584C5B4FED7BE
:1099B000000C39D810240401BB6FB4EF5FF0116ABA
:1099C000126A136A010E105C000E1158000E125834
:1099D000000E13581200EA6A080FE96E040EEA221C
:1099E0001200EA6A090FE96E040EEA221200080D5D
:1099F000F3CF10F0F4CF11F0000E1026040E112258
:109A00001200106E1F0EC514101012000401000E7B
:109A10000C6F090E0D6F040112000401106F11C4C8
:109A20000FF42FEF4CF0E824106EE66E760E020174
:109A3000DB6FDC6BA7EC3DF0E552E7CF10F01200D6
:109A4000140E03017D6F7E6B0301020E7B6F090E06
:109A50007C6F11EC22F0F00E09010215106E116AF4
:109A6000126A136A400E101805E1115003E11250FA
:109A700001E1135001E0000C0F0E0215040DF3CFAD
:109A800039F40401F350106E116A140E105E000ECA
:109A9000115A10C01CF9116A126A136AD880280E74
:109AA0001054000E1154000E1254000E135401E213
:109AB000000C09011C5100080BE21C5103017D6FD1
:109AC0007E6B03011D0E7B6F090E7C6F11EC22F083
:109AD0000CC916F90DC917F909010C6B0D6B140EA1
:109AE0001BD9020E086F090E096F26EC38F0F3CF70
:109AF00018F9F4CF19F90901181F191F1C51000892
:109B000010E21C5109D91D0E086F090E096F26ECD1
:109B100038F0F3CF1AF9F4CF1BF909011A1F1B1FF4
:109B200002D01A6B1B6B040EF7D8180E086F090EC3
:109B3000096F26EC38F0F3CF00F9F4CF01F90901F1
:109B4000F350161902E10151171901E0000C04014C
:109B5000020E496F090E4A6FB2D804013A513B1107
:109B60000CE03AC4E9FF3BC4EAFF12C9EEFF13C997
:109B7000EEFF14C9EEFF15C9EEFF3CC4E9FF3DC47A
:109B8000EAFF060EE3D80EC9EEFF0FC9EEFF10C9BB
:109B9000EEFF11C9EEFF3EC4E9FF3FC4EAFF0BC967
:109BA000EFFF3951126E136A09011250045D106EF5
:109BB00013500559116E40C4E9FF41C4EAFF10C0BB
:109BC000EEFF11C0EDFF010C0401140E396F090105
:109BD000450E926F936B140E040145250901946F95
:109BE000000E040146210901956F0401D02B000EDF
:109BF000D123D0C496F9D1C497F90901986B400ECE
:109C0000996F640E9A6F44C49BF99C6B9D6BB1C2B3
:109C10009EF9B2C29FF9B3C2A0F9B4C2A1F942C47D
:109C2000E9FF43C4EAFF060E91D8EECFA2F9EECFCA
:109C3000A3F9EECFA4F9EFCFA5F90401920E496F75
:109C4000090E4A6F3CD8140E67D8920E086F090EA1
:109C5000096F26EC38F0F3CF9CF9F4CF9DF9140E80
:109C60000401452503018C6F000E04014621030108
:109C70008D6F03018B6B42C4E9FF43C4EAFF42C40A
:109C800089F343C48AF3E3EC24F0140E0301796FE3
:109C90007A6B0301920E776F090E786FCEEC20F08D
:109CA000F36AF46A12000401395147250301936FE6
:109CB000000E040148210301946F05EF26F027D818
:109CC000020E35D8020E38D8020E2BD8020E39D823
:109CD000040E2DD8040E30D8040E23D8040E31D82B
:109CE000060E25D8060E28D8060E1BD8060E29D833
:109CF0000A0E1DD80A0E20D80A0E13D80A0E03D851
:109D0000CDC9EFFF120022D8010EA6EF4EF049C4D4
:109D1000E9FF4AC4EAFF120003010A6F0B6B03015B
:109D2000120014D8E552E750EF6E87EF4EF00ED8D0
:109D3000EFCFCDF987EF4EF0E6DFEF50E66E87EF1D
:109D40004EF0E1DFCDC9EFFF87EF4EF0E926000EC0
:049D5000EA221200F1
:0C9D54001C0E03017D6F7E6B0301000EEE
:109D60007B6F090E7C6F11EC22F027EC23F00401CD
:109D7000000E8F6F090E906F2FD900C910F001C926
:109D800011F0126A136A010E101817E1115015E153
:109D9000125013E1135011E109010451146E156AB8
:109DA000060E14180AE1155008E10551166E176ADF
:109DB000040E161801E1175001E0000C3BD9020E09
:109DC000101809E1115007E1125005E1135003E1A9
:109DD00038D9EF6A12D02ED9010E10180AE11150AD
:109DE00008E1125006E1135004E1010E2AD9EF6E8A
:109DF00004D0020E26D9EF6E000C0201B151090108
:109E0000185D2EE10201B2510901195D29E102013B
:109E1000B35109011A5D24E10201B45109011B5D2E
:109E20001FE188C4E9FF89C4EAFF08C9EEFF09C938
:109E3000EEFF0AC9EEFF0BC9EEFF0CC9EEFF0DC91C
:109E4000EEFF88C4E9FF89C4EAFF060E04D90EC9F3
:109E5000EEFF0FC9EEFF10C9EEFF11C9EEFF010CB6
:109E6000000C0301010E756F58EC20F009011C6F06
:109E7000106E116A126A136AE868101807E111502F
:109E800005E1125003E1135001E1000C0301966B50
:109E9000976B1CC995F318EC26F0010E0901006FB1
:109EA000016B026B080E036F060E046F040E056F44
:109EB0008EC410F0116A126A136A010E101810E1B4
:109EC00011500EE112500CE113500AE1010E066F21
:109ED000076B12691369146915691669176913D03C
:109EE000020E066F076B8CC4E9FF8DC4EAFFEECF4C
:109EF00012F9EECF13F9EECF14F9EECF15F9EECF3C
:109F000016F9EFCF17F9B5C208F9B6C209F9B7C209
:109F10000AF9B8C20BF9B9C20CF9BAC20DF9B1C24B
:109F20000EF9B2C20FF9B3C210F9B4C211F97BD85D
:109F3000EF500E190201BB151BE175D8010E8BD82D
:109F4000EF5009010F190201BC1512E16CD8020E85
:109F500082D8EF50090110190201BD1509E163D83B
:109F6000030E79D8EF50090111190201BE1509E05D
:109F7000BFC218F9C0C219F9C1C21AF9C2C21BF98D
:109F800009D051D8EECF18F9EECF19F9EECF1AF962
:109F9000EFCF1BF90401000E8F6F090E906F1CD8D4
:109FA0001C0E03018C6F8D6B0301060E8B6F03017A
:109FB000120E896F090E8A6FE3EC24F01C0E030168
:109FC000796F7A6B0301000E776F090E786FCEEC14
:109FD00020F060EC25F0010C39D819D8F3CFEEFF52
:109FE00011C0EDFF33D8020E36D811D8020EF3CFD0
:109FF000EBFF030E11C0EBFF29D8060E2CD807D8B3
:10A00000060EF3CFEBFF070E11C0EBFF1200EECFF1
:10A0100002F3EDCF03F3F2EC37F0F3CF10F0F4CF0F
:10A0200011F026EF50F08CC4E9FF8DC4EAFF060E54
:10A030002BEF50F006C910F007C911F0126A136A2D
:10A0400012008AC4E9FF8BC4EAFF12008FC4E9FF43
:0EA0500090C4EAFF1200E926000EEA22120078
:02A05E000D01F2
:10A06000FF51020A25E0030A05E0010A01E012009F
:10A07000FF2B1200890E0101A56FA66B0101A36BD6
:10A08000A46B0101A16FA26BCCEC2CF00101FB6F62
:10A09000106E116A126A136AE868101807E111500D
:10A0A00005E1125003E1135001E112000D01FF2BF5
:10A0B000FBC1AEF147EC2EF0000901E112000101F5
:10A0C000060EB06F090E2ED9050EB06F090E2AD9F3
:10A0D000080EB06F090E26D9070EB06F090E22D9EF
:10A0E0000A0EB06F090E1ED9090EB06F090E1AD9EB
:10A0F0000C0EB06F090E16D90B0EB06F090E12D9E7
:10A100000E0EB06F090E0ED90D0EB06F090E0AD9E2
:10A11000100EB06F090E06D90F0EB06F090EB16F99
:10A1200066EC2EF0090109C910F00AC911F00907FF
:10A13000000E0A5B1050111071E00101110EFC6F4E
:10A14000090EFD6F8ED80101000EB06F090EEAD81E
:10A15000020EB06F090EE6D8010EB06F090EE2D8FC
:10A16000040EB06F090EDED8030EB06F090EB16F8A
:10A1700066EC2EF00901200E0119D4E10251D2E162
:10A18000010E0319CFE10451CDE10101110EFE6F63
:10A19000090EFF6F9FD80009C5E0FBC1A8F12CECA8
:10A1A0002DF0000903E135EC48F0F7D70901076B02
:10A1B000840E086F06C9A9F138EC2DF005C9A9F184
:10A1C00038EC2DF008C9A9F138EC2DF007C9A9F138
:10A1D00038EC2DF0A3D8A2D8B8D822D89FD8010146
:10A1E000200EB0D8B2D89AD80101060EABD8010122
:10A1F000600EA8D893D8B1C2A9F138EC2DF0B2C244
:10A20000A9F138EC2DF0B3C2A9F138EC2DF0B4C2AD
:10A21000A9F138EC2DF0DEEC2DF084D7B4EF2EF060
:10A220000101200E8FD80901216B100E215D17E26C
:10A23000470E21250201DB6FDC6BA7EC3DF0090125
:10A24000226FE8380F0B410F01017CD80F0E090176
:10A250002215410F010176D80901212BE6D78EEF97
:10A2600051F00101210EB06F090EB16F66EC2EF0B6
:10A27000090121512107000924E059D82239F00BA6
:10A28000236F210754D821C910F0116A126A136A8A
:10A29000D8801E0E1054000E1154000E1254000EE1
:10A2A0001354E6E323512211E66E0101FCC1E9FFDC
:10A2B000FDC1EAFFFC2B000EFD23E552E750EF6ED7
:10A2C000D7D70F0E0101EA6AFC25E96EFD51EA229B
:10A2D000EF6A12000901216B0F0E215D1EE2470E8D
:10A2E00021250201DB6FDC6BA7EC3DF00901226F39
:10A2F0000101FEC1E9FFFFC1EAFFFE2B000EFF23B3
:10A30000EFCF23F909012351225D01E0000C235115
:10A31000225D01E0010C212BDFD7010C0101A96BAB
:10A3200038EF2DF0B16F66EC2EF001011200010143
:10A33000220EB06F090EB16F66EC2EF0410E0901CE
:10A34000225F1200A96F38EF2DF0E8DF0101010E46
:0CA35000F9DFE4DFE3DFE2DF8EEF51F025
:04A35C000301356B59
:10A3600034813493A8EC1EF0B4EC5DF0C0EC2CF01A
:10A370001AEC12F0160E53D9010B02E1BDEC30F0CD
:10A380001200160E4CD9010B2EE09AEC23F00009B6
:10A3900022E103013451020B1EE10201DB6BDC6B95
:10A3A000A7EC3DF00201B16F010E39D90201B26F85
:10A3B000020E35D90201B36F030E31D90201B46F19
:10A3C000BB69BC6BBD6BBE6B0401C19503013481DD
:10A3D0003483AAEC30F0D8EC30F00401C1A103D0F2
:10A3E0000301349134930901BE6B03013551040A12
:10A3F00001E1EAD0070A01E1ADD0050A01E197D0F9
:10A40000010A01E181D0050A39E0070A31E0050AB5
:10A4100003E0010A01E0F9D00301BD0E876F090EC8
:10A42000886F0301360E856F030E866FB2EC23F042
:10A43000000901E1EAD00901010EBE6FF5D8105004
:10A4400011101210131003E10301020E57D0ECD8C3
:10A45000060E101801E0B5D0115001E0B2D0125034
:10A4600001E0AFD0135001E0ACD00301050E46D09F
:10A47000C1EC5DF0000901E1C8D0C5D00401400E77
:10A48000406F030E416F0401BD0E3E6F090E3F6F1A
:10A490000401360E3C6F030E3D6F0401B90E3A6F96
:10A4A000090E3B6F20EC4DF000092BE00901010E75
:10A4B000BE6FBAD8101809E1115007E1125005E13A
:10A4C000135003E10301030E19D0AED8060E101885
:10A4D00009E1115007E1125005E1135003E10301B6
:10A4E000060E0CD0A1D8110E10180AE1115008E187
:10A4F000125006E1135004E10301070E356F85D0B9
:10A50000BE6B27EC23F07FD040C3BAF141C3BBF14F
:10A510000101B90EB86F090EB96F0101360EB66FA1
:10A52000030EB76FBCEC2EF000096FE06CD040C397
:10A5300086F041C387F00001B90E846F090E856F64
:10A540000001360E826F030E836F1EEC17F00009B8
:10A550005CE059D0356B40C310F041C311F0126A72
:10A56000136AD880290E1054000E1154000E125494
:10A57000000E135426E30301640EEE6F030EEF6F1B
:10A580000301620EEC6F030EED6F0301400EEA6FE4
:10A59000030EEB6F0301420EE86F030EE96F030138
:10A5A000BD0EE66F090EE76FC4EC55F0000909E037
:10A5B000080E0901BD5D05E1010EBE6F0301040E29
:10A5C000356F27EC23F021D00301010E746F1FECCF
:10A5D00020F000091AE064C3F8F365C3F9F362C31D
:10A5E000F6F363C3F7F340C3F5F30301420EF36FD1
:10A5F000030EF46F0301F26B0301360EF06F030ECE
:10A60000F16F3EEC56F00301356B35EC48F0090173
:10A61000BE5101E0E8D6F7EC15F0FAEF1FF00201A9
:10A62000DB6FDC6BA7EF3DF0BDC910F0116A126A59
:04A63000136A120097
:0CA634009398939A09014F6B030E4F5D41
:10A640000EE223D9EE6AED6A20D9020E45D91DD952
:10A65000040E42D91AD9060E3FD94F2BEFD703016A
:10A66000E06B0301FC6BFD6B0301FE6BFF6B1200E3
:10A670009250010B18E0FEC310F039D914E180505C
:10A68000010B1CD934D902E1000E01D0010E005D8E
:10A690000AE00301FE810901005103E00301FC818E
:10A6A00002D00301FC919250020B1EE0FEC310F099
:10A6B000126A136A020ED4D817E18050020B01E02F
:10A6C000010EFCD8020ECCD802E1000E01D0010E22
:10A6D000005D0AE00301FE830901005103E003016C
:10A6E000FC8302D00301FC939250040B1EE0FEC3D6
:10A6F00010F0126A136A040EB3D817E18050040BED
:10A7000001E0010EDBD8040EABD802E1000E01D04F
:10A71000010E005D0AE00301FE850901005103E01E
:10A720000301FC8512000301FC9512000901416B35
:10A73000C6C410F0DCD834E0C4C4A8F12CEC2DF071
:10A7400000092EE0C2D8D3D80BE00301FE91A8D8AF
:10A75000300E8FD8CCD802E1300E01D0310EA8D8FF
:10A76000B4D8020E7DD80CE00301FE9399D8310EC7
:10A7700080D8020E75D802E1300E01D0310E98D883
:10A78000A4D8040E6DD80CE00301FE9589D8320ED2
:10A7900070D8040E65D802E1300E01D0310E88D891
:10A7A000090141511200F36AF46A12000301E251F7
:10A7B000010A0BE0010A01E012009398E351E8B0AE
:10A7C0008A88E8B008D08A981200939AE351E8B0DA
:10A7D0008A8AE8A08A9A12000301E451050A2EE051
:10A7E000010A25E0070A1CE0010A13E0030A0AE057
:10A7F000010A01E01200E551E8B08980E8B023D0F9
:10A8000089901200E551E8B08982E8B01CD08992A5
:10A810001200E551E8B08984E8B015D0899412009F
:10A82000E551E8B08B84E8B00ED08B941200E5516E
:10A83000E8B08B82E8B007D08B921200E551E8B007
:10A840008B80E8A08B9012008A50200B01E0010E53
:10A85000E824106E8A50100B01E0010E1010120057
:10A860001016116A126A136A105011101210131088
:10A87000120038D83D0EA96F38EC2DF0FCC310F053
:10A88000FDC311F0126A136A12004F51080DF3CF85
:10A89000E9FFF4CFEAFFC80EE926030EEA22120010
:10A8A000090141810101780E1DD8340E72EF54F078
:10A8B000010118D83B0EA96F38EF2DF00901006F88
:10A8C000FCC310F0126A136A1200FEC310F0FFC33B
:10A8D00011F0126A136A1200E926000EEA22EE6AEB
:10A8E000ED6A1200A96F38EC2DF001011200010E83
:04A8F00030EF54F001
:0CA8F4000401C66B0401C76B0A0E0301CF
:10A90000286F296B0301000E266F090E276FFBECE1
:10A9100039F00101A56BA66B0101000EA36F090EB2
:10A92000A46F7D0E1ED9106E116E106A10C0E6FF66
:10A93000E66E7C0E16D9E552E7CF11F0E552E7CF6F
:10A9400010F001011010A16F11C0A2F1CCEC2CF09D
:10A950000401C46F106E116A126A136AE868101855
:10A9600005E1115003E1125001E1135012000401FE
:10A97000C751020A24E0030A10E0010A01E01200B4
:10A98000C4C4AEF147EC2EF000094FE0C5D802E197
:10A990000401C66B0401010E10D0C6C410F0EFD83C
:10A9A00044E0E4D842E0EE0EE66E960EE66E000E4F
:10A9B00095D8DEEC2DF00401020EC76F12000901DC
:10A9C000406BC4C4AEF147EC2EF0000905E0A4D8FA
:10A9D0002CE10401C66B12000401C8510401A15D01
:10A9E000106E050E105C1BE3A1C4C8F40401C90776
:10A9F00010E1140EC96FC6C410F0C1D80AE0B6D871
:10AA000008E0E70EE66E960EE66E000E67D80901C6
:10AA100040810CD80901401354D80901401340C9A2
:10AA200010F0ADD802E0DEEC2DF012000901416B10
:10AA3000426B42C910F0116A126A136A010E105C6F
:10AA4000000E1158000E1258000E135838E209017A
:10AA50004251EA6A090FE96E040EEA22EFCF10F0C4
:10AA60004251EA6A080FE96E040EEA22EF50105CC8
:10AA700024E042C90EF413EC4CF00901436FC6C444
:10AA800010F065D8E4E072D8E2E0090141810101EB
:10AA90006C0E72D80101330E6FD8340E09014225B5
:10AAA00001016AD801013D0E67D843C9A9F138EC0C
:10AAB0002DF001013B0E60D8CAD7422BBAD74151C5
:10AAC0001200870E4ED8020802E19BEF36F0870E87
:10AAD00048D8010802E196EF53F0000CE66E000E34
:10AAE000E66E090EE66E9DEC58F0106E050EE15E06
:10AAF0001050000EE66E090EE66EB6EC58F0E55208
:10AB0000E552F3CFACF1F4CFADF10101000EAA6F25
:10AB1000090EAB6F6BEF2DF0020E0101B46FB56B38
:10AB20000101000EB26F090EB36F80EC2EF0B4EC91
:10AB30002EF00301C60E116F040E126F0301000EFA
:10AB40000F6F090E106F18EC39F000091200010E9A
:10AB50001016116A126A136A105011101210131095
:10AB600012000201DB6FDC6BA7EF3DF0C4C4A8F15B
:10AB70002CEC2DF000091200A96F38EF2DF0116AAE
:08AB8000126A136AA7EF55F0F9
:08AB8800080E03017D6F7E6BD6
:10AB90000301000E7B6F090E7C6F11EC22F0080E92
:10ABA000106E18D9E850EF5E15D9EF5003017D6F94
:10ABB0007E6BE8C37BF3E9C37CF311EC22F002C99E
:10ABC0002AF903C92BF90901026B036B080E030173
:10ABD0000A6F0B6B0301000E086F090E096F26EC5C
:10ABE00038F0F3CF2CF9F4CF2DF909012C1F2D1FCC
:10ABF000F1D8EF5003010A6F0B6BE8C308F3E9C308
:10AC000009F326EC38F0F3CF2EF9F4CF2FF9090130
:10AC10002E1F2F1F040E03010A6F0B6B03012C0E56
:10AC2000086F090E096F26EC38F0F3CF28F9F4CF3E
:10AC300029F90301000EFA6F090EFB6F96D8E6C3DF
:10AC4000E9FFE7C3EAFF00C9EFFFECC3E9FFEDC38B
:10AC5000EAFF04C9EEFF05C9EDFFEEC3E9FFEFC34C
:10AC6000EAFF06C9EEFF07C9EDFF09012A512819BD
:10AC700002E12B51291901E0000C010C0301010E26
:10AC8000756F58EC20F009012A6F106E116A126A74
:10AC9000136AE868101807E1115005E1125003E14A
:10ACA000135001E11200140E0301966F976B2AC92D
:10ACB00095F318EC26F00301F551106E7DD810C005
:10ACC00028F911C029F90901016BF2C300F9026BDF
:10ACD000036BF6C304F9F7C305F9F8C306F9F9C322
:10ACE00007F90301F551E66EE66AF3C3E6FFF4C324
:10ACF000E6FF080EE66E090EE66E22EC58F0106EC6
:10AD0000060EE15E10500301000EFA6F090EFB6F94
:10AD10002CD828C90AF329C90BF30301000E086FC8
:10AD2000090E096F26EC38F0F3CF02F9F4CF03F9DE
:10AD3000F5C310F041D810C045F411C046F4040129
:10AD4000010E446FF0C342F4F1C343F4E4EC4DF060
:10AD500028C979F329C97AF30301000E776F090E28
:10AD6000786FCEEC20F060EF25F039D8040E15D8BE
:10AD7000040EF3CFEBFF050E29D8060E0ED8060EF3
:10AD8000F3CFEBFF070E22D8020E07D8020EF3CF47
:10AD9000EBFF030E11C0EBFF1200E926000EEA22C2
:10ADA000EECF02F3EDCF03F3F2EC37F0F3CF10F078
:10ADB000F4CF11F0EFEF56F0116A126A136A080E21
:10ADC0001026000E112212221322120011C0EBFFD6
:10ADD000EFEF56F0EAC3E9FFEBC3EAFF1200FAC354
:08ADE000E9FFFBC3EAFF1200CA
:08ADE800FF0EE3CFEAFFE55284
:10ADF000FF0EE3CFE9FFE552E66AE66AD9CFE6FF48
:10AE0000DACFE6FFFC0EE124D96EFF0EE220DA6E07
:10AE1000E66AE66AE66A200EEF5C06E0090EEF5C81
:10AE200003E0EF6603D03FD0EE50F5D72D0EEF5C78
:10AE300003E1FF0EE32A03D02B0EEF5C01E1EE509D
:10AE40002F0EEF6424D03A0EEF6021D0D890F90E87
:10AE5000E336FA0EE336FD0EDECFE3FFFE0EDDCF66
:10AE6000E3FFD890F90EE336FA0EE336D890F90EE8
:10AE7000E336FA0EE336FD0EE350DE26FE0EE35017
:10AE8000DD22300EEE5CDE26000EDD22D9D7FF0E6D
:10AE9000E3CFE8FFE85207E0F90EE31EE32AFA0EDB
:10AEA000D8B4E306E31EE552E552E552FF0EE3CFC8
:10AEB000DAFFE552FF0EE3CFD9FFE552E1CFE9FF1C
:10AEC000E2CFEAFFED52ED52EECFF3FFEFCFF4FF0A
:10AED0001200D9CFE6FFDACFE6FFFA0EE3CFD9FFB3
:10AEE000FB0EE3CFDAFFFD0EE35209E72D0EDE6E17
:10AEF000FC0EE31EE32AFD0ED8B4E306E31EE65281
:10AF0000E652E652FD0EE124E76EFF0EE220E46E0B
:10AF1000E652F70EE3CFE6FFF70EE3CFE6FFD9ECFC
:10AF200057F0F90EE124E96EFF0EE220EA6EC9EC5B
:10AF300057F00AE1C6EC57F009E1C9EC57F008E117
:10AF4000C6EC57F007E108D0D4EC57F0CFEC57F03F
:10AF5000D4EC57F0CFEC57F0D4EC57F0DE6AF90E92
:10AF6000E126FF0EE222FF0EE3CFDAFFE552FF0EED
:10AF7000E3CFD9FFE552FC0EE124E96EFF0EE2209B
:10AF8000EA6EEECFF3FFEFCFF4FF1200EF380F0BB6
:10AF90001200EF500F0B02E1EE52D8841200EF388E
:10AFA0000F0B300FDE6E1200EE500F0B300FDE6E07
:10AFB0001200FC0EE3CFE9FFFD0EE3CFEAFF100E17
:10AFC000E66EEE6AEE6AEF6AD890FD0EE336FE0E8C
:10AFD000E336ED36ED36EF36FF0EE30609E0FAEC28
:10AFE00057F0EE52FAEC57F0EE52FAEC57F0EDD77C
:10AFF000E56E1200030EEF24E8B6EF6E300EEF247C
:06B00000E8BEEF6E000C3B
:0AB00600FB0EE3CFF6FFFC0EE3CFD4
:10B01000F7FFFD0EE3CFF8FFFE0EE3CFE9FFFF0ED3
:10B02000E3CFEAFFF90EE35003E1FA0EE35009E043
:10B03000F90EE30602E2FA0EE3060900F550EE5CB3
:10B04000F1E01200D9CFE6FFDACFE6FFFA0EE3CF48
:10B05000D9FFFB0EE3CFDAFFFC0EE3CFE9FFFD0ED5
:10B06000E3CFEAFFE9CFF3FFEACFF4FFF80EE350B6
:10B0700003E1F90EE35008E0F80EE30602E2F90EF0
:10B08000E306DECFEEFFF2D7FF0EE3CFDAFFE552A5
:10B09000FF0EE3CFD9FFE5521200FE0EE3CFE9FF2A
:10B0A000FF0EE3CFEAFFE9CFF3FFEACFF4FFFB0E99
:10B0B000E35003E1FC0EE35009E0FB0EE30602E27D
:10B0C000FC0EE306FD0EE350EE6EF1D71200D9CF71
:10B0D000E6FFDACFE6FFFA0EE3CFD9FFFB0EE3CFB0
:10B0E000DAFFFC0EE3CFE9FFFD0EE3CFEAFFDE500F
:10B0F000EF5C02E1EE66FBD7F36EFF0EE3CFDAFF03
:10B10000E552FF0EE3CFD9FFE552F3501200FB0EDC
:10B11000E3CFF6FFFC0EE3CFF7FFFD0EE3CFF8FF22
:10B12000FE0EE3CFE9FFFF0EE3CFEAFF0900F55083
:10B13000EF5C02E1EE66FAD71200FB0EE3CFF6FFFA
:10B14000FC0EE3CFF7FFFD0EE3CFF8FFFE0EE3CFDB
:10B15000E9FFFF0EE3CFEAFFE9CFF3FFEACFF4FF09
:10B160000900F5CFEFFFEE66FBD71200FE0EE3CF2E
:10B17000E9FFFF0EE3CFEAFFF36AF46AEE5203E061
:10B18000F34AF42AFBD71200D9CFE6FFDACFE6FF65
:10B19000FA0EE3CFD9FFFB0EE3CFDAFFFC0EE3CFCD
:10B1A000E9FFFD0EE3CFEAFFE9CFF3FFEACFF4FFBB
:10B1B000F80EE35003E1F90EE3500BE0F80EE3065E
:10B1C00002E2F90EE306DECFEFFFEE66F1D7DD52C5
:10B1D000EFD7FF0EE3CFDAFFE552FF0EE3CFD9FF43
:10B1E000E5521200FE0EE3CFE9FFFF0EE3CFEAFFC8
:10B1F000E9CFF3FFEACFF4FF610EEF5C05E67B0ECB
:0EB20000EF5C02E7DF0EEF16EE52F6E11200F1
:02B20E005CC41E
:10B21000B8F40401B76B0401080EB66F87EF5FF056
:10B220005EC4A4F95FC4A5F9C750040B01E0010E88
:10B23000E0D8FAE1C580C5B0FED7A1B6010C5DC467
:10B24000BAF4DCD801E0010CC750040B01E0010E98
:10B25000D0D8FAE1C5BC19D0A5C9BAF4CFD801E05D
:10B26000010CC750040B01E0010EC3D8FAE1A4C9D8
:10B27000BAF4C4D801E0010CC750040B01E0010E80
:10B28000B8D8FAE1C5AC000C020C020C61C45EF443
:10B2900062C45FF460C45DF4C3DF0901086FE85065
:10B2A00005E173D80901086FE85002E00851120067
:10B2B000C750040B01E0010E9CD8FAE1C580C5B06F
:10B2C000FED7A1B6010C040160290401BA6F96D81B
:10B2D00001E0010CC750040B01E0010E8AD8FAE12D
:10B2E000C5AC000C020CC750040B01E0010E81D864
:10B2F000FAE163C4BAF482D801E0010CC750040B30
:10B3000001E0010E76D8FAE1C5AC000C020CC75082
:10B31000040B01E0010E6DD8FAE1C584C5B4FED777
:10B32000000C0401010EB96F96EC5FF0C9501200D9
:10B330000401B96B96EC5FF0C584C5B4FED7000C70
:10B3400065C461F466C462F464C460F49FDF0901FB
:10B35000006FE85018E1040169516907000910E025
:10B360000401010EB96F96EC5FF0040167C4E9FFB8
:10B3700068C4EAFF672B000E6823C9CFEFFFEBD745
:10B38000D7DF0901006F00511200C750040B01E024
:10B39000010E2FD8FAE1C584C5B4FED7A1B6010CC1
:10B3A000000CC750040B01E0010E23D8FAE1C58060
:10B3B000C5B0FED7A1B6010C6AC4BAF41FD801E02B
:10B3C000010CC750040B01E0010E13D8FAE1A1B63D
:10B3D000010CC5BC03D00901A86B03D00901040E00
:10B3E000A86FC584C5B4FED7A1B6010C0901A85148
:10B3F0001200106E1F0EC51410101200ADEC5FF09D
:04B40000000912002D
:0CB4040012000901406B416B446B91C4C5
:10B4100053FF92C454FF9BEC2BF00901456F400E83
:10B42000426F0F01420E476F090E486F0F01000E69
:10B43000456F090E466F91C4E9FF92C4EAFFEF50D1
:10B440000F01446F62EC29F00901436F442B476BF5
:10B450006C0E005D08E10151750A02E0050A1EE16B
:10B46000010E476F1BD06D0E005D18E145C910F04D
:10B47000116A98D805E0ADD86F0A02E1010E476F56
:10B48000A8D86C0A0BE1010E476F91C4E9FF92C482
:10B49000EAFF090EE926000EEA22EF88475116E17D
:10B4A00045C9A4F342510301A26FA36B000EA2276A
:10B4B000090EA3230301000EA06F090EA16F62EC19
:10B4C00006F0F35009014013F45041134351A7E132
:10B4D00070D8020E86D801E012006BD8040E81D815
:10B4E00004E0E2EC3DF036EF3EF063D8080E79D888
:10B4F00002E08AEF3EF05DD8100E73D802E0CDEF87
:10B500003EF057D8106A010E11164CD802E0C7EF72
:10B510003FF04FD8106A200E111644D802E001EF18
:10B5200040F047D8106A080E11163CD802E0D2EF5E
:10B5300042F03FD8106A100E111634D802E05BECCE
:10B5400043F012003DD8020EE926000EEA22EFCFAA
:10B5500000F936D8030EE926000EEA22EFCF01F9F2
:10B560002FD8EECF02F9EDCF03F997C404F998C4B0
:10B5700005F997C4E9FF98C4EAFFEF6A95C453FF41
:10B5800096C454FF9BEC2BF00901066F0301000EDB
:10B59000A56F090EA66FC9EC0DF002C9F3FF03C930
:10B5A000F4FF1200126A136A1050111012101310D7
:10B5B000120040C910F041C911F0126A136A12005A
:10B5C00095C4E9FF96C4EAFF040EE926000EEA22BC
:10B5D00012004251EA6A000FE96E090EEA22EF50AA
:0AB5E00012001016116AD2EF5AF0A3
:06B5EA000D0A50726573AA
:10B5F0007320616E79206B657920666F7220436FCE
:10B600006E66696775726174696F6E206D656E75BF
:10B610002E000D0A52756E6E696E67204170706C57
:10B6200069636174696F6E2C204950206164647293
:10B630006573733A2000444843502F476C65616E30
:10B64000696E672E2E2E000D0A0D0A0D4D6F647463
:10B65000726F6E69782057656220536572766572E5
:10B660000D0A0D0A09313A204368616E6765204270
:10B670006F6172642073657269616C206E756D62B2
:10B6800065722E0D0A09323A204368616E676520A3
:10B6900064656661756C74204950206164647265EC
:10B6A00073732E0D0A09333A204368616E67652073
:10B6B00064656661756C7420676174657761792073
:10B6C000616464726573732E0D0A09343A2043680D
:10B6D000616E67652064656661756C742073756260
:10B6E0006E6574206D61736B2E0D0A09353A204525
:10B6F0006E61626C652044484350202620495020EA
:10B70000476C65616E696E672E0D0A09363A2044F2
:10B71000697361626C65204448435020262049507B
:10B7200020476C65616E696E672E0D0A09373A20F5
:10B73000446F776E6C6F61642046696C6520537945
:10B740007374656D20496D6167652E0D0A09383A7D
:10B750002053617665202620517569742E0D0A0DDF
:10B760000A456E7465722061206D656E7520636890
:10B770006F6963652028312D38293A20000D0A4968
:10B780006E76616C696420696E7075742072656391
:10B790006569766564202D20496E7075742069672F
:10B7A0006E6F7265642E0D0A507265737320616E40
:10B7B00079206B657920746F20636F6E74696E7584
:0CB7C000652E2E2E0D0A001B5B324A0085
:04B7CC00040E6C6E8D
:10B7D000100E6B6EA39AA39812006C8A6B886B8E06
:10B7E000A38A0201AD8F12006C9A6B986B9EA39A8C
:10B7F000A3980201AD9F120002018A6B8AC288F2EF
:10B800008AC289F2906B90C28EF290C28FF21200BF
:10B81000060E6B1402E06B986B88A4AA17D0020185
:10B820009151905D0FE08E51EA6A8C25E96E8D5141
:10B83000EA226ECFEFFF8E2B91518E5D01E18E6B70
:10B84000902BEBD7AD896E50A86EE7D7120002019E
:10B850008A5103E1AD93A3981200895198D8EF5013
:10B860006D6E892B8B51895D01E1896B8A0712000E
:10B870000201ADB312D08A5110E0895188D8EFCFC0
:10B8800004F9892B8B51895D01E1896B8A07F29E4E
:10B8900004C96DFFAD83A388F28E1200020190519E
:10B8A0000EE08F51EA6A8C25E96E8D51EA22EFCFC6
:10B8B00000F98F2B91518F5D01E18F6B900709018A
:10B8C0000051120002018B518A5D03E135EC48F012
:10B8D000F9D7F29EADB305D0A8C46DFFAD83A388A0
:10B8E0000AD0885154D8A8C4EFFF882B8B51885DAB
:10B8F00001E1886B8A2BF28E12000401A9519F0886
:10B9000005E2A9390F0B0F0B570F04D0A9390F0B04
:10B910000F0B300F0401A86FD5DF0F0E0401A9151E
:10B92000090804E20F0EA915570F03D00F0EA91531
:10B93000300F0401A86F62EF5CF00401AAC4E9FFB4
:10B94000ABC4EAFFAA2B000EAB23EFCF00F9EF50F8
:10B9500006E000C9A8F4B6DF35EC48F0EED71200D7
:10B960000401ACC4F6FFAC2BADC4F7FF000EAD2351
:10B97000AEC4F8FFAE230800F5CF00F9F55006E09D
:10B9800000C9A8F49FDF35EC48F0EAD71200EA6A54
:0AB990008625E96E8751EA221200B5
:06B99A00040EAC6E100E5D
:10B9A000AB6E9D9A9D981200AC8AAB88AB8E9D8A37
:10B9B0000201AC8F1200AC9AAB98AB9E9D9A9D98F9
:10B9C0000201AC9F120002017E6B7EC27CF27EC23D
:10B9D0007DF2846B84C282F284C283F21200060E6E
:10B9E000AB1402E0AB98AB889EAA17D00201855138
:10B9F000845D0FE08251EA6A8025E96E8151EA2276
:10BA0000AECFEFFF822B8551825D01E1826B842BEB
:10BA1000EBD7AC89AE50A86EE7D7120002017E5179
:10BA200003E1AC939D9812007D5198D8EF50AD6E14
:10BA30007D2B7F517D5D01E17D6B7E071200020150
:10BA4000ACB312D07E5110E07D5188D8EFCF04F90D
:10BA50007D2B7F517D5D01E17D6B7E07F29E04C9E8
:10BA6000ADFFAC839D88F28E1200020184510EE07E
:10BA70008351EA6A8025E96E8151EA22EFCFA4F969
:10BA8000832B8551835D01E1836B84070901A451F8
:10BA9000120002017F517E5D03E135EC48F0F9D7D9
:10BAA000F29EACB305D0AFC4ADFFAC839D880AD085
:10BAB0007C5154D8AFC4EFFF7C2B7F517C5D01E1FA
:10BAC0007C6B7E2BF28E12000401B0519F0805E2C0
:10BAD000B0390F0B0F0B570F04D0B0390F0B0F0BF2
:10BAE000300F0401AF6FD5DF0F0E0401B015090848
:10BAF00004E20F0EB015570F03D00F0EB015300F24
:10BB00000401AF6F49EF5DF00401B1C4E9FFB2C4B5
:10BB1000EAFFB12B000EB223EFCF08F9EF5006E099
:10BB200008C9AFF4B6DF35EC48F0EED712000401D7
:10BB3000B3C4F6FFB32BB4C4F7FF000EB423B5C4EF
:10BB4000F8FFB5230800F5CF00F9F55006E000C96D
:10BB5000AFF49FDF35EC48F0EAD71200EA6A7A25A5
:08BB6000E96E7B51EA2212009C
:08BB680004014B6B4C694D69AF
:10BB70004E694F6950695169526B536B546B556BE9
:10BB8000120004014B5130E10401270E8A6F090EA7
:10BB90008B6F04011D0E886F090E896FAAEC4EF0A1
:10BBA000000931E027C910F0116A126A136A1050B7
:10BBB00011101210131015E11DC94CF41EC94DF4DB
:10BBC0001FC94EF420C94FF421C950F422C951F4C1
:10BBD00023C952F424C953F425C954F426C955F491
:10BBE000010C0401010E4B6F04018E6B04011D0E4C
:10BBF0008C6F090E8D6F31EC4FF0000903E00401EA
:10BC00004B6B010C000C010C56C4E9FF57C4EAFF52
:10BC1000EECF23F9EECF24F9EECF25F9EFCF26F9B9
:10BC20000401010E8E6F04011D0E8C6F090E8D6FC5
:10BC300031EF4FF058C4E9FF59C4EAFF04015251F3
:10BC4000EE1808E15351EE1805E15451EE1802E1E7
:10BC50005551EE1814E00201BF510401525D20E17C
:10BC60000201C0510401535D1BE10201C1510401F5
:10BC7000545D16E10201C2510401555D11E15AC43F
:10BC8000E9FF5BC4EAFF4CC4EEFF4DC4EEFF4EC4B7
:10BC9000EEFF4FC4EEFF50C4EEFF51C4EEFF010CA7
:02BCA000000C96
:0EBCA2000401996B120012000201966B96C20B
:10BCB00094F296C295F29C6B9CC29AF29CC29BF243
:10BCC000120002019C510EE09B51EA6A9825E96E30
:10BCD0009951EA22EFCF00F99B2B9D519B5D01E129
:10BCE0009B6B9C0709010051120002019451EA6A02
:10BCF0009225E96E9351EA229AC4EFFF942B975153
:10BD0000945D01E1946B962B120004019B519F08F6
:10BD100005E29B390F0B0F0B570F04D09B390F0B0C
:10BD20000F0B300F04019A6FE0DF0F0E04019B151B
:10BD3000090804E20F0E9B15570F03D00F0E9B1539
:10BD4000300F04019A6F75EF5EF004019CC4E9FFA7
:10BD50009DC4EAFF9C2B000E9D23EFCF00F9EF500E
:10BD600006E000C99AF4C1DF35EC48F0EED71200C6
:10BD700004019EC4F6FF9E2B9FC4F7FF000E9F2375
:10BD8000A0C4F8FFA0230800F5CF00F9F55006E0A5
:0EBD900000C99AF4AADF35EC48F0EAD7120099
:02BD9E005458F7
:10BDA000540048544D00434C4100435353004A5300
:10BDB000000047494600434749004A5047004A416E
:10BDC000520057415600545854005A5458005A488B
:10BDD00054005A434C005A4353005A4A53004854A3
:10BDE00054502F312E3020323030204F4B00436FD3
:10BDF0006E74656E742D747970653A2000436F6EB1
:10BE000074656E742D456E636F64696E673A206762
:10BE10007A69700D0A00457870697265733A20304E
:10BE20000D0A0043616368652D436F6E74726F6C19
:10BE30003A206D61782D6167653D3330302C206D7F
:10BE40007573742D726576616C69646174650D0A31
:10BE50000047455400494E4445582E48544D004C27
:09BE60004F47494E2E43474900AB
:01BE690000D8
:06BE6A002A0EF66E080E20
:10BE7000F76E000EF86E00010900F550FB6F090027
:10BE8000F550FC6F03E1FB6701D03DD00900F55090
:10BE9000F66F0900F550F76F0900F550F86F0900CB
:10BEA0000900F550E96E0900F550EA6E0900090035
:10BEB0000900F550F96F0900F550FA6F0900090003
:10BEC000F6CFFDF0F7CFFEF0F8CFFFF0F6C0F6FFAB
:10BED000F7C0F7FFF8C0F8FF0001F95302E1FA5389
:10BEE00007E00900F550EE6EF907F8E2FA07F9D716
:10BEF000FDC0F6FFFEC0F7FFFFC0F8FF0001FB0723
:08BF0000000EFC5BBFD712002C
:08BF0800C6BEC69E12003F0EEA
:10BF1000C716C66AC56A0401B651C612B751C71220
:10BF200094869488C68AB8C4C8FF1200C586C7B074
:10BF300003D035EC48F0FBD7C5B6FED70401B951A4
:10BF400002E0000E01D0010EE8B0C58AE8A0C59A53
:10BF5000C588C5B8FED7C9501200BAC4C9FFC6BE4D
:10BF6000FF0CC7B0FED7000CBBC4C9FFC6BE010C96
:10BF7000C7B0FED7C750040B01E0010E106E1F0EB4
:08BF8000C5141010F7E1000CDC
:08BF880041424344454647488D
:10BF9000494A4B4C4D4E4F50515253545556575899
:10BFA000595A6162636465666768696A6B6C6D6E35
:10BFB0006F707172737475767778797A3031323345
:09BFC0003435363738392B2F00D7
:06BFCA000401CA51CA0780
:10BFD000000907E009010D0E8D6F8D51F6E08D0708
:10BFE000FCD712000401CB51CB07000908E0080E72
:10BFF000E66E40EC60F0E55235EC48F0F3D7120005
:10C00000636865636B65640064697361626C656431
:10C01000003C212D2D002D2D3E006F6E006F6666B9
:10C02000004E6F7420496D706C656D656E7465644B
:01C03000000F
:0EC03200036A026A100EE76ED89006360736D3
:10C04000023603360B50025C0C50035805E30B50CC
:0EC05000025E0C50035A062AE72EF0D71200AB
:02C05E000401DB
:10C06000A16BA26BA36BA46BA56BA66B580ED66ECF
:10C070009E0ED76E010ED56ED58EF284F28A120016
:10C08000FF0EE350246E480E01D04C0EE76EE72EF3
:10C09000FED7E76AE72EFED7242EF7D7000012005E
:10C0A00056332E313000415554484F52495A41546D
:0CC0B000494F4E3A2042415349432000C2
:04C0BC001EEE00F084
:10C0C0002EEE00F0F86A0F9C35EC5FF04FEC48F074
:04C0D000FDD7120086
:0CC0D4000301FC6BFD6BFE6BFF6B1200A8
:02C0E00012004C
:0EC0E20000EE00F00F0EEE6AEA62FDD71200CB
:06C0F00056322E3531002E
:02C0F600000444
:08C0F800BA9500A3950087959D
:10C10000006F95004F95002E9500EF9400D294009B
:04C11000FF0000002C
:02C11400000029
:02C11600000027
:08C11800C79400BD9400A99436
:10C1200000A09400909400869400BD94007B94003D
:10C13000629400559400C79400C79400BD9400A970
:10C140009400A094009094002E9400079400A6936D
:01C1500000EE
:0FC151007C2424247D72737475767778797A7BD9
:10C16000242424242424243E3F4041424344454681
:10C170004748494A4B4C4D4E4F50515253545556D7
:10C180005724242424242458595A5B5C5D5E5F6044
:10C190006162636465666768696A6B6C6D6E6F7017
:02C1A00071002C
:0EC1A200D89600D39600CE9600C99600C4969B
:10C1B00000BF9600BA9600AE96009696008696004E
:10C1C0007C96007596005F96004A96002F96002494
:0BC1D00096000C9600D59500CC950061
:03C1DB000200144B
:02C1DE0001005E
:02C1E000FF005E
:02C1E200FF005C
:02C1E400FFFF5B
:0AC1E600BE0F00BB0F00B80F00747D
:05C1F0000F00710F00BB
:020000040030CA
:0100010046B8
:010002000EEF
:010003000EEE
:010005008377
:010006008178
:01000800FFF8
:010009008076
:01000A00FFF6
:01000B008074
:01000C00FFF4
:01000D0000F2
:0200000400F00A
:100000000A0100010004A3000000FF0000000A0133
:10001000000104012803010A0100010A010001078F
:10002000010700FFFFFFFFFFFFFF000000000000CF
:1000300000032E000061646D696E0000000070779F
:10004000000000000000004D58424F415244202063
:10005000202020202020000A0100016BD300000096
:10006000000001000201000000000000000000008C
:100070000000350050005000000000006CD300006C
:100080000000000000000000000000000000000070
:100090000000000000000000000000000000000060
:1000A0000000000000000000000000000000000050
:1000B0000000000000000000000000000000000040
:1000C0000000000000000000000000000000000030
:1000D0000000000000000000000000000000000020
:1000E0000000000000000000000000000000000010
:1000F0000000000000000000000000000000000000
:10010000646464640000000000000000000000005F
:0C0110006DD3016ED300FFFF1122339964
:00000001FF
